S00F0000746563776172652E737265632A
S31508002800000001208D220108055C00080B5C000809
S31508002810115C0008175C00081D5C00080000000039
S31508002820000000000000000000000000E11A010896
S31508002830235C000800000000311D0108315C000817
S31508002840DD220108DD220108DD220108DD2201085A
S31508002850DD220108DD220108DD220108DD2201084A
S31508002860DD220108DD220108DD220108DD2201083A
S315080028704D5C0008615C0008DD220108DD220108C4
S31508002880DD220108DD220108755C0008895C000864
S315080028909D5C0008B15C0008C55C0008DD220108E3
S315080028A0DD220108DD220108DD220108DD220108FA
S315080028B0DD2201080000000000000000DD220108FA
S315080028C0DD2201080000000000000000D95C0008B5
S315080028D000000000DD220108DD22010800000000DA
S315080028E0DD220108DD2201080000000000000000CA
S315080028F000000000000000000000000000000000CA
S31508002900000000000000000000000000DD220108B1
S315080029100000000000000000DD220108DD22010899
S31508002920DD220108DD220108ED5C0008DD22010830
S31508002930DD22010800000000000000000000000081
S31508002940DD220108DD220108DD220108DD22010859
S31508002950DD220108DD220108DD220108DD22010849
S31508002960DD220108DD220108DD2201080000000041
S31508002970DD220108DD220108000000000000000039
S31508002980DD220108DD220108DD2201082255AAEE12
S3150800299010B5054C237833B9044B13B10448AFF38B
S315080029A000800123237010BD4001002000000000B4
S315080029B0DC24010808B5034B1BB103490348AFF3F0
S315080029C0008008BD0000000044010020DC24010846
S315080029D081F0004102E000BF83F0004330B54FEAC2
S315080029E041044FEA430594EA050F08BF90EA020F2F
S315080029F01FBF54EA000C55EA020C7FEA645C7FEAC2
S31508002A00655C00F0E2804FEA5454D4EB5555B8BFE4
S31508002A106D420CDD2C4480EA020281EA030382EA55
S31508002A20000083EA010180EA020281EA0303362DE7
S31508002A3088BF30BD11F0004F4FEA01314FF4801CBA
S31508002A404CEA113102D0404261EB410113F0004FCC
S31508002A504FEA03334CEA133302D0524263EB430383
S31508002A6094EA050F00F0A780A4F10104D5F1200E21
S31508002A700DDB02FA0EFC22FA05F2801841F100017C
S31508002A8003FA0EF2801843FA05F359410EE0A5F150
S31508002A9020050EF1200E012A03FA0EFC28BF4CF081
S31508002AA0020C43FA05F3C01851EBE37101F0004537
S31508002AB007D54FF0000EDCF1000C7EEB00006EEB44
S31508002AC00101B1F5801F1BD3B1F5001F0CD34908CE
S31508002AD05FEA30004FEA3C0C04F101044FEA445225
S31508002AE012F5800F80F09A80BCF1004F08BF5FEAAC
S31508002AF0500C50F1000041EB045141EA050130BD8C
S31508002B005FEA4C0C404141EB0101013C28BFB1F59D
S31508002B10801FE9D291F0000F04BF01460020B1FAE8
S31508002B2081F308BF2033A3F10B03B3F120020CDABB
S31508002B300C3208DD02F1140CC2F10C0201FA0CF099
S31508002B4021FA02F10CE002F11402D8BFC2F1200CFE
S31508002B5001FA02F120FA0CFCDCBF41EA0C019040B4
S31508002B60E41AA2BF01EB0451294330BD6FEA0404FD
S31508002B701F3C1CDA0C340EDC04F11404C4F12002E8
S31508002B8020FA04F001FA02F340EA030021FA04F3FA
S31508002B9045EA030130BDC4F10C04C4F1200220FA51
S31508002BA002F001FA04F340EA0300294630BD21FA8F
S31508002BB004F0294630BD94F0000F83F4801306BF55
S31508002BC081F480110134013D4EE77FEA645C18BF49
S31508002BD07FEA655C29D094EA050F08BF90EA020FE0
S31508002BE005D054EA000C04BF1946104630BD91EAD8
S31508002BF0030F1EBF0021002030BD5FEA545C05D1DB
S31508002C004000494128BF41F0004130BD14F5800419
S31508002C103CBF01F5801130BD01F0004545F0FE418D
S31508002C2041F470014FF0000030BD7FEA645C1ABFC2
S31508002C30194610467FEA655C1CBF0B46024650EAF9
S31508002C40013406BF52EA033591EA030F41F4002125
S31508002C5030BD00BF90F0000F04BF0021704730B5AB
S31508002C604FF4806404F132044FF000054FF0000180
S31508002C7050E700BF90F0000F04BF0021704730B541
S31508002C804FF4806404F1320410F0004548BF404216
S31508002C904FF000013EE700BF42004FEAE2014FEA6B
S31508002CA031014FEA02701FBF12F07F4393F07F4F46
S31508002CB081F06051704732F07F4208BF704793F049
S31508002CC07F4F04BF41F40021704730B54FF460745C
S31508002CD001F0004521F000411CE700BF50EA01025F
S31508002CE008BF704730B54FF000050AE050EA010208
S31508002CF008BF704730B511F0004502D5404261EB78
S31508002D0041014FF4806404F132045FEA915C3FF4B8
S31508002D10D8AE4FF003025FEADC0C18BF03325FEA55
S31508002D20DC0C18BF033202EBDC02C2F1200300FA06
S31508002D3003FC20FA02F001FA03FE40EA0E0021FA2B
S31508002D4002F11444BDE600BF70B54FF0FF0C4CF419
S31508002D50E06C1CEA11541DBF1CEA135594EA0C0FCB
S31508002D6095EA0C0F00F0DEF82C4481EA030621EA06
S31508002D704C5123EA4C5350EA013518BF52EA033541
S31508002D8041F4801143F4801338D0A0FB02CE4FF0F3
S31508002D900005E1FB02E506F00042E0FB03E54FF023
S31508002DA00006E1FB03569CF0000F18BF4EF0010E1B
S31508002DB0A4F1FF04B6F5007F64F5407404D25FEA17
S31508002DC04E0E6D4146EB060642EAC62141EA5551CA
S31508002DD04FEAC52040EA5E504FEACE2EB4F1FD0C0C
S31508002DE088BFBCF5E06F1ED8BEF1004F08BF5FEA8A
S31508002DF0500E50F1000041EB045170BD06F000463C
S31508002E0046EA010140EA020081EA0301B4EB5C04E8
S31508002E10C2BFD4EB0C0541EA045170BD41F48011E0
S31508002E204FF0000E013C00F3AB8014F1360FDEBF05
S31508002E30002001F0004170BDC4F10004203C35DAE1
S31508002E400C341BDC04F11404C4F1200500FA05F364
S31508002E5020FA04F001FA05F240EA020001F0004205
S31508002E6021F0004110EBD37021FA04F642EB06017B
S31508002E705EEA430E08BF20EAD37070BDC4F10C04A5
S31508002E80C4F1200500FA04F320FA05F001FA04F269
S31508002E9040EA020001F0004110EBD37041F1000155
S31508002EA05EEA430E08BF20EAD37070BDC4F1200560
S31508002EB000FA05F24EEA020E20FA04F301FA05F2C8
S31508002EC043EA020321FA04F001F0004121FA04F270
S31508002ED020EA020000EBD3705EEA430E08BF20EA40
S31508002EE0D37070BD94F0000F0FD101F0004640007A
S31508002EF041EB010111F4801F08BF013CF7D041EAFC
S31508002F00060195F0000F18BF704703F000465200FF
S31508002F1043EB030313F4801F08BF013DF7D043EAD0
S31508002F200603704794EA0C0F0CEA135518BF95EA86
S31508002F300C0F0CD050EA410618BF52EA4306D1D10D
S31508002F4081EA030101F000414FF0000070BD50EA2C
S31508002F50410606BF1046194652EA430619D094EAB6
S31508002F600C0F02D150EA013613D195EA0C0F05D1A0
S31508002F7052EA03361CBF104619460AD181EA0301F4
S31508002F8001F0004141F0FE4141F470014FF00000AC
S31508002F9070BD41F0FE4141F4780170BD70B54FF047
S31508002FA0FF0C4CF4E06C1CEA11541DBF1CEA1355C7
S31508002FB094EA0C0F95EA0C0F00F0A7F8A4EB0504A9
S31508002FC081EA030E52EA03354FEA013100F08880A0
S31508002FD04FEA03334FF0805545EA131343EA126369
S31508002FE04FEA022245EA111545EA10654FEA00261E
S31508002FF00EF000419D4208BF964244F1FD0404F5D7
S31508003000407402D25B084FEA3202B61A65EB030532
S315080030105B084FEA32024FF480104FF4002CB6EBEF
S31508003020020E75EB030E22BFB61A754640EA0C006F
S315080030305B084FEA3202B6EB020E75EB030E22BFAF
S31508003040B61A754640EA5C005B084FEA3202B6EBF0
S31508003050020E75EB030E22BFB61A754640EA9C00AF
S315080030605B084FEA3202B6EB020E75EB030E22BF7F
S31508003070B61A754640EADC0055EA060E18D04FEA3D
S31508003080051545EA16754FEA06164FEAC30343EADD
S3150800309052734FEAC2025FEA1C1CC0D111F4801FAA
S315080030A00BD141EA00014FF000004FF0004CB6E7A3
S315080030B011F4801F04BF01430020B4F1FD0C88BF42
S315080030C0BCF5E06F3FF6AFAEB5EB030C04BFB6EB4D
S315080030D0020C5FEA500C50F1000041EB045170BD40
S315080030E00EF0004E4EEA113114EB5C04C2BFD4EB6D
S315080030F00C0541EA045170BD41F480114FF0000EF1
S31508003100013C90E645EA060E8DE60CEA135594EA6C
S315080031100C0F08BF95EA0C0F3FF43BAF94EA0C0F6F
S315080031200AD150EA01347FF434AF95EA0C0F7FF4E4
S3150800313025AF104619462CE795EA0C0F06D152EA38
S3150800314003353FF4FDAE1046194622E750EA41061C
S3150800315018BF52EA43067FF4C5AE50EA41047FF42D
S315080031600DAF52EA43057FF4EBAE12E74FEA410290
S31508003170B2F1E04324BFB3F5001CDCF1FE5C0DD9C7
S3150800318001F0004C4FEAC0024CEA5070B2F1004F11
S3150800319040EB830008BF20F00100704711F0804F14
S315080031A021D113F13872BCBF01F00040704741F4D9
S315080031B080114FEA5252C2F11802C2F1200C10FADD
S315080031C00CF320FA02F018BF40F001004FEAC123C1
S315080031D04FEAD32303FA0CFC40EA0C0023FA02F365
S315080031E04FEA4303CCE77FEA625307D150EA01333B
S315080031F01EBF4FF0FE4040F44000704701F000400B
S3150800320040F0FE4040F40000704700BF80B582B031
S3150800321000AF01237B600C4A00210C480AF0B6FE79
S3150800322003460B4A13600A4B1B68002B14BF012385
S315080032300023DBB21A467B6813407B607B6818461E
S315080032400837BD4680BD00BF302601085532000844
S315080032505C01002080B584B000AF78600123BB60B4
S3150800326001F018FE0246BB681340BB6000F0DAFBAB
S315080032700246BB681340BB6001F0ACFA0246BB6865
S315080032801340BB6000F0DEFF0246BB681340BB601C
S3150800329001F030F90246BB681340BB6001F0DEFB63
S315080032A00246BB681340BB6000F022FE0246BB68BC
S315080032B01340BB6001F01AFD0246BB681340BB60B1
S315080032C001F072F90246BB681340BB6000F0F2F9E0
S315080032D00246BB681340BB6000F032F80246BB6882
S315080032E01340BB60BB68002B1FD10AF029FE0220E1
S315080032F001F098FB104B1B689B0B642202FB03F33F
S31508003300FB600EE000BF00BF00BF00BF00BF00BFEC
S3150800331000BF00BF00BF00BF00BF00BFFB68013B86
S31508003320FB60FB68002BEDD1E1E7044B1B681846F0
S315080033300AF0BEFEFEE700BFA80000205C010020E0
S3150800334080B582B000AF01237B6044480AF0ACFF29
S315080033500346434A1360424B1B68002B14BF0123E4
S315080033600023DBB21A467B6813407B603D4A002186
S315080033703D480AF00BFE03463C4A13603B4B1B686C
S31508003380002B14BF01230023DBB21A467B681340C7
S315080033907B60374A102108200BF0B0F90346354AFE
S315080033A01360344B1B68002B14BF01230023DBB2C8
S315080033B01A467B6813407B602F4B022201212F4857
S315080033C00AF0C8FE03462E4A13602D4B1B68002BD5
S315080033D014BF01230023DBB21A467B6813407B60C7
S315080033E0284B0422012125480AF0B4FE0346264A42
S315080033F01360254B1B68002B14BF01230023DBB287
S315080034001A467B6813407B601D4B1B684FF47A7124
S3150800341018460AF01BFF0346002B0CBF01230023A6
S31508003420DBB21A467B6813407B60174B1B6840F675
S31508003430B83118460AF00AFF0346002B0CBF0123D1
S315080034400023DBB21A467B6813407B600F4801F005
S3150800345077F97B6818460837BD4680BD902601086F
S3150800346068010020542601089134000860010020F4
S315080034707826010864010020A026010859360008AC
S315080034806C010020B0260108700100207D36000876
S3150800349080B58CB000AF78606C4B18684FF0FF337E
S315080034A0002207210AF0B6FFF862FB6A03F001035F
S315080034B0002B00F0B880664B186807F1100100234E
S315080034C000220BF0EFF93B7C87F82B307B7E87F8E0
S315080034D02A3097F82A30012B2AD197F82B30142B4B
S315080034E00AD9FF2387F82030FA697B7E07F1200086
S315080034F0012101F0D9F896E097F82B30184600F02C
S315080035003FFB0346FB6097F82B3087F8203007F11E
S315080035102003591C07F10C030422184602F022FC6A
S31508003520FA697B7E07F12000052101F0BDF87AE0F3
S3150800353097F82A30022B0FD107F1080107F110037B
S3150800354001330422184602F00DFC97F82B30B968AF
S31508003550184600F089FA66E097F82A30002B5FD102
S3150800356097F82B30082B17DC002B5BDD013B072B6C
S3150800357058D801A252F823F09F350008A73500084D
S31508003580AF35000825360008BF350008D5350008D0
S31508003590F13500081B360008FF2B15D042E0012044
S315080035A000F0F0F83FE0002000F0ECF83BE0294B93
S315080035B01B6840F6B83118460AF048FE33E0002189
S315080035C0132000F0BBFA2EE0002000F0DBF804F030
S315080035D066FF28E0062387F82030042387F8213081
S315080035E0FA697B7E07F12000022101F05DF81AE0F6
S315080035F0072387F8203000F02FFB0346002B01D065
S31508003600FF2300E0002387F82130FA697B7E07F163
S315080036102000022101F048F805E000F055FB02E021
S3150800362000BF00E000BFFB6A03F00203002B02D0D4
S31508003630022001F0F7F9FB6A03F00403002B3FF4BC
S315080036402BAF002000F09EF826E700BF6801002097
S31508003650640100207001002080B582B000AF786058
S31508003660054B1B687A68114618460AF05DFE00BFCE
S315080036700837BD4680BD00BF6801002090B585B0FB
S3150800368000AF3C4684E80F00084B1868394600230B
S3150800369000220BF0A7F8064B1B68012118460AF012
S315080036A043FE00BF1437BD4690BD00BF640100202D
S315080036B06801002080B582B000AF01237B60284AEC
S315080036C0002128480AF062FC0346274A1360264B65
S315080036D01B68002B14BF01230023DBB21A467B6844
S315080036E013407B6021480AF0DFFD0346204A136039
S315080036F01F4B1B68002B14BF01230023DBB21A469D
S315080037007B6813407B601B4B012201211A480AF093
S3150800371021FD0346194A1360184B1B68002B14BF7A
S3150800372001230023DBB21A467B6813407B609FEDBA
S31508003730140A00F015F9114B1B68642118460AF0A3
S3150800374085FD0346002B0CBF01230023DBB21A4676
S315080037507B6813407B607B6818460837BD4680BD8A
S31508003760C0260108B537000874010020F4260108B0
S315080037707C010020E4260108013A000878010020AF
S315080037800000000080B582B000AF78607968032039
S3150800379001F0D6F87968122000F0D0F900BF083792
S315080037A0BD4680BD80B500AF122000F009FA034679
S315080037B0184680BD80B592B000AF78604FF0000320
S315080037C07B644FF000033B64624BBB63624B186833
S315080037D04FF0FF33002201210AF01CFE78637B6B51
S315080037E003F00103002BF1D05C4806F0EEF9FFF771
S315080037F0D9FF0346002B00F0A580002000F0E0F971
S315080038000346002B40F08780022000F0E7F987ED99
S315080038100C0A032000F0E2F987ED0B0A042000F0F9
S31508003820DDF987ED0A0A062000F0D8F987ED090ABE
S31508003830072000F0D3F987ED080A092000F0CEF931
S3150800384087ED070A052000F0C9F987ED060A97ED06
S31508003850077AD7ED067A77EE677AC7ED057A97ED98
S315080038600C7AD7ED057A67EE277AC7ED047A97EDD5
S31508003870057AD7ED0E7A67EE277A97ED107A77EE06
S31508003880277AC7ED107A97ED0B7AD7ED107A67EE9F
S31508003890277AC7ED037A97ED057AD7ED117A37EED1
S315080038A0677AD7ED0A7A67EE276A97ED0E7AC6EE3B
S315080038B0877AC7ED027A7B697B6497ED047AD7ED40
S315080038C0037A77EE277A97ED027A77EE277AC7EDAD
S315080038D00F7A97ED0F7AD7ED097AB4EEE77AF1EE1B
S315080038E010FA05DD7B6AFB634FF000033B640DE0CD
S315080038F097ED0F7AD7ED087AB4EEE77AF1EE10FA7B
S3150800390004D53B6AFB634FF000033B6497ED0F0A4F
S3150800391000F026F85AE7002000F052F90346012B7A
S315080039207FF454AF012000F059F9F0EE407AB0EE7A
S31508003930670A00F015F84FF000037B644FF00003A8
S315080039403B6443E74FF000037B644FF000033B649E
S315080039503CE700BFCDCCCC3D7C010020D003002045
S3150800396080B584B000AF87ED010A0123FB60D7ED6F
S31508003970017AB2EE087AF4EEC77AF1EE10FA01DDB2
S315080039801D4B7B60D7ED017AB8EE087AF4EEC77A5C
S31508003990F1EE10FA01D5194B7B607868FFF77CF9D0
S315080039A011A3D3E90023FFF719F802460B46104680
S315080039B019460FA3D3E90023FFF7F0FA02460B4690
S315080039C010461946FFF7D2FB034600EE103A00F000
S315080039D0ABFD0246FB681340FB60FB6818461037D0
S315080039E0BD4680BDAFF300804A0C022B87163440D3
S315080039F077BE9F1A2F0D414000004041000040C08D
S31508003A0080B582B000AF7860054B1B687A681146AE
S31508003A1018460AF089FC00BF0837BD4680BD00BFBE
S31508003A207C01002080B582B000AF01237B600C4882
S31508003A300AF056FD03460B4A13600A4B1B68002B17
S31508003A4014BF01230023DBB21A467B6813407B6050
S31508003A5000F0ECF87B6818460837BD4680BD00BF05
S31508003A60542801082802002080B582B000AF03461A
S31508003A703960FB71FB79134A1B0113441B7803F069
S31508003A800803002B19D1104B1B684FF0FF3118465D
S31508003A900AF0ACFDFB793968184600F0E3F90346ED
S31508003AA0002B04D0FB7909493A6841F83320064BC4
S31508003AB01B6818460AF0E5FD00E000BF0837BD465A
S31508003AC080BD00BF042701082802002080010020CD
S31508003AD080B582B000AF03463960FB71154B1B6891
S31508003AE04FF0FF3118460AF081FDFB793968184610
S31508003AF000F0B8F90346002B0DD1FB790E4ADB001E
S31508003B0013441A79FB7942F00202D1B20A4ADB0061
S31508003B1013440A461A71FB7907493A6841F8332073
S31508003B20044B1B6818460AF0ACFD00BF0837BD46B3
S31508003B3080BD00BF280200208001002080B582B029
S31508003B4000AF03463960FB713A68FB79114618469F
S31508003B50FFF7BEFF00BF0837BD4680BD80B582B0FF
S31508003B6000AF034687ED000AFB713A68FB791146F8
S31508003B701846FFF7ADFF00BF0837BD4680BD0000F9
S31508003B8080B584B000AF0346FB710B4B1B684FF042
S31508003B90FF3118460AF02AFDFB79084A52F83330F5
S31508003BA0FB60054B1B6818460AF06BFDFB68184658
S31508003BB01037BD4680BD00BF2802002080010020C6
S31508003BC080B582B000AF0346FB71FB791846FFF754
S31508003BD0D7FF034618460837BD4680BD80B582B074
S31508003BE000AF0346FB71FB791846FFF7C9FF03468A
S31508003BF007EE903AB0EE670A0837BD4680BD00006A
S31508003C0080B582B000AF0346FB71FB79064A1B01FB
S31508003C1013440433FA7919681046FFF759FF00BFB1
S31508003C200837BD4680BD00BF0427010880B582B0AD
S31508003C3000AF0023FB8007E0FB88DBB21846FFF7DE
S31508003C40DFFFFB880133FB80FB88142BF4D900BF08
S31508003C5000BF0837BD4680BD80B582B000AF0123DE
S31508003C607B6001F0CFF902467B6813407B60002336
S31508003C70FB7019E0FB78134A1B0113441B7803F009
S31508003C801003002B0DD0FB781846FFF779FF024684
S31508003C90FB781146184601F052F902467B68134034
S31508003CA07B60FB780133FB70FB78142BE2D901F0BB
S31508003CB08BF902467B6813407B607B681846083799
S31508003CC0BD4680BD0427010880B584B000AF012336
S31508003CD0FB600023FB721DE0FB7A1E4A1B0113449E
S31508003CE01B7803F01003002B11D03A1DFB7A1146FE
S31508003CF0184601F007F90246FB681340FB60FB68AB
S31508003D00002B04D0FB7A79681846FFF7E1FEFB7AA8
S31508003D100133FB72FB7A142BDED9FB68002B15D115
S31508003D200023BB720FE0BB7A0A4A1B0113441B78B7
S31508003D3003F01003002B03D0BB7A1846FFF760FF89
S31508003D40BB7A0133BB72BB7A142BECD900BF103790
S31508003D50BD4680BD0427010880B483B000AF7860F3
S31508003D607B68012B94BF01230023DBB218460C376E
S31508003D70BD465DF8047B704780B483B000AF034648
S31508003D803960FB71FB790D4A1B01134408331B6824
S31508003D903A689A420AD3FB79084A1B0113440C3342
S31508003DA01B683A689A4201D8012300E000231846A6
S31508003DB00C37BD465DF8047B704700BF0427010831
S31508003DC080B483B000AF03463960FB71FB790D4AB6
S31508003DD01B01134408331B683A689A420ADBFB79CD
S31508003DE0084A1B0113440C331B683A689A4201DCE3
S31508003DF0012300E0002318460C37BD465DF8047B16
S31508003E00704700BF0427010880B483B000AF03469B
S31508003E1087ED000AFB71FB79114A1B01134408332D
S31508003E20D3ED007A97ED007AB4EEE77AF1EE10FA60
S31508003E300FDBFB790A4A1B0113440C33D3ED007AD6
S31508003E4097ED007AB4EEE77AF1EE10FA01D801237D
S31508003E5000E0002318460C37BD465DF8047B704722
S31508003E600427010880B582B000AF03463960FB71AC
S31508003E70FB791E4A1B0113441B7803F00103002B30
S31508003E8009D0D7ED007AFB79B0EE670A1846FFF736
S31508003E90BBFF034626E0FB79144A1B0113441B7833
S31508003EA003F00203002B07D03A68FB79114618463F
S31508003EB0FFF786FF034615E0FB790C4A1B011344FE
S31508003EC01B7803F00403002B05D03B681846FFF760
S31508003ED043FF034606E03A68FB7911461846FFF7A2
S31508003EE04BFF034618460837BD4680BD0427010820
S31508003EF080B582B000AF01237B6020480AF0F0FA53
S31508003F0003461F4A13601E4B1B68002B14BF012370
S31508003F100023DBB21A467B6813407B60184B1B688C
S31508003F204FF0FF3118460AF061FB002000F0C4FC90
S31508003F3000228221002000F0F3F802467B68134035
S31508003F407B60002000F0DAFC012000F0B5FC0022BE
S31508003F508221002000F0E4F802467B6813407B606B
S31508003F60012000F0CBFC064B1B6818460AF089FBBB
S31508003F707B6818460837BD4680BD00BF642801081F
S31508003F803C02002080B588B000AF0346B9607A606D
S31508003F90FB730123BB61BB6800221A700023FB82F6
S31508003FA00123FB77FB7B002B02D10123FB7704E07F
S31508003FB0FB7B012B01D10023FB77584B1B684FF085
S31508003FC0FF3118460AF012FBFB7F184600F074FC16
S31508003FD00022A021002000F0A3F80246BB69134086
S31508003FE0BB61FB7F184600F089FC4C4B1B681846E2
S31508003FF00AF047FB64200AF07CF8484B1B684FF030
S31508004000FF3118460AF0F2FAFB7F184600F054FC16
S3150800401007F1160301221946012000F0C7F80246E7
S31508004020BB691340BB61FB7F184600F067FC3B4B3E
S315080040301B6818460AF025FBBB69002B08D1BB682C
S315080040401B7843F00203DAB2BB681A70002360E0FB
S31508004050FB8A03F00103002B36D0304B1B684FF068
S31508004060FF3118460AF0C2FAFB7F184600F024FC16
S315080040700022B968072000F099F80246BB69134088
S31508004080BB61FB7F184600F039FCFB7F184600F041
S3150800409013FC00228221002000F042F80246BB6988
S315080040A01340BB61FB7F184600F028FC1B4B1B68BE
S315080040B018460AF0E6FABB681B7843F00103DAB241
S315080040C0BB681A70002324E0FB8A5B089BB2FB825C
S315080040D0FA8A7B681A80114B1B684FF0FF31184625
S315080040E00AF084FAFB7F184600F0E6FB00228421DA
S315080040F0002000F015F80246BB691340BB61FB7F40
S31508004100184600F0FBFB054B1B6818460AF0B9FA7F
S31508004110BB6918462037BD4680BD00BF3C0200205B
S3150800412080B584B000AF03463A60FB710B46BB808E
S315080041300123FB603B68002B1AD0FB7963F07F03F1
S31508004140DAB2184B1A70BB88DBB21B12DAB2154BFF
S315080041505A70BB88DAB2134B9A70134B03229A81B2
S31508004160114800F09BFC0246FB681340FB6013E015
S31508004170FB7963F07F03DAB20A4B1A70BB88DAB2AE
S31508004180084B5A70084B02229A81074800F086FCB1
S315080041900246FB681340FB60FB6818461037BD46AD
S315080041A080BD00BF340200200000002080B586B024
S315080041B000AF0346B9607A60FB7301237B617B68B5
S315080041C0002B1FD01C4AFB7B13701B4B00225A7016
S315080041D0194B00229A70194B03229A81174800F04E
S315080041E05DFC02467B6913407B61154B5B781B02BD
S315080041F01AB2134B9B781BB213431BB29AB2BB6815
S315080042001A8014E00C4AFB7B13700B4B00225A7081
S315080042100A4B02229A81094800F040FC02467B6953
S3150800422013407B61064B5B789AB2BB681A807B6940
S3150800423018461837BD4680BD34020020000000200D
S315080042402C02002080B582B000AF01237B601D4A96
S3150800425000211D4809F09AFE03461C4A13601B4BB1
S315080042601B68002B14BF01230023DBB21A467B68A8
S3150800427013407B6016480AF017F80346154A136080
S31508004280144B1B68002B14BF01230023DBB21A460C
S315080042907B6813407B6010480AF022F903460F4AF0
S315080042A013600E4B1B68002B14BF01230023DBB2DF
S315080042B01A467B6813407B607B6818460837BD46FC
S315080042C080BD00BF94280108E14200085002002082
S315080042D0B828010854020020C828010858020020FE
S315080042E080B590B000AF7860012009F002FF08227F
S315080042F05E495F4802F028F95E4B18684FF0FF33B5
S31508004300002203210AF086F878637B6B03F0020328
S31508004310002B02D00423FB8707E07B6B03F0010325
S31508004320002B00F0A0800023FB87534B1B684FF03F
S31508004330FF3118460AF05AF90023BB870EE0BA8FF8
S31508004340FB8F1344494A32F81320BB8F9B00403336
S315080043503B4443F8242CBB8F0133BB87BB8F032B0D
S31508004360EDD91420FFF73AFC87ED0C0A00237B876A
S3150800437033E07B8F9B0040333B4453F8243C07EEE5
S31508004380903AF8EE677AF3EE006A87EEA67ADFEDE2
S315080043903B6AC7EE267A97ED0C7A67EE277AC7ED61
S315080043A00B7A7B8F364A9B00134493ED007AD7ED40
S315080043B00B7A27EE277A7B8F324A9B001344D3ED7C
S315080043C0007A7B8F77EE677A9B0040333B44343B19
S315080043D0C3ED007A7B8F01337B877B8F032BC8D98C
S315080043E0D7ED057AB0EE670A0B20FFF7B7FBD7EDD6
S315080043F0067AB0EE670A0C20FFF7B0FB97ED057A50
S31508004400D7ED067AC7EE276AB0EE660A0D20FFF7E3
S31508004410A5FB97ED057AD7ED067A67EE277AB0EE13
S31508004420670A0E20FFF79AFBD7ED037AB0EE670A04
S315080044300F20FFF793FBD7ED047AB0EE670A10203A
S31508004440FFF78CFB97ED037AD7ED047A67EE277AA8
S31508004450B0EE670A1120FFF781FB074B1B68184669
S315080044600AF00FF948E700BF46E700BF4002002000
S3150800447070020020540200205802002000008045E7
S31508004480742801088428010880B582B000AF7860D6
S31508004490044B1B680221184609F046FF00BF08377F
S315080044A0BD4680BD5402002080B582B000AF78605A
S315080044B0044B1B680121184609F036FF00BF083770
S315080044C0BD4680BD5402002080B483B000AF78603A
S315080044D07B689B6D7B689B6D7B689B6D7B689B6D22
S315080044E07B68DB6CDB6B00BF0C37BD465DF8047B75
S315080044F07047000080B582B000AF01237B600021C1
S31508004500084804F0E9F80346002B0CBF01230023F2
S31508004510DBB21A467B6813407B607B68184608370F
S31508004520BD4680BD6803002080B584B000AF87ED26
S31508004530010A0123FB6097ED010A00F013F8B86041
S31508004540BB6800220021064804F013F903461A4600
S31508004550FB681340FB60FB6818461037BD4680BDF4
S315080045606803002080B52DED028B84B000AF87ED7F
S31508004570010AD7ED017A9FED0B7A27EE878A142078
S31508004580FFF72CFBB0EE407AC8EE077AFCEEE77A26
S3150800459017EE903AFB60FB6818461037BD46BDEC2F
S315080045A0028B80BD00F07F4580B582B000AF012345
S315080045B07B60042000F000FA0346DAB2364B1B781B
S315080045C01343DAB2344B1A70032000F0F5F90346A8
S315080045D05B00DAB2304B1B781343DAB22E4B1A70F3
S315080045E0022000F0E9F903469B00DAB22A4B1B7851
S315080045F01343DAB2284B1A70012000F0DDF903469E
S31508004600DB00DAB2244B1B781343DAB2224B1A705A
S31508004610224B1B68204A1278520113431F4A136023
S315080046201F49204803F0E5F80346002B0CBF012379
S315080046300023DBB21A467B6813407B60174919488A
S3150800464003F0D7F80346002B0CBF01230023DBB287
S315080046501A467B6813407B60124803F094F90346B8
S31508004660002B0CBF01230023DBB21A467B681340DC
S315080046707B6002210B4803F0ACFB0346002B0CBF02
S3150800468001230023DBB21A467B6813407B607B68F4
S3150800469018460837BD4680BD600200206C00002021
S315080046A0440000201C03002080B58CB000AFF860E1
S315080046B07A601A460B46FB721346BB720123FB62ED
S315080046C000237B85FB7A082B01D9002330E07B6821
S315080046D09BB21B029AB2BB7A9BB21B019BB21343D5
S315080046E09AB2154B1B789BB213439BB243F41073D3
S315080046F07B857B8D3B6100237B610023BB610023A7
S31508004700FB61FB7A3B62002387F8243007F110012E
S315080047100123FA68094803F07AF90346002B0CBF0F
S3150800472001230023DBB21A46FB6A1340FB62FB6ACD
S3150800473018463037BD4680BD600200201C030020A5
S3150800474080B483B000AF7860044A7B68136000BF0A
S315080047500C37BD465DF8047B704700BF5C0200203D
S3150800476090B591B000AF786007F11C0307F12402F9
S315080047700021786803F01BFA7B6A1B0A03F0010321
S31508004780BB617B6A1B09DBB203F00303DBB27B75F3
S315080047907B6BDBB23B753B7D9AB207F10C0107F1E7
S315080047A01C03184601F0DEFA044B1C6807F10C03DB
S315080047B00FCBA04700BF4437BD4690BD5C02002022
S315080047C080B483B000AF786000BF0C37BD465DF893
S315080047D0047B704780B584B000AF0123BB60334BC0
S315080047E01B6E324A43F001031366304B1B6E03F00F
S315080047F001037B607B680023FB731EE0FB7B2C4A6E
S315080048005B01134408331B68002B01D1012300E028
S315080048100023BA681340BB60FB7B254A5B0113443F
S315080048201A68FB7B5B0122490B4404331946104680
S3150800483004F0A2FEFB7B0133FB73FB7B042BDDD963
S315080048400023FB732AE0FB7B1A4A5B0113440833F7
S315080048501B68012B07D0FB7B164A5B011344083300
S315080048601B68112B01D1012300E00023BA6813400D
S31508004870BB60FB7B184600F041F8FB7B0D4A5B01E9
S3150800488013441A68FB7B5B010A490B440433194637
S31508004890104604F071FEFB7B0133FB73FB7B032B95
S315080048A0D1D9BB6818461037BD4680BD00100240F6
S315080048B0D82801087829010880B582B000AF0346D8
S315080048C0FB71FB790C4A5B0113441868FB790A4AA9
S315080048D05B01134404331B6899B2FB79064A5B01F2
S315080048E013441C331B68DBB21A4604F0C7FF00BF2B
S315080048F00837BD4680BD00BF7829010880B582B05B
S3150800490000AF0346FB71FB790C4A5B011344186838
S31508004910FB790A4A5B01134404331B6899B2FB7995
S31508004920064A5B01134418331B68DBB21A4604F0C7
S31508004930A5FF00BF0837BD4680BD00BF782901081E
S3150800494080B582B000AF03463960FB713B68002B27
S3150800495016D0FB79174A5B0113441868FB79154A88
S315080049605B01134404331B6899B2FB79114A5B0156
S3150800497013441C331B68DBB21A4604F07FFF15E0AC
S31508004980FB790C4A5B0113441868FB79094A5B01F9
S31508004990134404331B6899B2FB79064A5B01134436
S315080049A018331B68DBB21A4604F068FF00BF0837E5
S315080049B0BD4680BD7829010880B584B000AF03469E
S315080049C0FB71FB79164A5B0113441A68FB79144993
S315080049D05B010B4404331B689BB21946104604F06E
S315080049E035FF0346FB73FB790D4A5B0113441C3301
S315080049F01B68012B02D1FB7B012B0AD0FB79084AE5
S31508004A005B01134418331B68012B04D1FB7B002B75
S31508004A1001D1012300E0002318461037BD4680BDAA
S31508004A20D828010880B582B000AF0346FB71FB7930
S31508004A30094A5B0113441A68FB7907495B010B4471
S31508004A4004331B689BB21946104604F02FFF00BFBB
S31508004A500837BD4680BD00BF7829010880B582B0F9
S31508004A6000AF01237B600B4809F01EFC03460A4A87
S31508004A701360094B1B68002B14BF01230023DBB20C
S31508004A801A467B6813407B607B6818460837BD4624
S31508004A9080BD00BF082A01086402002090B585B0D1
S31508004AA000AF78600023FB607B681B781946474A8D
S31508004AB00B469B000B449B00134404331B684FF0C2
S31508004AC0FF31184609F092FD414B18687B681B7840
S31508004AD019463E4A0B469B000B449B0013440C3375
S31508004AE01A687B681B781C46384923469B00234472
S31508004AF09B000B4410331B681343194609F058FCF6
S31508004B007B681B781946314A0B469B000B449B0071
S31508004B10134418687B6859687B689A687B689B8920
S31508004B2006F054FA0346002B0CBF01230023DBB220
S31508004B30BB60BB68002B1FD0254B18687B681B78A9
S31508004B401946224A0B469B000B449B0013440C3320
S31508004B501A687B681B781C461C4923469B0023441D
S31508004B609B000B4410331B6842EA03014FF0FF33E6
S31508004B70002209F04FFCF8607B681B781946134A37
S31508004B800B469B000B449B00134410331A68FB68C2
S31508004B901340002B0CBF01230023DBB21A46BB6867
S31508004BA01340BB607B681B781946084A0B469B0076
S31508004BB00B449B00134404331B68184609F061FD37
S31508004BC0BB6818461437BD4690BD00BF9400002048
S31508004BD06402002080B584B000AF7860786800F081
S31508004BE061F80346FB73094B1868FA7B08491346B4
S31508004BF09B0013449B000B440C331B68194609F0B1
S31508004C0093FB00BF1037BD4680BD00BF640200207D
S31508004C109400002080B584B000AF7860786800F012
S31508004C2041F80346FB73094B1868FA7B0849134693
S31508004C309B0013449B000B440C331B68194609F070
S31508004C4073FB00BF1037BD4680BD00BF640200205D
S31508004C509400002080B584B000AF78607B681B6E36
S31508004C607B689B6DDB6B7B685B6DDB6B786800F044
S31508004C7019F80346FB73094B1868FA7B084913466B
S31508004C809B0013449B000B4410331B68194609F01C
S31508004C904BFB00BF1037BD4680BD00BF6402002035
S31508004CA09400002080B485B000AF78600023FB73C1
S31508004CB00FE0FA7B0C4913469B0013449B000B44F8
S31508004CC01B687A689A4201D1FB7B06E0FB7B0133BD
S31508004CD0FB73FB7B002BECD0002318461437BD462C
S31508004CE05DF8047B704700BF9400002080B582B051
S31508004CF000AF01237B600C4A00210C4809F046F9F5
S31508004D0003460B4A13600A4B1B68002B14BF01238A
S31508004D100023DBB21A467B6813407B607B68184623
S31508004D200837BD4680BD00BF182A0108354D000862
S31508004D306802002080B586B000AF786001237B61E9
S31508004D400023FB740A2009F0D4F907F1100207F1D1
S31508004D50130319460020FFF715F902467B6913402D
S31508004D607B617B69002B08D03B8A184600F050F817
S31508004D70F0EE407AC7ED027A09E0FB7C03F0010306
S31508004D80002B224BBB600023FB7401237B6107F1D8
S31508004D90100207F1130319460120FFF7F3F802463C
S31508004DA07B6913407B617B69002B08D03B8A1846D8
S31508004DB000F02EF8F0EE407AC7ED037A09E0FB7CA6
S31508004DC003F00103002B114BFB600023FB74012346
S31508004DD07B61D7ED027AB0EE670A0820FEF7BEFEC1
S31508004DE0D7ED037AB0EE670A0920FEF7B7FE97ED0E
S31508004DF0027AD7ED037A77EE677AB0EE670A0A2069
S31508004E00FEF7ACFE642009F074F99EE77B9488C32C
S31508004E1080B485B000AF0346FB80FB8807EE903A66
S31508004E20B8EEE77ADFED176AC7EE267AC7ED037A9A
S31508004E30D7ED037A9FED147A67EE877AC7ED027A83
S31508004E40D7ED027A9FED117A77EE877AC7ED027A67
S31508004E5097ED027AD7ED037A67EE277AC7ED027ADD
S31508004E60D7ED027A9FED0A7A77EEC77AC7ED027A0E
S31508004E70BB6807EE903AB0EE670A1437BD465DF890
S31508004E80047B704700000046DB8A1F416DE76B43D1
S31508004E9042E0754380B582B000AF01237B601748B6
S31508004EA009F01EFB0346164A1360154B1B68002BB8
S31508004EB014BF01230023DBB21A467B6813407B60CC
S31508004EC000F0A0F802467B6813407B60002006F0DD
S31508004ED03DFE0346002B0CBF01230023DBB21A4616
S31508004EE07B6813407B6000F06FF802467B681340CE
S31508004EF07B607B6818460837BD4680BD3C2A01089A
S31508004F006C02002080B584B000AF03463960FB719F
S31508004F100123FB60FB799BB23968184607F048FE07
S31508004F200346002B0CBF01230023DBB21A46FB689D
S31508004F301340FB60FB6818461037BD4680BD80B538
S31508004F4084B000AF03463960FB710123FB60002380
S31508004F507B81FB799BB23A681146184607F04DFEED
S31508004F6003467B817B8903F48073002B21D007F0ED
S31508004F705FFE03461A467B8913437B817B89002B98
S31508004F800CBF01230023DBB21A46FB681340FB6003
S31508004F90FB799BB23A681146184607F02EFE03467F
S31508004FA0002B0CBF01230023DBB21A46FB68134013
S31508004FB0FB607B89DBB2FF2B01D10023FB60FB681A
S31508004FC018461037BD4680BD80B582B000AF0123B4
S31508004FD07B6004F0E7F80346002B0CBF012300238F
S31508004FE0DBB21A467B6813407B60054B1B68184684
S31508004FF009F047FB7B6818460837BD4680BD00BFE9
S315080050006C02002080B582B000AF01237B600C4B98
S315080050101B684FF0FF31184609F0E8FA04F0A0F8CB
S315080050200346002B0CBF01230023DBB21A467B681C
S3150800503013407B607B6818460837BD4680BD00BFB5
S315080050406C02002080B400AF034B044A9A6000BF8C
S31508005050BD465DF8047B704700ED00E000280008B7
S3150800506080B500AFFFF7EEFF00F08DFE00F026F8E2
S3150800507000F084FA00F048FA00F072F800F014F92B
S3150800508000F06AF900F002FA00F0A2F900F0E0F97F
S3150800509000F040F908F00AFF054A0021054808F023
S315080050A075FF0346044A136008F024FFFEE700BFB5
S315080050B04C2A0108BD560008D404002080B596B0D5
S315080050C000AF07F114034422002118460DF03CF9FD
S315080050D03B4600221A605A609A60DA601A614FF4F9
S315080050E0007004F091FD0346002B01D000F0F4FA9D
S315080050F009237B614FF4A023BB610123BB62022312
S31508005100FB6303233B6404237B641023BB640723EC
S31508005110FB6402233B6502237B6507F114031846EB
S3150800512004F0C8FD0346002B01D000F0D5FA0F2382
S315080051303B6003237B600023BB600023FB600023E6
S315080051403B613B460421184605F0C8F90346002B87
S3150800515001D000F0C1FA00BF5837BD4680BD000037
S3150800516080B586B000AF3B4600221A605A609A6046
S31508005170DA601A615A61464B464A1A60444B002265
S315080051805A60434B00229A60414B0022DA60404B3A
S3150800519001221A613E4B08225A613D4B00221A76BB
S315080051A03B4B01225A763A4B0422DA61384B0022ED
S315080051B083F82020364B00229A62354B0022DA62A9
S315080051C0334B012283F83020314B00225A63304B8F
S315080051D0012283F838202E4B1C22DA632C4B8022BE
S315080051E01A642B4B00225A64294B01229A642848D8
S315080051F001F062F80346002B01D000F06DFA264B49
S315080052003B6006237B600723BB607F23FB60042388
S315080052103B6100237B613B4619461D4801F0D6FBDE
S315080052200346002B01D000F057FA1C4B3B600C23B9
S315080052307B603B461946164801F0C8FB0346002B1F
S3150800524001D000F049FA164B3B6012237B603B46BF
S3150800525019460F4801F0BAFB0346002B01D000F0AF
S315080052603BFA104B3B6018237B603B4619460848BF
S3150800527001F0ACFB0346002B01D000F02DFA7F218C
S31508005280034802F029F900BF1837BD4680BD00BFA4
S31508005290700200200000045040002019000021433D
S315080052A08000501D0080F03E80B500AF174B184AAD
S315080052B01A60164B20225A60144B00229A60134B30
S315080052C00022DA60114B4FF440221A610F4B4FF45B
S315080052D0A0025A610D4B00221A760C4B00225A7610
S315080052E00A4B00229A76094B0122DA76074B0022EE
S315080052F01A77064B00225A77044802F07FF90346CC
S31508005300002B01D000F0E8F900BF80BD1C03002087
S315080053100064004080B500AF0D4B0E4A1A600C4B76
S3150800532000221A710A4B00225A71094B00225A614F
S31508005330074B00229A61064B01221A62044803F0C1
S31508005340BFF80346002B01D000F0C6F900BF80BDA8
S31508005350440300200030024080B58AB000AF3B1DF0
S315080053602422002118460CF0EFFF174B174A1A6043
S31508005370154803F08FF90346002B01D000F0ACF96D
S3150800538000237B600023BB600023FB6000233B6196
S3150800539000237B613B1D002219460B4803F00EFAD9
S315080053A00346002B01D000F097F93B1D0022194651
S315080053B0054803F01DFB0346002B01D000F08CF9CD
S315080053C000BF2837BD4680BD680300200074004032
S315080053D080B500AF1B4B1C4A1A601A4B1B4A5A6011
S315080053E0184B00229A60174B0122DA60154B0022EF
S315080053F01A61144B00225A61124B00229A61114B12
S315080054000022DA610F4B00221A620E4804F068FA8D
S315080054100346002B01D000F05FF90021094804F08B
S31508005420EEFA0346002B01D000F056F90021054894
S3150800543004F030FB0346002B01D000F04DF900BF05
S3150800544080BD00BF7C03002000540040EC9C9010F7
S3150800545080B500AF0B4B0C4A1A600A4B06225A60FD
S31508005460084B40F6FF72DA60064B96229A600548AA
S3150800547004F05CFB0346002B01D000F02DF900BFB9
S3150800548080BD00BFD00300200030004080B500AFCB
S315080054901B4B1C4A1A601A4B4FF482725A60184BFF
S315080054A000229A60164B4FF4E062DA60144B002231
S315080054B01A61134B01225A61114B4FF400729A611B
S315080054C00F4B3022DA610E4B00221A620C4B002277
S315080054D05A620B4B00229A62094B0722DA62084B82
S315080054E000221A63064B00225A63054805F0CAFCD7
S315080054F00346002B01D000F0EFF800BF80BD00BFC7
S31508005500E00300200030014080B582B000AF1A4B9E
S315080055109B6C194A43F001039364174B9B6C03F089
S3150800552001037B607B68144B9B6C134A43F00203B0
S315080055309364114B9B6C03F002033B603B680022AB
S3150800554005210C2002F081FF0C2002F09AFF0022B0
S3150800555005210D2002F079FF0D2002F092FF0022AE
S3150800556005213A2002F071FF3A2002F08AFF00BFB7
S315080055700837BD4680BD00BF0010024080B588B020
S3150800558000AF07F10C0300221A605A609A60DA60CD
S315080055901A61474BDB6C464A43F00403D364444B19
S315080055A0DB6C03F00403BB60BB68414BDB6C404A11
S315080055B043F00103D3643E4BDB6C03F001037B60CD
S315080055C07B683B4BDB6C3A4A43F00203D364384BA7
S315080055D0DB6C03F002033B603B6800224FF480411A
S315080055E0344804F04BF900224FF480714FF0904094
S315080055F004F044F9002260212F4804F03FF94FF4E3
S315080056008043FB6001233B6100237B610023BB6170
S3150800561007F10C031946274803F0AEFF4FF4004381
S31508005620FB6000233B6100237B6107F10C031946ED
S31508005630204803F0A1FF4FF48073FB6001233B6110
S3150800564000237B610023BB6107F10C0319464FF069
S31508005650904003F091FF4FF40043FB6000233B6149
S3150800566000237B6107F10C0319464FF0904003F0C5
S3150800567083FF9823FB6000233B6100237B6107F1CE
S315080056800C0319460C4803F077FF6023FB600123DF
S315080056903B6100237B610023BB6107F10C031946BC
S315080056A0054803F069FF00BF2037BD4680BD00BF2F
S315080056B000100240000800480004004880B582B087
S315080056C000AF7860FDF7A2FD024B1B68184608F08C
S315080056D0EFFCFEE7D404002080B400AF72B600BF2A
S315080056E0FEE7000080B582B000AF114B1B6E104A72
S315080056F043F0010313660E4B1B6E03F001037B6038
S315080057007B680B4B9B6D0A4A43F080539365084BA5
S315080057109B6D03F080533B603B6800220F216FF0BE
S31508005720010002F092FE00BF0837BD4680BD00BFEB
S315080057300010024080B5A0B000AF786007F16C0396
S3150800574000221A605A609A60DA601A6107F1180333
S315080057505422002118460CF0F7FD7B681B68444A62
S31508005760934240F081804FF48043BB614FF0405331
S315080057703B6607F11803184605F09CF80346002B0C
S3150800578001D0FFF7A9FF3B4BDB6C3A4A43F40053C1
S31508005790D364384BDB6C03F400537B617B69354B70
S315080057A0DB6C344A43F00103D364324BDB6C03F001
S315080057B001033B613B692F4BDB6C2E4A43F0020326
S315080057C0D3642C4BDB6C03F00203FB60FB680623F7
S315080057D0FB660B233B6700237B6707F16C031946BF
S315080057E04FF0904003F0C8FE0323FB660B233B678C
S315080057F000237B6707F16C0319461F4803F0BCFEBC
S315080058001E4B1F4A1A601D4B00225A601B4B002272
S315080058109A601A4B0022DA60184B80221A61174BDD
S315080058204FF480725A61154B4FF480629A61134B9C
S315080058302022DA61114B4FF400521A620F4803F026
S31508005840EBF90346002B01D0FFF746FF7B680B4AAE
S31508005850DA640A4A7B68936200220521122002F064
S31508005860F4FD122002F00DFE00BF8037BD4680BD54
S31508005870000004500010024000040048D402002032
S315080058803004024080B58AB000AF786007F114038F
S3150800589000221A605A609A60DA601A617B681B688F
S315080058A0284A934249D1284B9B6D274A43F00073F7
S315080058B09365254B9B6D03F000733B613B69224B57
S315080058C0DB6C214A43F00103D3641F4BDB6C03F006
S315080058D00103FB60FB684FF4C0537B610223BB6185
S315080058E00023FB6103233B6209237B6207F1140350
S315080058F019464FF0904003F03FFE00220521132081
S3150800590002F0A3FD132002F0BCFD0022052114209D
S3150800591002F09BFD142002F0B4FD0022052115209B
S3150800592002F093FD152002F0ACFD00220521162099
S3150800593002F08BFD162002F0A4FD00BF2837BD46F5
S3150800594080BD00BF006400400010024080B485B0EE
S3150800595000AF78607B681B680A4A93420BD10A4BF2
S315080059609B6C094A43F480539364074B9B6C03F47E
S315080059708053FB60FB6800BF1437BD465DF8047BA7
S31508005980704700BF003002400010024080B58AB060
S3150800599000AF786007F1140300221A605A609A6013
S315080059A0DA601A617B681B68154A934224D1154B45
S315080059B09B6D144A43F000539365124B9B6D03F09D
S315080059C000533B613B690F4BDB6C0E4A43F0010306
S315080059D0D3640C4BDB6C03F00103FB60FB681023FC
S315080059E07B610323BB610023FB6107F1140319469E
S315080059F04FF0904003F0C0FD00BF2837BD4680BD7C
S31508005A00007400400010024080B59EB000AF786078
S31508005A1007F1640300221A605A609A60DA601A6114
S31508005A2007F110035422002118460CF08DFC7B6800
S31508005A301B681F4A934237D140233B610023FB630F
S31508005A4007F11003184604F035FF0346002B01D072
S31508005A50FFF742FE174BDB6C164A43F00103D3648B
S31508005A60144BDB6C03F00103FB60FB684FF4C06367
S31508005A707B661223BB660023FB6603233B6704236E
S31508005A807B6707F1640319464FF0904003F074FDF5
S31508005A90084B9B6D074A43F400139365054B9B6DB2
S31508005AA003F40013BB60BB6800BF7837BD4680BDF2
S31508005AB0005400400010024080B58AB000AF7860FC
S31508005AC007F1140300221A605A609A60DA601A61B4
S31508005AD07B681B68454A934240F08380444B1B6EA3
S31508005AE0434A43F480531366414B1B6E03F48053B9
S31508005AF03B613B693E4BDB6C3D4A43F00103D36493
S31508005B003B4BDB6C03F00103FB60FB68E0237B6126
S31508005B100223BB610023FB6103233B6205237B62EF
S31508005B2007F1140319464FF0904003F025FD314B59
S31508005B30314A1A602F4B01225A602E4B00229A6076
S31508005B402C4B0022DA602B4B80221A61294B00224B
S31508005B505A61284B00229A61264B0022DA61254BAE
S31508005B6000221A62234803F057F80346002B01D097
S31508005B70FFF7B2FD7B681F4A9A651E4A7B689362E7
S31508005B801E4B1F4A1A601D4B01225A601B4B1022DE
S31508005B909A601A4B0022DA60184B80221A61174B5A
S31508005BA000225A61154B00229A61144B0022DA61D1
S31508005BB0124B00221A62114803F02EF80346002BF6
S31508005BC001D0FFF789FD7B680C4A5A650B4A7B684A
S31508005BD0936200220521232002F037FC232002F0DD
S31508005BE050FC00BF2837BD4680BD00BF00300140CD
S31508005BF000100240440400201C0002408C040020CF
S31508005C003000024080B400AFFEE780B400AFFEE784
S31508005C1080B400AFFEE780B400AFFEE780B400AF03
S31508005C20FEE780B400AF00BFBD465DF8047B704751
S31508005C3080B500AF00F0FCF80BF0D2F80346012B54
S31508005C4001D00CF0A9F800BF80BD000080B500AFF8
S31508005C50024803F03AF900BF80BD00BF44040020A3
S31508005C6080B500AF024803F030F900BF80BD00BF21
S31508005C708C04002080B500AF024800F0E9FC00BFA4
S31508005C8080BD00BF7002002080B500AF024802F058
S31508005C90C6F800BF80BD00BF1C03002080B500AF5A
S31508005CA0024802F0BCF800BF80BD00BF1C030020FC
S31508005CB080B500AF024802F0B2F800BF80BD00BF51
S31508005CC01C03002080B500AF024802F0A8F800BF08
S31508005CD080BD00BF1C03002080B500AF024805F058
S31508005CE001FB00BF80BD00BFE003002080B500AF08
S31508005CF0024803F0EAF800BF80BD00BFD4020020C6
S31508005D0080B400AF154BD3F88830144A43F47003B7
S31508005D10C2F88830124B1B68114A43F0010313601E
S31508005D200F4B00229A600E4B1B680D4A23F0A853AE
S31508005D3023F4102313600A4B4FF48052DA60084BA1
S31508005D401B68074A23F480231360054B00229A61D7
S31508005D5000BFBD465DF8047B704700BF00ED00E05C
S31508005D600010024080B584B000AFF860B9601346F1
S31508005D70FB80FB881A46F968B8680CF0D7FA00BFAA
S31508005D801037BD4680BD80B582B000AF0023FB71D9
S31508005D90032002F04FFB0F2000F00EF80346002BFD
S31508005DA002D00123FB7101E0FFF79CFCFB79184642
S31508005DB00837BD4680BD000080B584B000AF786066
S31508005DC00023FB73174B1B78002B23D0164B1A683E
S31508005DD0144B1B7819464FF47A73B3FBF1F3B2FBF5
S31508005DE0F3F3184602F05FFB0346002B0FD17B68DE
S31508005DF00F2B09D8002279684FF0FF3002F025FBF7
S31508005E000A4A7B68136007E00123FB7304E0012359
S31508005E10FB7301E00123FB73FB7B18461037BD4675
S31508005E2080BD00BFB0000020A8000020AC00002004
S31508005E3080B400AF064B1B781A46064B1B68134402
S31508005E40044A136000BFBD465DF8047B704700BF77
S31508005E50B0000020D804002080B400AF034B1B68B4
S31508005E601846BD465DF8047B704700BFD80400207D
S31508005E7080B584B000AF7860FFF7EEFFB8607B6846
S31508005E80FB60FB68B3F1FF3F05D00A4B1B781A4647
S31508005E90FB681344FB6000BFFFF7DEFF0246BB68E2
S31508005EA0D31AFA689A42F7D800BF00BF1037BD4622
S31508005EB080BD00BFB000002080B483B000AF78601A
S31508005EC039607B689B6823F47C123B681A437B68BD
S31508005ED09A6000BF0C37BD465DF8047B704780B4F6
S31508005EE083B000AF786039607B689B6823F0E07206
S31508005EF03B681A437B689A6000BF0C37BD465DF85D
S31508005F00047B704780B483B000AF78607B689B6879
S31508005F1003F0E07318460C37BD465DF8047B7047FE
S31508005F2080B487B000AFF860B9607A603B60FB6800
S31508005F3060331A46BB689B0013447B617B691A6809
S31508005F40084B13407A6802F0F8413A680A4313434B
S31508005F5043F000427B691A6000BF1C37BD465DF8F6
S31508005F60047B704700F0FF0380B485B000AF78600B
S31508005F7039607B6860331A463B689B001344FB60B4
S31508005F80FB681B6803F0F84318461437BD465DF8EE
S31508005F90047B704780B487B000AFF860B9607A6058
S31508005FA0FB6860331A46BB689B0013447B617B69B8
S31508005FB01B6823F000427B681A437B691A6000BF9E
S31508005FC01C37BD465DF8047B704780B483B000AFCC
S31508005FD078607B68DB6803F44063002B01D10123FA
S31508005FE000E0002318460C37BD465DF8047B704771
S31508005FF080B487B000AFF860B9607A60FB68303368
S315080060001A46BB681B0A9B0003F00C0313447B610A
S315080060107B691A68BB6803F01F031F2101FA03F3A3
S31508006020DB431A407B689B0E03F01F01BB6803F035
S315080060301F0301FA03F31A437B691A6000BF1C3772
S31508006040BD465DF8047B704780B483B000AF7860C6
S315080060507B68DB6C03F0C003002B01D1012300E051
S31508006060002318460C37BD465DF8047B704780B49C
S3150800607087B000AFF860B9607A60FB6814331A46D7
S31508006080BB685B0E9B0003F0040313447B617B69CA
S315080060901A68BB681B0D03F01F03072101FA03F3F7
S315080060A0DB431A40BB681B0D03F01F03796801FA2E
S315080060B003F31A437B691A6000BF1C37BD465DF8B7
S315080060C0047B704780B485B000AFF860B9607A6029
S315080060D0FB68D3F8B020BB68C3F31203DB431A404E
S315080060E07B6803F018030849D940BB680B40C3F323
S315080060F012031A43FB68C3F8B02000BF1437BD4625
S315080061005DF8047B704700BFFFFF070080B483B0CB
S3150800611000AF78607B689B6823F0204323F03F0339
S315080061207A68936000BF0C37BD465DF8047B7047FC
S3150800613080B483B000AF78607B689B6803F0005337
S31508006140B3F1005F01D1012300E0002318460C37A4
S31508006150BD465DF8047B704780B483B000AF7860B5
S315080061607B689B6823F0104323F03F0343F080527B
S315080061707B689A6000BF0C37BD465DF8047B7047A4
S3150800618080B483B000AF78607B689B6803F0805367
S31508006190B3F1805F01D1012300E0002318460C37D4
S315080061A0BD465DF8047B704780B483B000AF786065
S315080061B07B689B6823F0004323F03F0343F001020A
S315080061C07B689A6000BF0C37BD465DF8047B704754
S315080061D080B483B000AF78607B689B6823F0004387
S315080061E023F03F0343F002027B689A6000BF0C3736
S315080061F0BD465DF8047B704780B483B000AF786015
S315080062007B689B6803F00103012B01D1012300E0A1
S31508006210002318460C37BD465DF8047B704780B4EA
S3150800622083B000AF78607B689B6803F00203022B9B
S3150800623001D1012300E0002318460C37BD465DF85E
S31508006240047B704780B483B000AF78607B689B6836
S3150800625023F0004323F03F0343F004027B689A606F
S3150800626000BF0C37BD465DF8047B704780B483B029
S3150800627000AF78607B689B6803F00403042B01D1A8
S31508006280012300E0002318460C37BD465DF8047B61
S31508006290704780B483B000AF78607B689B6803F072
S315080062A00803082B01D1012300E0002318460C3708
S315080062B0BD465DF8047B704780B588B000AF78604E
S315080062C00023FB770023BB607B68002B01D10123E9
S315080062D02CE17B681B69002B7B685B6D002B09D161
S315080062E07868FFF727FA7B6800229A657B680022A0
S315080062F083F850207B681B681846FFF719FF03468A
S31508006300002B04D07B681B681846FFF7FFFE7B68E6
S315080063101B681846FFF734FF0346002B15D17B6828
S315080063201B681846FFF718FF824B1B689B09824AB1
S31508006330A2FB03239B0901335B00BB6002E0BB6839
S31508006340013BBB60BB68002BF9D17B681B6818460C
S31508006350FFF716FF0346002B0DD17B685B6D43F0F4
S3150800636010027B685A657B689B6D43F001027B6867
S315080063709A650123FB777B681B681846FFF776FF4B
S3150800638078617B685B6D03F01003002B40F0C580D5
S315080063907B69002B40F0C1807B685B6D23F48173B9
S315080063A043F002027B685A657B681B681846FFF74C
S315080063B023FF0346002B0BD16048FFF71DFF03465A
S315080063C0002B05D17B685B6819465D48FFF774FDAD
S315080063D07B685B7E5A037B685B6B1A437B68DB686A
S315080063E01A437B689B681A437B6893F820301B0422
S315080063F01343BB617B6893F82030012B06D17B6879
S315080064005B6A013B5B04BA691343BB617B689B6AA1
S31508006410002B09D07B689B6A03F470727B68DB6A81
S315080064201343BA691343BB617B681B68DA68454B3B
S3150800643013407A681268B9690B43D3607B681B6896
S315080064401846FFF713FF38617B681B681846FFF785
S3150800645020FFF8603B69002B3DD1FB68002B3AD141
S315080064607B681B7E9A037B6893F830305B00134386
S31508006470BB617B681B68DB6823F4804323F0020357
S315080064807A681268B9690B43D3607B6893F8383029
S31508006490012B18D17B681B681B6923F4FF6323F063
S315080064A004037A68D16B7A68126C11437A68526C65
S315080064B011437A68926C0A431A437B681B6842F058
S315080064C001021A6107E07B681B681A697B681B680A
S315080064D022F001021A617B681B69012B0CD17B68CB
S315080064E01B681B6B23F00F017B68DB695A1E7B68F0
S315080064F01B680A431A6307E07B681B681A6B7B688C
S315080065001B6822F00F021A637B685B6D23F0030396
S3150800651043F001027B685A6507E07B685B6D43F0D0
S3150800652010027B685A650123FB77FB7F18462037E4
S31508006530BD4680BDA8000020632D3E05000004501E
S315080065400003045007C0F0FF80B586B000AFF860BE
S31508006550B9607A60FB681B681846FFF787FE034632
S31508006560002B67D1FB6893F85030012B01D1022329
S3150800657063E0FB68012283F85020F86800F006FE05
S315080065800346FB75FB7D002B4FD1FB685B6D23F43F
S31508006590706323F0010343F48072FB685A65FB6855
S315080065A05B6D03F48053002B06D0FB689B6D23F0CC
S315080065B00602FB689A6502E0FB6800229A65FB689A
S315080065C0DB6C204ADA62FB68DB6C1F4A1A63FB68DD
S315080065D0DB6C1E4A5A63FB681B681C221A60FB6840
S315080065E0002283F85020FB681B685A68FB681B6802
S315080065F042F010025A60FB681B68DA68FB681B6881
S3150800660042F00102DA60FB68D86CFB681B6840330D
S315080066101946BA687B6802F0B7FB0346FB75FB6848
S315080066201B681846FFF70EFE06E0FB68002283F893
S31508006630502001E00223FB75FB7D18461837BD463E
S3150800664080BD00BF577300082F7400084B740008FC
S3150800665080B588B000AF78600023FB617B681B6853
S315080066601B68BB617B681B685B687B61BB6903F061
S315080066700203002B17D07B6903F00203002B12D00C
S315080066807B685B6D03F01003002B05D17B685B6D9F
S3150800669043F400627B685A65786800F0A5FF7B685A
S315080066A01B6802221A60BB6903F00403002B04D09E
S315080066B07B6903F00403002B09D1BB6903F00803C7
S315080066C0002B5ED07B6903F00803002B59D07B684A
S315080066D05B6D03F01003002B05D17B685B6D43F4FB
S315080066E000727B685A657B681B681846FFF76DFC65
S315080066F00346002B3ED07B681B68DB683B613B6921
S3150800670003F40053002B35D17B681B681B6803F024
S315080067100803082B2ED17B681B681846FFF7A6FDD1
S315080067200346002B1AD17B681B685A687B681B686E
S3150800673022F00C025A607B685B6D23F480727B68DA
S315080067405A657B685B6D03F48053002B12D17B6816
S315080067505B6D43F001027B685A650BE07B685B6DF5
S3150800676043F010027B685A657B689B6D43F0010213
S315080067707B689A657868FDF787FE7B681B680C223C
S315080067801A60BB6903F02003002B04D07B6903F071
S315080067902003002B09D1BB6903F04003002B72D0FC
S315080067A07B6903F04003002B6DD07B685B6D03F0BB
S315080067B01003002B05D17B685B6D43F400527B68A0
S315080067C05A657B681B681846FFF73EFCF8607B68CD
S315080067D01B681846FFF7F9FBB8607B681B68DB681F
S315080067E03B61FB68002B47D03B6903F00073002B25
S315080067F007D0BB68002B3FD03B6903F40053002B3E
S315080068003AD17B681B681B6803F04003402B33D1E1
S315080068103B6903F40013002B2ED17B681B681846CE
S31508006820FFF737FD0346002B1AD17B681B685A68A9
S315080068307B681B6822F060025A607B685B6D23F4F4
S3150800684080527B685A657B685B6D03F48073002B06
S3150800685012D17B685B6D43F001027B685A650BE0D9
S315080068607B685B6D43F010027B685A657B689B6D9D
S3150800687043F001027B689A65786800F08DFE7B68B4
S315080068801B6860221A60BB6903F08003002B11D0D5
S315080068907B6903F08003002B0CD07B685B6D43F4A7
S315080068A080327B685A65786800F086F87B681B68D2
S315080068B080221A60BB6903F48073002B12D07B69AF
S315080068C003F48073002B0DD07B685B6D43F40032B4
S315080068D07B685A65786800F073FE7B681B684FF41E
S315080068E080721A60BB6903F40073002B12D07B69AF
S315080068F003F40073002B0DD07B685B6D43F4802294
S315080069007B685A65786800F065FE7B681B684FF4FB
S3150800691000721A60BB6903F01003002B2AD07B694A
S3150800692003F01003002B25D07B685B6B002B02D18C
S315080069300123FB6108E07B681B68DB6803F0010341
S31508006940002B01D00123FB61FB69012B0ED17B686B
S315080069505B6D43F480627B685A657B689B6D43F088
S3150800696002027B689A657868FDF7AEFD7B681B684E
S3150800697010221A60BB6903F48063002B18D07B6968
S3150800698003F48063002B13D07B685B6D43F480426D
S315080069907B685A657B689B6D43F008027B689A653D
S315080069A07B681B684FF480621A60786800F0FEFD09
S315080069B000BF2037BD4680BD80B483B000AF786085
S315080069C000BF0C37BD465DF8047B704780B5B6B08E
S315080069D000AF78603960002387F8D7300023FB6062
S315080069E07B6893F85030012B01D10223B9E37B6809
S315080069F0012283F850207B681B681846FFF736FC8F
S31508006A000346002B40F09E833B685B68052B24D821
S31508006A103B685B68023B032B1BD801A252F823F0A4
S31508006A20316A0008396A0008416A0008496A00089C
S31508006A303B680C225A6011E03B6812225A600DE04E
S31508006A403B6818225A6009E03B684FF480725A6026
S31508006A5004E03B6806225A6000E000BF7B681868BD
S31508006A603B6859683B681B681A46FFF7C1FA7B689A
S31508006A701B681846FFF7FAFBC7F8D0007B681B6847
S31508006A801846FFF706FCC7F8CC00D7F8D030002B1D
S31508006A9040F0A681D7F8CC30002B40F0A1817B6866
S31508006AA018683B6819683B689B681A46FFF7DFFA5F
S31508006AB03B685A697B681B68DB68DB0803F00303DD
S31508006AC05B0002FA03F3C7F8C8303B681B69042B5E
S31508006AD00AD07B6818683B6819693B681A68D7F852
S31508006AE0C830FFF71DFA7BE17B681B680021184652
S31508006AF0FFF73AFA0346C3F31203002B0AD17B6861
S31508006B001B6800211846FFF72FFA03469B0E03F071
S31508006B101F021EE07B681B6800211846FFF724FA4F
S31508006B200346C7F8BC30D7F8BC3093FAA3F3C7F8C6
S31508006B30B830D7F8B830C7F8C030D7F8C030002B0F
S31508006B4001D1202304E0D7F8C030B3FA83F3DBB2CF
S31508006B501A463B681B68C3F31203002B05D13B6832
S31508006B601B689B0E03F01F0318E03B681B68C7F8F9
S31508006B70B030D7F8B03093FAA3F3C7F8AC30D7F8EB
S31508006B80AC30C7F8B430D7F8B430002B01D1202385
S31508006B9004E0D7F8B430B3FA83F3DBB29A4206D1ED
S31508006BA07B681B68002200211846FFF7F3F97B680B
S31508006BB01B6801211846FFF7D7F90346C3F31203EA
S31508006BC0002B0AD17B681B6801211846FFF7CCF910
S31508006BD003469B0E03F01F021EE07B681B6801211B
S31508006BE01846FFF7C1F90346C7F8A430D7F8A4300A
S31508006BF093FAA3F3C7F8A030D7F8A030C7F8A8309F
S31508006C00D7F8A830002B01D1202304E0D7F8A83004
S31508006C10B3FA83F3DBB21A463B681B68C3F3120365
S31508006C20002B05D13B681B689B0E03F01F0318E079
S31508006C303B681B68C7F89830D7F8983093FAA3F3DF
S31508006C40C7F89430D7F89430C7F89C30D7F89C30FA
S31508006C50002B01D1202304E0D7F89C30B3FA83F344
S31508006C60DBB29A4206D17B681B68002201211846CE
S31508006C70FFF790F97B681B6802211846FFF774F93D
S31508006C800346C3F31203002B0AD17B681B68022153
S31508006C901846FFF769F903469B0E03F01F021EE02C
S31508006CA07B681B6802211846FFF75EF90346C7F89A
S31508006CB08C30D7F88C3093FAA3F3C7F88830D7F816
S31508006CC08830C7F89030D7F89030002B01D12023B0
S31508006CD004E0D7F89030B3FA83F3DBB21A463B6880
S31508006CE01B68C3F31203002B05D13B681B689B0E78
S31508006CF003F01F0316E03B681B68C7F88030D7F817
S31508006D00803093FAA3F3FB67FB6FC7F88430D7F894
S31508006D108430002B01D1202304E0D7F88430B3FA5D
S31508006D2083F3DBB29A4206D17B681B6800220221F4
S31508006D301846FFF72FF97B681B6803211846FFF7EB
S31508006D4013F90346C3F31203002B0AD17B681B68A9
S31508006D5003211846FFF708F903469B0E03F01F02A6
S31508006D6017E07B681B6803211846FFF7FDF8034602
S31508006D707B677B6F93FAA3F33B673B6FBB67BB6F7E
S31508006D80002B01D1202303E0BB6FB3FA83F3DBB2F8
S31508006D901A463B681B68C3F31203002B05D13B68F0
S31508006DA01B689B0E03F01F0311E03B681B68BB665C
S31508006DB0BB6E93FAA3F37B667B6EFB66FB6E002BBA
S31508006DC001D1202303E0FB6EB3FA83F3DBB29A42C8
S31508006DD006D17B681B68002203211846FFF7DAF8FC
S31508006DE07B681B681846FFF707FA0346002B40F036
S31508006DF03F817B6818683B6819683B68DB681A46F8
S31508006E00FFF760F93B68DB688E4A934240F03081B1
S31508006E107B6818683B681B68C3F31203002B0BD109
S31508006E203B681B689B0E013303F01F03092B94BFB5
S31508006E3001230023DBB219E03B681B68FB65FB6D89
S31508006E4093FAA3F3BB65BB6D3B663B6E002B01D182
S31508006E50202303E03B6EB3FA83F3DBB2013303F07E
S31508006E601F03092B94BF01230023DBB2002B79D023
S31508006E703B681B68C3F31203002B07D13B681B68EA
S31508006E809B0E01339B0603F0F84215E03B681B682E
S31508006E903B653B6D93FAA3F3FB64FB6C7B657B6DEB
S31508006EA0002B01D1202303E07B6DB3FA83F3DBB219
S31508006EB001339B0603F0F8423B681B68C3F31203D1
S31508006EC0002B09D13B681B689B0E013303F01F0397
S31508006ED0012101FA03F317E03B681B687B647B6CAE
S31508006EE093FAA3F33B643B6CBB64BB6C002B01D1E8
S31508006EF0202303E0BB6CB3FA83F3DBB2013303F060
S31508006F001F03012101FA03F342EA03013B681B68E8
S31508006F10C3F31203002B0AD13B681B689B0E01338F
S31508006F2003F01F0213465B0013441B0518E03B6879
S31508006F301B68BB63BB6B93FAA3F37B637B6BFB6337
S31508006F40FB6B002B01D1202303E0FB6BB3FA83F321
S31508006F50DBB2013303F01F0213465B0013441B0523
S31508006F600B4380E03B681B68C3F31203002B07D171
S31508006F703B681B689B0E01339B0603F0F84215E03D
S31508006F803B681B68FB62FB6A93FAA3F3BB62BB6AA6
S31508006F903B633B6B002B01D1202303E03B6BB3FA29
S31508006FA083F3DBB201339B0603F0F8423B681B68A8
S31508006FB0C3F31203002B09D13B681B689B0E0133F0
S31508006FC003F01F03012101FA03F317E03B681B686E
S31508006FD03B623B6A93FAA3F3FB61FB697B627B6ABC
S31508006FE0002B01D1202303E07B6AB3FA83F3DBB2DB
S31508006FF0013303F01F03012101FA03F342EA0301F7
S315080070003B681B68C3F31203002B0DD13B681B6852
S315080070109B0E013303F01F0213465B0013441E3B0D
S315080070201B0543F000731DE03B681B687B617B69A9
S3150800703093FAA3F33B613B69BB61BB69002B03D1A0
S31508007040202305E000007F40BB69B3FA83F3DBB277
S31508007050013303F01F0213465B0013441E3B1B0556
S3150800706043F000730B433A6892681946FEF7FFFF30
S315080070703B681A683D4B1340002B6CD03C48FEF722
S3150800708041FFC7F8C4003B681B683A4A934227D1B8
S31508007090D7F8C43003F40003002B21D17B681B68A2
S315080070A0354A934257D1D7F8C43043F400031946FA
S315080070B02F48FEF714FF314B1B689B09304AA2FB89
S315080070C003239B095A1C13465B0013449B00FB6071
S315080070D002E0FB68013BFB60FB68002BF9D13AE054
S315080070E03B681B68274A934213D1D7F8C43003F08C
S315080070F08073002B0DD17B681B681F4A93422AD1E7
S31508007100D7F8C43043F0807319461948FEF7E7FEEE
S3150800711021E03B681B681C4A93421CD1D7F8C4304F
S3150800712003F48003002B16D17B681B68124A93422E
S3150800713011D1D7F8C43043F4800319460C48FEF73A
S31508007140CEFE08E07B685B6D43F020027B685A65DB
S31508007150012387F8D7307B68002283F8502097F8F8
S31508007160D7301846D837BD4680BD00BF0000088016
S3150800717000030450000052C700000450A800002075
S31508007180632D3E05000084CB0100008080B584B0E5
S3150800719000AF78600023BB607B681B681846FFF762
S315080071A02BF80346002B69D17B681B689A68364B17
S315080071B01340002B0DD07B685B6D43F010027B6893
S315080071C05A657B689B6D43F001027B689A650123CB
S315080071D055E07B681B681846FEF7E6FF2B48FEF766
S315080071E091FE034603F40003002B13D0284B1B68BB
S315080071F09B09284AA2FB03239B095A1C13465B00DA
S3150800720013449B00BB6002E0BB68013BBB60BB68E4
S31508007210002BF9D1FEF720FEF86028E07B681B6892
S315080072201846FEF7E9FF0346002B04D17B681B6866
S315080072301846FEF7B9FFFEF70FFE0246FB68D31A9B
S31508007240022B14D97B681B681B6803F00103012B0A
S315080072500DD07B685B6D43F010027B685A657B68CE
S315080072609B6D43F001027B689A65012307E07B6802
S315080072701B681B6803F00103012BCFD100231846B6
S315080072801037BD4680BD00BF3F0000800003045094
S31508007290A8000020632D3E0580B584B000AF786055
S315080072A07B681B681846FEF7BAFFF8607B681B68A0
S315080072B01846FEF7A1FF0346002B47D0FB68002BB4
S315080072C044D17B681B689B6803F00D03012B0CD126
S315080072D07B681B681846FEF77BFF7B681B680322E2
S315080072E01A60FEF7B9FDB86029E07B685B6D43F06C
S315080072F010027B685A657B689B6D43F001027B68C8
S315080073009A65012323E0FEF7A7FD0246BB68D31A58
S31508007310022B14D97B681B689B6803F00103002BBA
S315080073200DD07B685B6D43F010027B685A657B68FD
S315080073309B6D43F001027B689A65012307E07B6831
S315080073401B689B6803F00103002BDCD10023184659
S315080073501037BD4680BD80B584B000AF78607B68C5
S315080073609B6AFB60FB685B6D03F05003002B4BD1F7
S31508007370FB685B6D43F40072FB685A65FB681B6823
S315080073801B6803F00803002B21D0FB681B6818460E
S31508007390FEF71BFE0346002B32D0FB681B68DB6832
S315080073A003F40053002B2BD1FB685B6D23F480722A
S315080073B0FB685A65FB685B6D03F48053002B1FD18D
S315080073C0FB685B6D43F00102FB685A6518E0FB68D1
S315080073D01B68DB6803F00203002B11D1FB685B6DA9
S315080073E023F48072FB685A65FB685B6D03F480536F
S315080073F0002B05D1FB685B6D43F00102FB685A65FB
S31508007400F868FDF741F80EE0FB685B6D03F01003C2
S31508007410002B03D0F868FDF757F804E0FB68DB6C2F
S315080074205B6B7868984700BF1037BD4680BD80B54E
S3150800743084B000AF78607B689B6AFB60F868FDF7EC
S3150800744033F800BF1037BD4680BD80B584B000AFA5
S3150800745078607B689B6AFB60FB685B6D43F0400263
S31508007460FB685A65FB689B6D43F00402FB689A65E6
S31508007470F868FDF729F800BF1037BD4680BD80B40F
S3150800748083B000AF786039607B689B6823F040431F
S3150800749023F03F033A6802F08042134343F0004268
S315080074A07B689A6000BF0C37BD465DF8047B704761
S315080074B080B483B000AF78607B689B6803F00043B4
S315080074C0B3F1004F01D1012300E0002318460C3721
S315080074D0BD465DF8047B704780B584B000AF786020
S315080074E039600023BB607B6893F85030012B01D1CB
S315080074F002234DE07B68012283F850207868FFF765
S31508007500CBFE0346FB73FB7B002B36D17B685B6D9A
S3150800751023F4885323F0020343F002027B685A657A
S315080075207B681B6839681846FFF7A9FF14E0BB6833
S315080075300133BB60BB68B3F5912F0DD37B685B6DD8
S3150800754023F0120343F010027B685A657B68002219
S3150800755083F8502001231BE07B681B681846FFF759
S31508007560A7FF0346002BE2D17B685B6D23F003037C
S3150800757043F001027B685A6505E07B685B6D43F062
S3150800758010027B685A657B68002283F85020FB7BD3
S3150800759018461037BD4680BD80B483B000AF78600A
S315080075A000BF0C37BD465DF8047B704780B483B0D6
S315080075B000AF786000BF0C37BD465DF8047B7047A6
S315080075C080B483B000AF786000BF0C37BD465DF865
S315080075D0047B704780B483B000AF786000BF0C3777
S315080075E0BD465DF8047B704780B483B000AF786011
S315080075F000BF0C37BD465DF8047B704780B584B084
S3150800760000AF78607B68002B01D10123EDE07B6831
S3150800761093F82030DBB2002B02D17868FEF732F9F6
S315080076207B681B681A687B681B6842F001021A604F
S31508007630FEF712FCF86012E0FEF70EFC0246FB6845
S31508007640D31A0A2B0BD97B685B6A43F400327B6832
S315080076505A627B68052283F820200123C5E07B68EF
S315080076601B685B6803F00103002BE5D07B681B6889
S315080076701A687B681B6822F002021A60FEF7ECFBA8
S31508007680F86012E0FEF7E8FB0246FB68D31A0A2BFD
S315080076900BD97B685B6A43F400327B685A627B6865
S315080076A0052283F8202001239FE07B681B685B681E
S315080076B003F00203002BE5D17B681B7E012B08D162
S315080076C07B681B681A687B681B6842F080021A6030
S315080076D007E07B681B681A687B681B6822F08002D3
S315080076E01A607B685B7E012B08D17B681B681A6869
S315080076F07B681B6842F040021A6007E07B681B68DB
S315080077001A687B681B6822F040021A607B689B7EB9
S31508007710012B08D17B681B681A687B681B6842F0D6
S3150800772020021A6007E07B681B681A687B681B687A
S3150800773022F020021A607B68DB7E012B08D17B6869
S315080077401B681A687B681B6822F010021A6007E03B
S315080077507B681B681A687B681B6842F010021A600F
S315080077607B681B7F012B08D17B681B681A687B68BE
S315080077701B6842F008021A6007E07B681B681A68F3
S315080077807B681B6822F008021A607B685B7F012B06
S3150800779008D17B681B681A687B681B6842F004027C
S315080077A01A6007E07B681B681A687B681B6822F00A
S315080077B004021A607B689A687B68DB681A437B68F0
S315080077C01B691A437B685B6942EA03017B685B684D
S315080077D05A1E7B681B680A43DA617B6800225A6274
S315080077E07B68012283F82020002318461037BD46FF
S315080077F080BD80B487B000AF786039607B681B684D
S315080078007B617B6893F82030FB74FB7C012B03D0EB
S31508007810FB7C022B40F0AA807B69D3F8003243F048
S3150800782001027B69C3F800223B685B6903F01F030A
S31508007830012202FA03F3FB607B69D3F81C22FB687A
S31508007840DB431A407B69C3F81C223B68DB69002BC3
S3150800785023D17B69D3F80C22FB68DB431A407B698A
S31508007860C3F80C223B68DB6819043B685B689BB26B
S315080078703A68526919437B69483243F832103B68C3
S315080078809B6819043B681B689AB23B685B690A43A4
S3150800789079694833DB000B445A603B68DB69012B86
S315080078A022D17B69D3F80C22FB681A437B69C3F89B
S315080078B00C223B681B6819043B685B689BB23A68F4
S315080078C0526919437B69483243F832103B689B6812
S315080078D019043B68DB689AB23B685B690A437969B5
S315080078E04833DB000B445A603B689B69002B09D17F
S315080078F07B69D3F80422FB68DB431A407B69C3F82B
S31508007900042207E07B69D3F80422FB681A437B69E3
S31508007910C3F804223B681B69002B09D17B69D3F89D
S315080079201422FB68DB431A407B69C3F8142207E07C
S315080079307B69D3F81422FB681A437B69C3F81422BF
S315080079403B681B6A012B07D17B69D3F81C22FB68AD
S315080079501A437B69C3F81C227B69D3F8003223F0EB
S3150800796001027B69C3F80022002306E07B685B6A94
S3150800797043F480227B685A62012318461C37BD46A9
S315080079805DF8047B704780B584B000AF78607B688B
S3150800799093F82030DBB2012B2ED17B68022283F8C4
S315080079A020207B681B681A687B681B6822F0010226
S315080079B01A60FEF751FAF86012E0FEF74DFA024631
S315080079C0FB68D31A0A2B0BD97B685B6A43F400322F
S315080079D07B685A627B68052283F82020012312E01F
S315080079E07B681B685B6803F00103002BE5D17B68A5
S315080079F000225A62002306E07B685B6A43F4002291
S31508007A007B685A62012318461037BD4680BD80B48C
S31508007A1089B000AFF860B9607A603B60FB6893F89C
S31508007A202030FB77FB681B689B68BB61FB7F012BDB
S31508007A3003D0FB7F022B40F0AD80BB6903F0806367
S31508007A40002B0AD1BB6903F00063002B05D1BB6983
S31508007A5003F08053002B00F09580BB691B0E03F0E2
S31508007A6003037B6101227B699A403B681A60BB6805
S31508007A709B68002B0DD1BB681B685A05BB68DB6881
S31508007A80F96809681A437B6918331B010B441A60A5
S31508007A900FE0BB685B68DA00BB689B681A43BB6883
S31508007AA0DB68F96809681A437B6918331B010B44BC
S31508007AB01A60FB681968BB681A697B6918331B0169
S31508007AC00B4404331A60BB681B7D012B11D1FB687C
S31508007AD01A687B6918331B01134404331B68FA6858
S31508007AE0116843F480727B6918331B010B44043315
S31508007AF01A607B6807331B781A067B6806331B787F
S31508007B001B041A437B6805331B781B0213437A68E8
S31508007B10043212781046FA68116843EA00027B6953
S31508007B201B010B4403F5C6731A607B6803331B7885
S31508007B301A067B6802331B781B041A437B680133D9
S31508007B401B781B0213437A6812781046FA68116884
S31508007B5043EA00027B691B010B4403F5C4731A60F0
S31508007B60FB681A687B6918331B0113441B68FA689B
S31508007B70116843F001027B6918331B010B441A6034
S31508007B8000230EE0FB685B6A43F40012FB685A6246
S31508007B90012306E0FB685B6A43F48022FB685A62AD
S31508007BA0012318462437BD465DF8047B704780B428
S31508007BB087B000AFF860B9607A603B60FB6893F8FD
S31508007BC02030FB75FB7D012B03D0FB7D022B40F09B
S31508007BD0F380BB68002B0ED1FB681B68DB6803F0DB
S31508007BE00303002B16D1FB685B6A43F40012FB689B
S31508007BF05A620123E7E0FB681B681B6903F003036D
S31508007C00002B07D1FB685B6A43F40012FB685A62D3
S31508007C100123D8E0FB681A68BB681B331B011344B1
S31508007C201B6803F004027B689A607B689B68002BDC
S31508007C300CD1FB681A68BB681B331B0113441B680D
S31508007C405B0DC3F30A027B681A600BE0FB681A68CF
S31508007C50BB681B331B0113441B68DB0823F0604217
S31508007C607B685A60FB681A68BB681B331B011344A0
S31508007C701B6803F002027B68DA60FB681A68BB6857
S31508007C801B331B01134404331B6803F00F027B6884
S31508007C901A61FB681A68BB681B331B01134404335B
S31508007CA01B681B0ADAB27B689A61FB681A68BB68AC
S31508007CB01B331B01134404331B681B0C9AB27B68E5
S31508007CC05A61FB681A68BB681B01134403F5DC7329
S31508007CD01B68DAB23B681A70FB681A68BB681B0136
S31508007CE0134403F5DC731B681A0A3B680133D2B2E6
S31508007CF01A70FB681A68BB681B01134403F5DC732A
S31508007D001B681A0C3B680233D2B21A70FB681A68F1
S31508007D10BB681B01134403F5DC731B681A0E3B682A
S31508007D200333D2B21A70FB681A68BB681B01134486
S31508007D3003F5DE731A683B680433D2B21A70FB681F
S31508007D401A68BB681B01134403F5DE731B681A0A1D
S31508007D503B680533D2B21A70FB681A68BB681B0108
S31508007D60134403F5DE731B681A0C3B680633D2B25C
S31508007D701A70FB681A68BB681B01134403F5DE73A7
S31508007D801B681A0E3B680733D2B21A70BB68002B01
S31508007D9008D1FB681B68DA68FB681B6842F020029A
S31508007DA0DA6007E0FB681B681A69FB681B6842F023
S31508007DB020021A61002306E0FB685B6A43F480220E
S31508007DC0FB685A62012318461C37BD465DF8047BDA
S31508007DD0704780B485B000AF786039607B6893F8E7
S31508007DE02030FB73FB7B012B02D0FB7B022B09D1D6
S31508007DF07B681B6859697B681B683A680A435A613D
S31508007E00002306E07B685B6A43F480227B685A623B
S31508007E10012318461437BD465DF8047B704780B5C4
S31508007E208AB000AF786000237B627B681B685B6959
S31508007E303B627B681B685B68FB617B681B689B68A9
S31508007E40BB617B681B68DB687B617B681B681B6999
S31508007E503B617B681B689B69FB603B6A03F0010317
S31508007E60002B7CD0BB6903F00103002B23D07B6871
S31508007E701B6801229A60BB6903F00203002B03D03A
S31508007E80786800F083F916E0BB6903F00403002B59
S31508007E9004D07B6A43F400637B620CE0BB6903F0A1
S31508007EA00803002B04D07B6A43F480537B6202E00C
S31508007EB0786800F089F9BB6903F48073002B24D035
S31508007EC07B681B684FF480729A60BB6903F4007381
S31508007ED0002B03D0786800F063F916E0BB6903F459
S31508007EE08063002B04D07B6A43F400537B620CE06A
S31508007EF0BB6903F40063002B04D07B6A43F4804318
S31508007F007B6202E0786800F069F9BB6903F48033A4
S31508007F10002B24D07B681B684FF480329A60BB69BB
S31508007F2003F40033002B03D0786800F043F916E019
S31508007F30BB6903F48023002B04D07B6A43F4004317
S31508007F407B620CE0BB6903F40023002B04D07B6A38
S31508007F5043F480337B6202E0786800F049F93B6AB3
S31508007F6003F00803002B0CD07B6903F01003002BE9
S31508007F7007D07B6A43F400737B627B681B68102218
S31508007F80DA603B6A03F00403002B0BD07B6903F02D
S31508007F900803002B06D07B681B680822DA6078681D
S31508007FA000F030F93B6A03F00203002B09D07B6826
S31508007FB01B68DB6803F00303002B02D07868FCF724
S31508007FC0CFFB3B6A03F04003002B0CD03B6903F060
S31508007FD01003002B07D07B6A43F480637B627B68BF
S31508007FE01B6810221A613B6A03F02003002B0BD092
S31508007FF03B6903F00803002B06D07B681B68082240
S315080080001A61786800F012F93B6A03F01003002B36
S3150800801009D07B681B681B6903F00303002B02D099
S31508008020786800F0F9F83B6A03F40033002B0BD0AC
S31508008030FB6903F01003002B06D07B681B6810222F
S315080080405A60786800F0FCF83B6A03F48033002B2A
S315080080500BD0FB6903F00803002B06D07B681B686E
S3150800806008225A60786800F0F5F83B6A03F4004382
S31508008070002B7BD0FB6903F00403002B72D03B6A0C
S3150800808003F48073002B08D0FB6803F00103002B70
S3150800809003D07B6A43F001037B623B6A03F40073F7
S315080080A0002B08D0FB6803F00203002B03D07B6A81
S315080080B043F002037B623B6A03F48063002B08D01B
S315080080C0FB6803F00403002B03D07B6A43F0040328
S315080080D07B623B6A03F40063002B43D0FB6803F022
S315080080E07003002B3ED0FB6803F07003602B2BD087
S315080080F0602B2ED8502B22D0502B2AD8402B19D0A3
S31508008100402B26D8302B10D0302B22D8102B02D05B
S31508008110202B05D01DE07B6A43F008037B6219E03B
S315080081207B6A43F010037B6214E07B6A43F020030A
S315080081307B620FE07B6A43F040037B620AE07B6A5E
S3150800814043F080037B6205E07B6A43F480737B62BD
S3150800815000E000BF7B681B689A697B681B6822F091
S3150800816070029A617B681B6804225A607B6A002B3E
S3150800817008D07B685A6A7B6A1A437B685A627868B1
S31508008180FCF71EFB00BF2837BD4680BD80B483B010
S3150800819000AF786000BF0C37BD465DF8047B7047BA
S315080081A080B483B000AF786000BF0C37BD465DF879
S315080081B0047B704780B483B000AF786000BF0C378B
S315080081C0BD465DF8047B704780B483B000AF786025
S315080081D000BF0C37BD465DF8047B704780B483B09A
S315080081E000AF786000BF0C37BD465DF8047B70476A
S315080081F080B483B000AF786000BF0C37BD465DF829
S31508008200047B704780B483B000AF786000BF0C373A
S31508008210BD465DF8047B704780B483B000AF7860D4
S3150800822000BF0C37BD465DF8047B704780B483B049
S3150800823000AF786000BF0C37BD465DF8047B704719
S3150800824080B483B000AF786000BF0C37BD465DF8D8
S31508008250047B704780B483B000AF786000BF0C37EA
S31508008260BD465DF8047B704780B485B000AF786082
S315080082707B6803F00703FB600C4BDB68BB60BA68DE
S315080082804FF6FF031340BB60FB681A02BB68134333
S3150800829043F0BF6343F40033BB60044ABB68D36052
S315080082A000BF1437BD465DF8047B704700ED00E05B
S315080082B080B400AF044BDB681B0A03F007031846BB
S315080082C0BD465DF8047B704700ED00E080B483B0DE
S315080082D000AF0346FB7197F90730002B0BDBFB79E0
S315080082E003F01F02074997F907305B09012000FAD6
S315080082F002F241F8232000BF0C37BD465DF8047B27
S31508008300704700BF00E100E080B483B000AF0346C9
S315080083103960FB7197F90730002B0ADB3B68DAB244
S315080083200C4997F907301201D2B20B4483F800239F
S315080083300AE03B68DAB20849FB7903F00F03043B0D
S315080083401201D2B20B441A7600BF0C37BD465DF84F
S31508008350047B704700E100E000ED00E080B489B0DE
S3150800836000AFF860B9607A60FB6803F00703FB6149
S31508008370FB69C3F10703042B28BF0423BB61FB6910
S315080083800433062B02D9FB69033B00E000237B611B
S315080083904FF0FF32BB6902FA03F3DA43BB681A40AF
S315080083A07B699A404FF0FF317B6901FA03F3D943A1
S315080083B07B680B40134318462437BD465DF8047B9B
S315080083C07047000080B400AFBFF34F8F00BF064B65
S315080083D0DB6803F4E0620449044B1343CB60BFF344
S315080083E04F8F00BF00BFFDE700ED00E00400FA056F
S315080083F080B582B000AF78607B68013BB3F1807FBF
S3150800840001D301230FE00A4A7B68013B53600F2121
S315080084104FF0FF30FFF778FF054B00229A60044BB8
S3150800842007221A60002318460837BD4680BD00BFDC
S3150800843010E000E080B582B000AF78607868FFF79A
S3150800844013FF00BF0837BD4680BD80B586B000AFB4
S315080084500346B9607A60FB7300237B61FFF728FF48
S3150800846078617A68B9687869FFF778FF024697F9FC
S315080084700F3011461846FFF747FF00BF1837BD46AD
S3150800848080BD80B582B000AF0346FB7197F907300F
S315080084901846FFF71BFF00BF0837BD4680BD80B5ED
S315080084A000AFFFF78FFF80B582B000AF78607868BD
S315080084B0FFF79EFF034618460837BD4680BD0000F5
S315080084C080B582B000AF78607B68002B01D10123AC
S315080084D054E07B685B7FDBB2002B05D17B6800220A
S315080084E01A777868FDF732FA7B6802225A777B6832
S315080084F01B79002B0CD17B681B68224A5A617B6862
S315080085001B689A687B681B6822F018029A600CE060
S315080085107B6899687B68DB681A46786800F034F8E7
S315080085200346002B01D0012328E07B685B79002BEA
S3150800853005D17B681B684FF0FF321A6104E07B683F
S315080085401B687A6812691A617B681B689B6823F046
S3150800855060017B685A697B681B680A439A607B6876
S315080085601B689B6823F080017B689A697B681B6897
S315080085700A439A607B6801225A770023184608370F
S31508008580BD4680BDB71DC10480B487B000AFF86092
S31508008590B9607A600023FB751F233B6100BF3B6906
S315080085A05A1E3A61002B09D03B6903F01F03BA68CB
S315080085B022FA03F303F00103002BF0D07B68182B93
S315080085C046D801A252F823F05786000851860008BB
S315080085D05186000851860008518600085186000811
S315080085E0518600085186000845860008518600080D
S315080085F051860008518600085186000851860008F1
S3150800860051860008518600083986000851860008F8
S3150800861051860008518600085186000851860008D0
S3150800862051860008518600082D8600083B69062BEE
S3150800863013D90123FB7510E03B69072B0FD90123DA
S31508008640FB750CE03B690F2B0BD90123FB7508E082
S315080086500123FB7506E000BF04E000BF02E000BF8F
S3150800866000E000BFFB7D002B0DD1FB681B68BA68D4
S315080086705A61FB681B689B6823F01801FB681B6836
S315080086807A680A439A60FB7D18461C37BD465DF832
S31508008690047B704780B582B000AF78607B68002B9A
S315080086A001D1012314E07B681B79DBB2002B05D1CD
S315080086B07B6800225A717868FDF768F97B680222A0
S315080086C01A717B6800221A617B6801221A710023DD
S315080086D018460837BD4680BD80B483B000AF7860C1
S315080086E039607B685B79012B01D102233BE07B680B
S315080086F001225A717B6802221A717B681B68196805
S315080087003B6803F0100301229A407B681B680A4302
S315080087101A603B68002B0FD17B681B681B6803F047
S315080087203C03042B18D17B681B685A687B681B6856
S3150800873042F001025A600FE07B681B681B6803F46D
S315080087407013B3F5802F07D17B681B685A687B685E
S315080087501B6842F002025A607B6801221A717B6824
S3150800876000225A71002318460C37BD465DF8047B73
S31508008770704780B487B000AFF860B9607A603B6034
S3150800878000237B61FB681B687B61BB68002B05D1F6
S315080087907A697B68134408337B6104E07A697B68ED
S315080087A0134414337B617B691A463B6813600023C4
S315080087B018461C37BD465DF8047B704780B588B0FF
S315080087C000AFF860B9607A600023FB61FB685B79EB
S315080087D0012B01D1022307E1FB6801225A71FB68CC
S315080087E002221A71BB681B68042B74D1FDF734FB8F
S315080087F0F8617B68002B34D111E0FDF72DFB0246AA
S31508008800FB69D31A012B0AD9FB681B6943F00802D6
S31508008810FB681A61FB6803221A710323E4E0FB680C
S315080088201B685B6B03F40043002BE6D10120FDF7C0
S315080088301FFBFB681B68BA6892691A641EE0FDF79D
S315080088400BFB0246FB69D31A012B0AD9FB681B6985
S3150800885043F00802FB681A61FB6803221A710323B6
S31508008860C2E0FB681B685B6B002BE8DB0120FDF7A9
S31508008870FFFAFB681B68BA6892695A64FB681B684A
S315080088809A6C7B6803F0100340F2FF3101FA03F398
S31508008890DB4302EA0301BB68DA697B6803F010036D
S315080088A09A40FB681B680A439A64FB681B68DA6C83
S315080088B07B6803F01003FF2101FA03F3DB4302EAA6
S315080088C00301BB681A6A7B6803F010039A40FB68C9
S315080088D01B680A43DA64BB681B69012B1DD1FB6858
S315080088E01B689B6BBB617B6803F010031F2202FAAF
S315080088F003F3DB43BA691340BB61BB685B697B6101
S315080089007B6803F010037A6902FA03F3BA69134322
S31508008910BB61FB681B68BA699A63FB681B68DB6BFB
S31508008920BB617B6803F01003072202FA03F3DB43FB
S31508008930BA691340BB61BB681A68BB689B681A436F
S31508008940BB68DB6813437B617B6803F010037A69B5
S3150800895002FA03F3BA691343BB61FB681B68BA6979
S31508008960DA63FB681B6819687B6803F010034FF429
S31508008970804202FA03F3DA43FB681B680A401A606E
S31508008980FB681B681B68BB617B6803F0100340F635
S31508008990FC7202FA03F3DB43BA691340BB61BB6896
S315080089A05B687B617B6803F010037A6902FA03F35C
S315080089B0BA691343BB61FB681B68BA691A60FB682E
S315080089C01B6819687B6803F01003C02202FA03F3D8
S315080089D0DA43FB681B680A401A60FB6801221A71B1
S315080089E0FB6800225A71002318462037BD4680BD11
S315080089F080B58AB000AFF860B9607A60002387F85E
S31508008A002730FB68002B03D1012387F82730FDE0C8
S31508008A10FB681B79DBB2022B03D1012387F82730C9
S31508008A20F4E0FB685B79012B01D10223F0E0FB68D7
S31508008A3001225A71FB681B68DA6B7B6803F0100326
S31508008A40072101FA03F31340BB61FB681B68196829
S31508008A507B6803F01003012202FA03F3DA43FB688A
S31508008A601B680A401A60FB681B68D96B7B6803F0B1
S31508008A701003072202FA03F3DA43FB681B680A406D
S31508008A80DA63FB681B687B617B68002B03D17B6913
S31508008A9008337B6102E07B6914337B617B691A4684
S31508008AA04FF400631360FB681B6819687B6803F062
S31508008AB010034FF480429A40FB681B680A431A6009
S31508008AC010233B620823FB6137E0FB681B689A6B3F
S31508008AD07B6803F010031F2101FA03F3DB4302EA64
S31508008AE003017B6803F010033A6A9A40FB681B6827
S31508008AF00A439A630120FDF7BBF9FB681B685A6BAA
S31508008B007B6803F010034FF4804101FA03F31A401F
S31508008B107B6803F010034FF4804101FA03F39A428D
S31508008B2004D13A6AFB69D31A3B6203E03A6AFB69E5
S31508008B3013443B62FB695B08FB61FB69002BC4D1EC
S31508008B40FB681B689A6B7B6803F010031F2101FA08
S31508008B5003F3DB4302EA03017B6803F010033A6A76
S31508008B609A40FB681B680A439A630120FDF780F95F
S31508008B70FB681B685A6B7B6803F010034FF480414F
S31508008B8001FA03F31340002B17D13B6A01333B620A
S31508008B90FB681B689A6B7B6803F010031F2101FAB8
S31508008BA003F3DB4302EA03017B6803F010033A6A26
S31508008BB09A40FB681B680A439A63FB681B68196836
S31508008BC07B6803F010034FF4804202FA03F3DA439A
S31508008BD0FB681B680A401A60BB683A6A5A61BB6838
S31508008BE001221A61FB681B68DA6B7B6803F01003C5
S31508008BF0072101FA03F3DB4302EA0301FB681B685A
S31508008C00BA690A43DA63FB6800225A7197F8273073
S31508008C1018462837BD4680BD80B485B000AF786059
S31508008C207B68002B01D1012398E07B681B681A46F4
S31508008C304D4B9A420FD87B681B681A464B4B134418
S31508008C404B4AA2FB03231B099A007B685A647B687C
S31508008C50484A1A640EE07B681B681A46464B13445A
S31508008C60434AA2FB03231B099A007B685A647B6864
S31508008C70424A1A647B68022283F825207B681B68AF
S31508008C801B68FB60FB6823F4FF4323F07003FB605B
S31508008C907B689A687B68DB681A437B681B691A439A
S31508008CA07B685B691A437B689B691A437B68DB6947
S31508008CB01A437B681B6A1343FA681343FB607B6895
S31508008CC01B68FA681A607B689B68B3F5804F39D0D1
S31508008CD07B681B6C274A93421AD1294B1A687B6812
S31508008CE05B6C03F01C030F2101FA03F3DB432449F1
S31508008CF013400B60224B1A687B6859687B685B6C6B
S31508008D0003F01C0301FA03F31D4913430B6019E032
S31508008D101C4B1A687B685B6C03F01C030F2101FA75
S31508008D2003F3DB43174913400B60164B1A687B683D
S31508008D3059687B685B6C03F01C0301FA03F311495D
S31508008D4013430B607B680022DA637B68012283F891
S31508008D5025207B68002283F8242000231846143730
S31508008D60BD465DF8047B704707040240F8FFFDBF67
S31508008D70CDCCCCCC00000240F8FBFDBF000402407D
S31508008D80A8000240A804024080B586B000AFF8608B
S31508008D90B9607A603B600023FB75FB6893F8243062
S31508008DA0012B01D102234BE0FB68012283F8242022
S31508008DB0FB6893F82530DBB2012B3AD1FB68022217
S31508008DC083F82520FB680022DA63FB681B681A68AB
S31508008DD0FB681B6822F001021A603B687A68B9686A
S31508008DE0F86800F021F9FB681B6B002B08D0FB68BC
S31508008DF01B681A68FB681B6842F00E021A600FE0CF
S31508008E00FB681B681A68FB681B6822F004021A6074
S31508008E10FB681B681A68FB681B6842F00A021A603E
S31508008E20FB681B681A68FB681B6842F001021A6037
S31508008E3005E0FB68002283F824200223FB75FB7DEE
S31508008E4018461837BD4680BD80B584B000AF786037
S31508008E500023FB737B6893F82530DBB2022B05D021
S31508008E607B680422DA630123FB7329E07B681B68AD
S31508008E701A687B681B6822F00E021A607B681B68FA
S31508008E801A687B681B6822F001021A607B685B6CB3
S31508008E9003F01C027B681B6C012101FA02F25A607E
S31508008EA07B68012283F825207B68002283F824202A
S31508008EB07B689B6B002B03D07B689B6B7868984715
S31508008EC0FB7B18461037BD4680BD80B584B000AF21
S31508008ED078607B681B6C1B68FB607B681B681B687B
S31508008EE0BB607B685B6C03F01C0304229A40FB683A
S31508008EF01340002B26D0BB6803F00403002B21D0B7
S31508008F007B681B681B6803F02003002B07D17B686E
S31508008F101B681A687B681B6822F004021A607B6863
S31508008F205B6C03F01C027B681B6C042101FA02F2DD
S31508008F305A607B681B6B002B71D07B681B6B78684B
S31508008F4098476CE07B685B6C03F01C0302229A402E
S31508008F50FB681340002B2ED0BB6803F00203002BDE
S31508008F6029D07B681B681B6803F02003002B0BD1F4
S31508008F707B681B681A687B681B6822F00A021A60FD
S31508008F807B68012283F825207B685B6C03F01C0252
S31508008F907B681B6C022101FA02F25A607B68002288
S31508008FA083F824207B68DB6A002B38D07B68DB6A71
S31508008FB07868984733E07B685B6C03F01C030822EB
S31508008FC09A40FB681340002B2AD0BB6803F00803BD
S31508008FD0002B25D07B681B681A687B681B6822F003
S31508008FE00E021A607B685B6C03F01C027B681B6CC4
S31508008FF0012101FA02F25A607B680122DA637B6872
S31508009000012283F825207B68002283F824207B68C8
S315080090105B6B002B04D07B685B6B7868984700BF56
S3150800902000BF1037BD4680BD80B485B000AFF8607C
S31508009030B9607A603B60FB685B6C03F01C02FB68F6
S315080090401B6C012101FA02F25A60FB681B683A6838
S315080090505A60FB689B68102B08D1FB681B687A6806
S315080090609A60FB681B68BA68DA6007E0FB681B68E9
S31508009070BA689A60FB681B687A68DA6000BF1437BA
S31508009080BD465DF8047B704780B586B000AFF860D2
S31508009090B960C7E9002300233B612F4B1B78012BDE
S315080090A001D1022353E02C4B01221A704CF25030A6
S315080090B000F088F80346FB75FB7D002B43D1264B51
S315080090C000225A60254B1B6803F48063002B09D0E5
S315080090D0224B1B68214A23F4806313601E4B02222D
S315080090E01A7702E01C4B00221A77FB68002B07D17F
S315080090F0D7E90023B86800F0BDF801233B6110E00A
S31508009100FB68012B02D0FB68022B0AD13B68194683
S31508009110B86800F0D5F8FB68022B02D14FF480231B
S315080091203B614CF2503000F04DF80346FB753B6945
S31508009130002B06D0094B5A693B69DB4307491340A4
S315080091404B6100F0CFF9044B00221A70FB7D1846DC
S315080091501837BD4680BD00BFB4000020002002407D
S3150800916080B483B000AF0023FB710B4B5B69002B07
S315080091700BDA094B094A9A60074B094A9A60064B6B
S315080091805B69002B01DA0123FB71FB7918460C3762
S31508009190BD465DF8047B7047002002402301674501
S315080091A0AB89EFCD80B400AF054B5B69044A43F049
S315080091B00043536100231846BD465DF8047B70479B
S315080091C00020024080B584B000AF7860FCF744FE0A
S315080091D0F8600DE07B68B3F1FF3F09D0FCF73CFE71
S315080091E00246FB68D31A7A689A4201D8032336E006
S315080091F01D4B1B6903F48033002BEBD11A4B1A69FC
S315080092001A4B1340BB60BB68002B1ED0184B5A681C
S31508009210BB681343164A5360BB6803F04043002BF0
S3150800922007D0114B9A69BB6803F040430E491343B4
S315080092308B61BB6823F04043002B04D00A4ABB6805
S3150800924023F040431361012309E0074B1B6903F030
S315080092500103002B02D0044B01221A610023184691
S315080092601037BD4680BD00BF00200240FAC3020089
S31508009270B400002080B485B000AFF860C7E90023C9
S315080092800E4B5B690D4A43F001035361FB683A686C
S315080092901A60BFF36F8F00BFD7E900014FF00002D5
S315080092A04FF000030A000023F968043113460B60E7
S315080092B000BF1437BD465DF8047B704700200240A6
S315080092C080B489B000AF786039604023FB777B684B
S315080092D0BB613B687B61144B5B69134A43F480238B
S315080092E05361EFF31083FB60FB683B6172B600BF06
S315080092F07B691A68BB691A60BB690433BB617B6901
S3150800930004337B61FB7F013BFB77FB7F002BEFD1AF
S315080093103B69BB60BB6883F3108800BF00BF243776
S31508009320BD465DF8047B70470020024080B584B0D6
S3150800933000AF78603960484B1B78012B01D10223B6
S3150800934085E0454B01221A704CF25030FFF73AFF80
S315080093500346FB73FB7B002B75D13F4B00225A60FB
S315080093603E4B1B6803F40073002B13D03B4B1B6862
S3150800937003F48063002B09D0384B1B68374A23F463
S3150800938080631360344B03221A7716E0324B0122AE
S315080093901A7712E0314B1B6803F48063002B09D05F
S315080093A02E4B1B682D4A23F4806313602A4B022236
S315080093B01A7702E0284B00221A777B681B68012B74
S315080093C011D17B685B68184600F04AF84CF25030B9
S315080093D0FFF7F8FE0346FB73204B5B691F4A23F031
S315080093E0040353612DE03B684FF0FF321A607B6837
S315080093F09B68BB601DE07B685B681946B86800F02F
S315080094004DF84CF25030FFF7DDFE0346FB73134B65
S315080094105B69124A23F47E7323F002035361FB7BD4
S31508009420002B03D03B68BA681A600AE0BB680133B0
S31508009430BB607B689A687B68DB681344BA689A42A3
S31508009440D9D300F04FF8044B00221A70FB7B18465C
S315080094501037BD4680BD00BFB40000200020024082
S3150800946080B483B000AF78607B6803F00103002BFB
S3150800947005D0094B5B69084A43F004035361064B60
S315080094805B69054A43F48033536100BF0C37BD4618
S315080094905DF8047B704700BF0020024080B483B0AB
S315080094A000AF786039600E4B5B6923F47E727B6887
S315080094B0DB0003F4FF630A4913434B61084B5B69FE
S315080094C0074A43F002035361054B5B69044A43F4B8
S315080094D08033536100BF0C37BD465DF8047B704787
S315080094E00020024080B483B000AF214B1B7FFB7184
S315080094F0FB79012B02D0FB79032B17D11D4B1B6877
S315080095001C4A23F4007313601A4B1B68194A43F468
S3150800951000631360174B1B68164A23F40063136035
S31508009520144B1B68134A43F400731360FB79022B30
S3150800953002D0FB79032B11D10E4B1B680D4A43F45D
S31508009540805313600B4B1B680A4A23F4805313603D
S31508009550084B1B68074A43F480631360044B0022D8
S315080095601A7700BF0C37BD465DF8047B704700BF0D
S31508009570B40000200020024080B487B000AF7860B5
S31508009580396000237B6148E13B681A6801217B69E1
S3150800959001FA03F31340FB60FB68002B00F03A81E5
S315080095A03B685B6803F00303012B05D03B685B68E7
S315080095B003F00303022B30D17B689B683B617B6910
S315080095C05B00032202FA03F3DB433A6913403B616B
S315080095D03B68DA687B695B0002FA03F33A6913436E
S315080095E03B617B683A699A607B685B683B610122EC
S315080095F07B6902FA03F3DB433A6913403B613B6834
S315080096005B681B0903F001027B6902FA03F33A69F6
S3150800961013433B617B683A695A603B685B6803F0B1
S315080096200303032B17D07B68DB683B617B695B0010
S31508009630032202FA03F3DB433A6913403B613B68B2
S315080096409A687B695B0002FA03F33A6913433B6144
S315080096507B683A69DA603B685B6803F00303022BB0
S3150800966023D17B69DA087B68083253F822303B61DC
S315080096707B6903F007039B000F2202FA03F3DB431F
S315080096803A6913403B613B681A697B6903F0070333
S315080096909B0002FA03F33A6913433B617B69DA08D4
S315080096A07B680832396943F822107B681B683B617E
S315080096B07B695B00032202FA03F3DB433A69134032
S315080096C03B613B685B6803F003027B695B0002FA57
S315080096D003F33A6913433B617B683A691A603B684E
S315080096E05B6803F44033002B00F09480524B1B6EEA
S315080096F0514A43F0010313664F4B1B6E03F00103F7
S31508009700BB60BB684D4A7B699B08023352F823301D
S315080097103B617B6903F003039B000F2202FA03F304
S31508009720DB433A6913403B617B68B3F1904F0DD038
S315080097307B68434A934207D07B68424A934201D1E9
S31508009740022304E0072302E0012300E000237A69EC
S3150800975002F00302920093403A6913433B6137498A
S315080097607B699B0802333A6941F82320364B9B688C
S315080097703B61FB68DB433A6913403B613B685B68C6
S3150800978003F48013002B03D03A69FB6813433B614B
S315080097902D4A3B6993602C4BDB683B61FB68DB43D6
S315080097A03A6913403B613B685B6803F40013002B7E
S315080097B003D03A69FB6813433B61234A3B69D3608C
S315080097C0214B5B683B61FB68DB433A6913403B61AD
S315080097D03B685B6803F40033002B03D03A69FB68E7
S315080097E013433B61184A3B695360174B1B683B613F
S315080097F0FB68DB433A6913403B613B685B6803F4EB
S315080098008033002B03D03A69FB6813433B610E4A49
S315080098103B6913607B6901337B613B681A687B6926
S3150800982022FA03F3002B7FF4AFAE00BF00BF1C374C
S31508009830BD465DF8047B70470010024000000140F9
S3150800984000040048000800480004014080B485B0C0
S3150800985000AF78600B467B807B681A697B8813406B
S31508009860002B02D00123FB7301E00023FB73FB7B73
S3150800987018461437BD465DF8047B704780B483B03C
S3150800988000AF78600B467B8013467B707B78002B95
S3150800989003D07A887B689A6102E07A887B689A6244
S315080098A000BF0C37BD465DF8047B704780B485B0B1
S315080098B000AF78600B467B807B685B69FB607A88C3
S315080098C0FB6813401A04FB68D9437B880B401A438C
S315080098D07B689A6100BF1437BD465DF8047B704704
S315080098E080B582B000AF78607B68002B01D1012378
S315080098F081E07B6893F84130DBB2002B06D17B68A8
S31508009900002283F840207868FCF77EF87B682422DA
S3150800991083F841207B681B681A687B681B6822F0FD
S3150800992001021A607B685A687B681B6822F07062BD
S315080099301A617B681B689A687B681B6822F4004278
S315080099409A607B68DB68012B07D17B689A687B681D
S315080099501B6842F400429A6006E07B689A687B6856
S315080099601B6842F404429A607B68DB68022B04D1C8
S315080099707B681B684FF400625A607B681B685B68EB
S315080099807A68126843F0007343F4004353607B68B7
S315080099901B68DA687B681B6822F40042DA607B6819
S315080099A01A697B685B6942EA03017B689B691A024C
S315080099B07B681B680A43DA607B68D9697B681A6A20
S315080099C07B681B680A431A607B681B681A687B6891
S315080099D01B6842F001021A607B6800225A647B68A1
S315080099E0202283F841207B6800221A637B680022C4
S315080099F083F84220002318460837BD4680BD80B448
S31508009A0083B000AF786039607B6893F84130DBB289
S31508009A10202B38D17B6893F84030012B01D10223E3
S31508009A2032E07B68012283F840207B68242283F891
S31508009A3041207B681B681A687B681B6822F0010254
S31508009A401A607B681B681A687B681B6822F4805258
S31508009A501A607B681B6819687B681B683A680A4342
S31508009A601A607B681B681A687B681B6842F00102EB
S31508009A701A607B68202283F841207B68002283F8DD
S31508009A804020002300E0022318460C37BD465DF847
S31508009A90047B704780B485B000AF786039607B6816
S31508009AA093F84130DBB2202B39D17B6893F84030EC
S31508009AB0012B01D1022333E07B68012283F8402081
S31508009AC07B68242283F841207B681B681A687B68B8
S31508009AD01B6822F001021A607B681B681B68FB6022
S31508009AE0FB6823F47063FB603B681B02FA68134348
S31508009AF0FB607B681B68FA681A607B681B681A68D3
S31508009B007B681B6842F001021A607B68202283F892
S31508009B1041207B68002283F84020002300E00223CE
S31508009B2018461437BD465DF8047B704780B584B087
S31508009B3000AF78607B68002B01D1012341E07B6888
S31508009B401B684CF6CC421A607B681B6845F2555276
S31508009B501A607B681B687A6852685A607B681B685B
S31508009B607A6892689A60FCF777F9F8600FE0FCF774
S31508009B7073F90246FB68D31A312B08D97B681B6830
S31508009B80DB6803F00703002B01D0032319E07B6889
S31508009B901B68DB6803F00703002BE8D17B681B68AA
S31508009BA01A697B68DB689A4205D07B681B687A6805
S31508009BB0D2681A6104E07B681B684AF6AA221A6012
S31508009BC0002318461037BD4680BD80B483B000AF69
S31508009BD078607B681B684AF6AA221A600023184632
S31508009BE00C37BD465DF8047B7047000080B400AFB3
S31508009BF0044B1B6803F4C0631846BD465DF8047B36
S31508009C00704700BF0070004080B485B000AF786030
S31508009C107B68B3F5007F30D1234B1B6803F4C06320
S31508009C20B3F5007F38D0204B1B6823F4C0631E4A67
S31508009C3043F4007313601D4B1B68322202FB03F3C7
S31508009C401B4AA2FB03239B0C0133FB6002E0FB6863
S31508009C50013BFB60144B5B6903F48063B3F5806FCB
S31508009C6002D1FB68002BF2D10F4B5B6903F48063CA
S31508009C70B3F5806F10D103230FE00B4B1B6803F479
S31508009C80C063B3F5806F07D0074B1B6823F4C06326
S31508009C90054A43F480631360002318461437BD460B
S31508009CA05DF8047B704700BF00700040A8000020E4
S31508009CB083DE1B4380B588B000AF78607B68002BD5
S31508009CC002D1012300F002BC964B9B6803F00C03FB
S31508009CD0BB61944BDB6803F003037B617B681B68FD
S31508009CE003F01003002B00F0E480BB69002B07D0BB
S31508009CF0BB690C2B40F08B807B69012B40F0878079
S31508009D00884B1B6803F00203002B05D07B689B6910
S31508009D10002B01D10123D9E37B681A6A814B1B68A2
S31508009D2003F00803002B04D07E4B1B6803F0F003F6
S31508009D3005E07C4BD3F894301B0903F0F0039342FB
S31508009D4023D27B681B6A184600F054FD0346002B95
S31508009D5001D00123BAE3734B1B68724A43F0080328
S31508009D601360704B1B6823F0F0027B681B6A6D4911
S31508009D7013430B606B4B5B6823F47F427B68DB699C
S31508009D801B02684913434B6025E0664B1B68654A0E
S31508009D9043F008031360634B1B6823F0F0027B68EB
S31508009DA01B6A604913430B605E4B5B6823F47F4272
S31508009DB07B68DB691B025B4913434B60BB69002B5D
S31508009DC009D17B681B6A184600F014FD0346002B70
S31508009DD001D001237AE300F081FC0246514B9B68CF
S31508009DE01B0903F00F035049CB5C03F01F0322FA4B
S31508009DF003F34E4A13604E4B1B681846FBF7DCFF0D
S31508009E000346FB73FB7B002B52D0FB7B5EE37B6830
S31508009E109B69002B32D0434B1B68424A43F001032F
S31508009E201360FCF719F8386108E0FCF715F80246E4
S31508009E303B69D31A022B01D9032347E3394B1B6825
S31508009E4003F00203002BF0D0364B1B68354A43F06B
S31508009E5008031360334B1B6823F0F0027B681B6A08
S31508009E60304913430B602F4B5B6823F47F427B68B2
S31508009E70DB691B022B4913434B601AE0294B1B680D
S31508009E80284A23F001031360FBF7E6FF386108E070
S31508009E90FBF7E2FF02463B69D31A022B01D90323DB
S31508009EA014E3204B1B6803F00203002BF0D100E0FB
S31508009EB000BF7B681B6803F00103002B73D0BB69E6
S31508009EC0082B05D0BB690C2B0ED17B69032B0BD154
S31508009ED0144B1B6803F40033002B63D07B685B6864
S31508009EE0002B5FD10123F1E27B685B68B3F5803F05
S31508009EF006D10C4B1B680B4A43F48033136025E0EC
S31508009F007B685B68B3F5A02F14D1064B1B68054A1E
S31508009F1043F480231360034B1B68024A43F48033DF
S31508009F20136013E000100240702A0108A800002000
S31508009F30AC000020A04B1B689F4A23F480331360B3
S31508009F409D4B1B689C4A23F4802313607B685B68DF
S31508009F50002B13D0FBF780FF386108E0FBF77CFF86
S31508009F6002463B69D31A642B01D90323AEE2924B0E
S31508009F701B6803F40033002BF0D014E0FBF76CFFEA
S31508009F80386108E0FBF768FF02463B69D31A642B81
S31508009F9001D903239AE2884B1B6803F40033002B8C
S31508009FA0F0D100E000BF7B681B6803F00203002BBA
S31508009FB060D0BB69042B05D0BB690C2B19D17B6912
S31508009FC0022B16D17C4B1B6803F48063002B05D04B
S31508009FD07B68DB68002B01D1012377E2764B5B684F
S31508009FE023F0F8527B681B691B06734913434B60C1
S31508009FF040E07B68DB68002B23D06F4B1B686E4AFA
S3150800A00043F480731360FBF727FF386108E0FBF71A
S3150800A01023FF02463B69D31A022B01D9032355E2D3
S3150800A020654B1B6803F48063002BF0D0624B5B68BA
S3150800A03023F0F8527B681B691B065F4913434B6084
S3150800A04018E05D4B1B685C4A23F480731360FBF7CA
S3150800A05003FF386108E0FBF7FFFE02463B69D31AA7
S3150800A060022B01D9032331E2534B1B6803F48063A7
S3150800A070002BF0D17B681B6803F00803002B3CD04B
S3150800A0807B685B69002B1CD04B4BD3F894304A4A4B
S3150800A09043F00103C2F89430FBF7DEFE386108E0AE
S3150800A0A0FBF7DAFE02463B69D31A022B01D90323D2
S3150800A0B00CE2414BD3F8943003F00203002BEFD0A7
S3150800A0C01BE03D4BD3F894303B4A23F00103C2F81A
S3150800A0D09430FBF7C1FE386108E0FBF7BDFE024687
S3150800A0E03B69D31A022B01D90323EFE1324BD3F88C
S3150800A0F0943003F00203002BEFD17B681B6803F052
S3150800A1000403002B00F0A6800023FB772A4B9B6DE7
S3150800A11003F08053002B0DD1274B9B6D264A43F045
S3150800A12080539365244B9B6D03F08053BB60BB68DB
S3150800A1300123FB77214B1B6803F48073002B18D18E
S3150800A1401E4B1B681D4A43F480731360FBF784FE9D
S3150800A150386108E0FBF780FE02463B69D31A022BFA
S3150800A16001D90323B2E1154B1B6803F48073002B56
S3150800A170F0D07B689B68012B08D10F4BD3F8903041
S3150800A1800D4A43F00103C2F8903029E07B689B68CA
S3150800A190052B15D1084BD3F89030074A43F0040332
S3150800A1A0C2F89030044BD3F89030034A43F00103C9
S3150800A1B0C2F8903014E000BF001002400070004062
S3150800A1C09A4BD3F89030994A23F00103C2F890309D
S3150800A1D0964BD3F89030954A23F00403C2F8903092
S3150800A1E07B689B68002B16D0FBF736FE38610AE0C1
S3150800A1F0FBF732FE02463B69D31A41F28832934294
S3150800A20001D9032362E1894BD3F8903003F00203A6
S3150800A210002BEDD015E0FBF71FFE38610AE0FBF7CF
S3150800A2201BFE02463B69D31A41F28832934201D992
S3150800A23003234BE17D4BD3F8903003F00203002B48
S3150800A240EDD1FB7F012B05D1784B9B6D774A23F027
S3150800A250805393657B681B6803F02003002B3CD072
S3150800A2607B685B6A002B1CD0704BD3F898306F4A1A
S3150800A27043F00103C2F89830FBF7EEFD386108E0B9
S3150800A280FBF7EAFD02463B69D31A022B01D90323E1
S3150800A2901CE1664BD3F8983003F00203002BEFD08D
S3150800A2A01BE0624BD3F89830604A23F00103C2F8EA
S3150800A2B09830FBF7D1FD386108E0FBF7CDFD024683
S3150800A2C03B69D31A022B01D90323FFE0574BD3F876
S3150800A2D0983003F00203002BEFD17B689B6A002BB2
S3150800A2E000F0F3807B689B6A022B40F0C9804F4BD5
S3150800A2F0DB687B617B6903F003027B68DB6A9A4251
S3150800A3002CD17B6903F070027B681B6B013B1B0138
S3150800A3109A4223D17B6903F4FE427B685B6B1B027E
S3150800A3209A421BD17B6903F078427B689B6BDB06FC
S3150800A3309A4213D17B6903F4C0027B68DB6B5B0826
S3150800A340013B5B059A4209D17B6903F0C0627B68D1
S3150800A3501B6C5B08013B5B069A426BD0BB690C2BF6
S3150800A36062D0324B1B6803F08063002B01D00123B7
S3150800A370ACE02E4B1B682D4A23F080731360FBF765
S3150800A3806BFD386108E0FBF767FD02463B69D31AA7
S3150800A390022B01D9032399E0244B1B6803F00073B1
S3150800A3A0002BF0D1214BDA68214B13407A68D16A29
S3150800A3B07A68126B013A120111437A68526B1202DB
S3150800A3C011437A68D26B5208013A520511437A68EA
S3150800A3D0126C5208013A520611437A68926BD206F9
S3150800A3E00A4312491343CB60104B1B680F4A43F0CC
S3150800A3F0807313600D4BDB680C4A43F08073D3609F
S3150800A400FBF72AFD386108E0FBF726FD02463B69A3
S3150800A410D31A022B01D9032358E0044B1B6803F017
S3150800A4200073002BF0D050E001234FE000100240EB
S3150800A4308C809D01274B1B6803F00073002B44D1C9
S3150800A440244B1B68234A43F080731360214BDB6857
S3150800A450204A43F08073D360FBF7FEFC386108E0BE
S3150800A460FBF7FAFC02463B69D31A022B01D90323F0
S3150800A4702CE0184B1B6803F00073002BF0D024E087
S3150800A480BB690C2B1FD0134B1B68124A23F0807331
S3150800A4901360FBF7E1FC386108E0FBF7DDFC0246D8
S3150800A4A03B69D31A022B01D903230FE0094B1B681A
S3150800A4B003F00073002BF0D1064BDA680549064B0A
S3150800A4C01340CB6001E0012300E000231846203743
S3150800A4D0BD4680BD00100240FCFFEEFE80B584B08C
S3150800A4E000AF786039607B68002B01D10123E7E073
S3150800A4F0754B1B6803F007033A689A4210D9724BEA
S3150800A5001B6823F0070270493B6813430B606E4BC8
S3150800A5101B6803F007033A689A4201D00123CFE08B
S3150800A5207B681B6803F00203002B10D07B689A68CF
S3150800A530664B9B6803F0F0039A4208D9634B9B6805
S3150800A54023F0F0027B689B68604913438B607B6845
S3150800A5501B6803F00103002B4CD07B685B68032B58
S3150800A56007D15A4B1B6803F00073002B21D1012336
S3150800A570A6E07B685B68022B07D1544B1B6803F483
S3150800A5800033002B15D101239AE07B685B68002B0A
S3150800A59007D14E4B1B6803F00203002B09D1012398
S3150800A5A08EE04A4B1B6803F48063002B01D101231C
S3150800A5B086E0464B9B6823F003027B685B68434949
S3150800A5C013438B60FBF748FCF8600AE0FBF744FC92
S3150800A5D00246FB68D31A41F28832934201D9032313
S3150800A5E06EE03A4B9B6803F00C027B685B689B0045
S3150800A5F09A42EBD17B681B6803F00203002B10D04C
S3150800A6007B689A68314B9B6803F0F0039A4208D23C
S3150800A6102E4B9B6823F0F0027B689B682B491343FB
S3150800A6208B60294B1B6803F007033A689A4210D2DD
S3150800A630254B1B6823F0070223493B6813430B602D
S3150800A640214B1B6803F007033A689A4201D001239D
S3150800A65036E07B681B6803F00403002B08D01B4B0D
S3150800A6609B6823F4E0627B68DB68184913438B60B8
S3150800A6707B681B6803F00803002B09D0134B9B6803
S3150800A68023F460527B681B69DB00104913438B6017
S3150800A69000F024F802460D4B9B681B0903F00F03D4
S3150800A6A00B49CB5C03F01F0322FA03F3094A136034
S3150800A6B0094B1B681846FBF77FFB0346FB72FB7AC0
S3150800A6C018461037BD4680BD0020024000100240E3
S3150800A6D0702A0108A8000020AC00002080B489B0C8
S3150800A6E000AF0023FB610023BB613E4B9B6803F070
S3150800A6F00C033B613B4BDB6803F00303FB603B69E0
S3150800A700002B05D03B690C2B21D1FB68012B1ED1F0
S3150800A710344B1B6803F00803002B07D1314BD3F8E1
S3150800A72094301B0A03F00F03FB6105E02D4B1B68F1
S3150800A7301B0903F00F03FB612B4AFB6952F8233010
S3150800A740FB613B69002B0DD1FB69BB610AE03B69E4
S3150800A750042B02D1254BBB6104E03B69082B01D1D0
S3150800A760234BBB613B690C2B34D11E4BDB6803F0D2
S3150800A7700303BB60BB68022B03D0BB68032B03D063
S3150800A78005E01A4B7B6105E0194B7B6102E0FB692A
S3150800A7907B6100BF134BDB681B0903F0070301331A
S3150800A7A07B60104BDB681B0A03F07F037A6903FBA7
S3150800A7B002F27B68B2FBF3F37B610A4BDB685B0E44
S3150800A7C003F0030301335B003B607A693B68B2FB25
S3150800A7D0F3F3BB61BB6918462437BD465DF8047BB5
S3150800A7E0704700BF00100240802A01080024F400C8
S3150800A7F0005A620280B586B000AF786000233B61DC
S3150800A8002A4B9B6D03F08053002B03D0FFF7EEF91C
S3150800A810786114E0254B9B6D244A43F08053936579
S3150800A820224B9B6D03F08053FB60FB68FFF7DEF954
S3150800A83078611E4B9B6D1D4A23F0805393657B6997
S3150800A840B3F5007F0BD17B68802B19D97B68A02BC9
S3150800A85002D902233B6113E001233B6110E07B68C8
S3150800A860802B02D903233B610AE07B68802B02D147
S3150800A87002233B6104E07B68702B01D101233B6115
S3150800A8800B4B1B6823F0070209493B6913430B600E
S3150800A890074B1B6803F007033A699A4201D0012364
S3150800A8A000E0002318461837BD4680BD0010024058
S3150800A8B00020024080B586B000AF78600023FB74A4
S3150800A8C00023BB747B681B6803F40063002B31D03C
S3150800A8D07B68DB6BB3F5400F1AD0B3F5400F14D87D
S3150800A8E0002B09D0B3F5000F0FD15D4BDB685C4A2E
S3150800A8F043F48033D3600CE07B68043300211846A8
S3150800A90000F0CEF90346FB7403E00123FB7400E074
S3150800A91000BFFB7C002B0BD1514BD3F8883023F4B6
S3150800A92040027B68DB6B4E491343C1F8883001E06F
S3150800A930FB7CBB747B681B6803F40033002B00F0B8
S3150800A9409E8000237B74464B9B6D03F08053002B3F
S3150800A95001D1012300E00023002B0DD0404B9B6D55
S3150800A9603F4A43F0805393653D4B9B6D03F08053FC
S3150800A970BB60BB6801237B743A4B1B68394A43F4B6
S3150800A98080731360FBF768FAF86009E0FBF764FA6E
S3150800A9900246FB68D31A022B02D90323FB7405E08F
S3150800A9A0304B1B6803F48073002BEFD0FB7C002B25
S3150800A9B05AD12B4BD3F8903003F440737B617B69F3
S3150800A9C0002B1ED07B681B6D7A699A4219D0244BDE
S3150800A9D0D3F8903023F440737B61214BD3F8903041
S3150800A9E01F4A43F48033C2F890301D4BD3F8903099
S3150800A9F01B4A23F48033C2F89030194A7B69C2F89F
S3150800AA0090307B6903F00103002B16D0FBF724FA7C
S3150800AA10F8600BE0FBF720FA0246FB68D31A41F20E
S3150800AA208832934202D90323FB7406E00C4BD3F811
S3150800AA30903003F00203002BECD0FB7C002B0BD1EB
S3150800AA40074BD3F8903023F440727B681B6D04499A
S3150800AA501343C1F8903009E0FB7CBB7406E000BFE5
S3150800AA600010024000700040FB7CBB747B7C012B0D
S3150800AA7005D18A4B9B6D894A23F0805393657B6881
S3150800AA801B6803F00103002B0AD0844BD3F88830E7
S3150800AA9023F003027B681B6A80491343C1F8883098
S3150800AAA07B681B6803F00203002B0AD07B4BD3F8A4
S3150800AAB0883023F00C027B685B6A78491343C1F837
S3150800AAC088307B681B6803F02003002B0AD0734B81
S3150800AAD0D3F8883023F440627B689B6A6F49134336
S3150800AAE0C1F888307B681B6803F40073002B0AD012
S3150800AAF06A4BD3F8883023F440227B685B6B67493E
S3150800AB001343C1F888307B681B6803F48063002B05
S3150800AB100AD0624BD3F8883023F440127B689B6BCB
S3150800AB205E491343C1F888307B681B6803F040030D
S3150800AB30002B0AD0594BD3F8883023F440527B684F
S3150800AB40DB6A56491343C1F888307B681B6803F4EF
S3150800AB508073002B0AD0514BD3F8883023F4403247
S3150800AB607B681B6B4D491343C1F888307B681B68AB
S3150800AB7003F40053002B28D0484BD3F8883023F031
S3150800AB8040627B681B6C45491343C1F888307B6873
S3150800AB901B6CB3F1006F06D1404BDB683F4A43F4A8
S3150800ABA08013D36011E07B681B6CB3F1806F0CD106
S3150800ABB07B6804330121184600F072F80346FB74DB
S3150800ABC0FB7C002B01D0FB7CBB747B681B6803F401
S3150800ABD08023002B28D0314BD3F8883023F04062ED
S3150800ABE07B685B6C2D491343C1F888307B685B6CC6
S3150800ABF0B3F1006F06D1294BDB68284A43F480136A
S3150800AC00D36011E07B685B6CB3F1806F0CD17B6815
S3150800AC1004330121184600F043F80346FB74FB7C15
S3150800AC20002B01D0FB7CBB747B681B6803F4804354
S3150800AC30002B1CD0194BD3F8883023F040527B6880
S3150800AC409B6C16491343C1F888307B689B6CB3F13B
S3150800AC50805F0CD17B6804330221184600F020F887
S3150800AC600346FB74FB7C002B01D0FB7CBB747B6822
S3150800AC701B6803F40043002B0AD0084BD3F888302E
S3150800AC8023F080427B68DB6C04491343C1F88830A3
S3150800AC90BB7C18461837BD4680BD00BF0010024071
S3150800ACA080B584B000AF786039600023FB73744BBD
S3150800ACB0DB6803F00303002B18D0714BDB6803F045
S3150800ACC003027B681B689A420DD17B681B68002BC0
S3150800ACD009D06B4BDB681B0903F007035A1C7B681A
S3150800ACE05B689A4247D00123FB7344E07B681B6884
S3150800ACF0032B18D0032B25D8012B02D0022B09D001
S3150800AD0020E05F4B1B6803F00203002B1DD10123D3
S3150800AD10FB731AE05A4B1B6803F48063002B16D1A9
S3150800AD200123FB7313E0564B1B6803F40033002B17
S3150800AD300FD1534B1B6803F48023002B09D1012341
S3150800AD40FB7306E00123FB7304E000BF02E000BFCB
S3150800AD5000E000BFFB7B002B0DD1494BDB6823F0DD
S3150800AD6073027B6819687B685B68013B1B010B43B0
S3150800AD7043491343CB60FB7B002B7CD1404B1B68BC
S3150800AD803F4A23F080631360FBF766F8B86009E072
S3150800AD90FBF762F80246BB68D31A022B02D90323D3
S3150800ADA0FB7305E0364B1B6803F00063002BEFD1FD
S3150800ADB0FB7B002B5FD13B68002B10D1304B1B6906
S3150800ADC023F0784323F4FE437A68926811027A687E
S3150800ADD0D268D2060A432A4913430B6127E03B6827
S3150800ADE0012B12D1264B1B6923F4C00323F4FE431F
S3150800ADF07A68926811027A6812695208013A52050D
S3150800AE000A431F4913430B6111E01D4B1B6923F0CD
S3150800AE10C06323F4FE437A68926811027A6852691D
S3150800AE205208013A52060A43154913430B61144B5B
S3150800AE301B68134A43F080631360FBF70DF8B8608C
S3150800AE4009E0FBF709F80246BB68D31A022B02D9B8
S3150800AE500323FB7305E00A4B1B6803F00063002B12
S3150800AE60EFD0FB7B002B06D1054B1A697B689B69E3
S3150800AE70034913430B61FB7B18461037BD4680BD5B
S3150800AE800010024080B584B000AF78607B68002B64
S3150800AE9001D1012395E07B685B6A002B08D17B68AA
S3150800AEA05B68B3F5827F09D07B680022DA6105E02A
S3150800AEB07B6800221A617B6800225A617B6800223F
S3150800AEC09A627B6893F85D30DBB2002B06D17B680B
S3150800AED0002283F85C207868FAF7EEFD7B68022288
S3150800AEE083F85D207B681B681A687B681B6822F0FC
S3150800AEF040021A607B68DB68B3F5E06F02D900236D
S3150800AF00FB6002E04FF48053FB607B68DB68B3F5B7
S3150800AF10706F07D07B68DB68B3F5E06F02D07B689B
S3150800AF2000229A627B685B6803F482727B689B687E
S3150800AF3003F404431A437B681B6903F002031A43AC
S3150800AF407B685B6903F001031A437B689B6903F41A
S3150800AF5000731A437B68DB6903F038031A437B687E
S3150800AF601B6A03F0800342EA03017B689B6A03F4C9
S3150800AF7000527B681B680A431A607B689B691B0C36
S3150800AF8003F004027B685B6A03F010031A437B68CC
S3150800AF905B6B03F008031A437B68DB6803F4706392
S3150800AFA042EA0301FB6803F480527B681B680A4384
S3150800AFB05A607B6800221A667B68012283F85D2046
S3150800AFC0002318461037BD4680BD000080B586B000
S3150800AFD000AFF860B9607A607B800023FB75FB6878
S3150800AFE093F85C30012B01D102236CE1FB68012246
S3150800AFF083F85C20FB6893F85D30BB75FB685B687B
S3150800B0003B61BB7D012B0DD03B69B3F5827F06D131
S3150800B010FB689B68002B02D1BB7D042B02D0022360
S3150800B020FB754BE1BB68002B05D07B68002B02D073
S3150800B0307B88002B02D10123FB753FE1FB6893F85F
S3150800B0405D30DBB2042B03D0FB68052283F85D2054
S3150800B050FB6800221A66FB68BA689A63FB687A88F6
S3150800B0609A87FB687A88DA87FB687A681A64FB68C5
S3150800B0707A88A3F84420FB687A88A3F84620FB68F8
S3150800B0800022DA64FB6800221A65FB681B685A68A6
S3150800B090FB681B6822F4C0425A60FB68DB68B3F59C
S3150800B0A0E06F08D9FB681B685A68FB681B6822F4BE
S3150800B0B080525A606FE0FB681B685A68FB681B6819
S3150800B0C042F480525A60FB685B6D9B69B3F5806FEA
S3150800B0D026D1FB689B8F03F00103002B0FD1FB6879
S3150800B0E01B685A68FB681B6822F480425A60FB6832
S3150800B0F0DB8F9BB25B089AB2FB68DA8710E0FB68C5
S3150800B1001B685A68FB681B6842F480425A60FB68F1
S3150800B110DB8F9BB25B089BB201339AB2FB68DA8776
S3150800B120FB689B6D9B69B3F5806F34D1FB681B6820
S3150800B1305A68FB681B6822F480525A60FB68B3F8A9
S3150800B14046309BB203F00103002B11D1FB681B6844
S3150800B1505A68FB681B6822F400525A60FB68B3F809
S3150800B16046309BB25B089AB2FB68A3F8462012E009
S3150800B170FB681B685A68FB681B6842F400525A60F1
S3150800B180FB68B3F846309BB25B089BB201339AB2B0
S3150800B190FB68A3F84620FB6893F85D30DBB2042B06
S3150800B1A008D1FB689B6D4A4A1A63FB689B6D494A3E
S3150800B1B0DA6207E0FB689B6D474A1A63FB689B6D7A
S3150800B1C0464ADA62FB689B6D454A5A63FB689B6D83
S3150800B1D000229A63FB68986DFB681B680C33194656
S3150800B1E0FB681B6C1A46FB68B3F846309BB2FDF742
S3150800B1F0CBFD0346002B0CD0FB681B6E43F01002F8
S3150800B200FB681A660123FB75FB68012283F85D203B
S3150800B21054E0FB681B685A68FB681B6842F0010229
S3150800B2205A60FB685B6D00221A63FB685B6D00223F
S3150800B230DA62FB685B6D00225A63FB685B6D00226D
S3150800B2409A63FB68586DFB689B6B1946FB681B681D
S3150800B2500C331A46FB68DB8F9BB2FDF795FD034658
S3150800B260002B0CD0FB681B6E43F01002FB681A66B5
S3150800B2700123FB75FB68012283F85D201EE0FB684D
S3150800B2801B681B6803F04003402B07D0FB681B684C
S3150800B2901A68FB681B6842F040021A60FB681B6864
S3150800B2A05A68FB681B6842F020025A60FB681B68F4
S3150800B2B05A68FB681B6842F002025A60FB68002263
S3150800B2C083F85C20FB7D18461837BD4680BD00BF55
S3150800B2D045B600080DB5000861B60008B5B5000802
S3150800B2E07DB6000880B588B000AF78607B681B68BB
S3150800B2F05B68FB617B681B689B68BB61BB699B09D4
S3150800B30003F00103002B0FD1BB6903F00103002BE7
S3150800B3100AD0FB699B0903F00103002B04D07B6864
S3150800B320DB6C78689847D7E0BB695B0803F00103D4
S3150800B330002B0AD0FB69DB0903F00103002B04D0BC
S3150800B3407B681B6D78689847C6E0BB695B0903F0A4
S3150800B3500103002B0CD1BB699B0903F00103002BE9
S3150800B36006D1BB691B0A03F00103002B00F0B48069
S3150800B370FB695B0903F00103002B00F0AD80BB6994
S3150800B3809B0903F00103002B23D07B6893F85D30FB
S3150800B390DBB2032B11D07B681B6E43F004027B687B
S3150800B3A01A6600237B617B681B68DB687B617B68A8
S3150800B3B01B689B687B617B690BE000233B617B68AC
S3150800B3C01B68DB683B617B681B689B683B613B6964
S3150800B3D082E0BB695B0903F00103002B14D07B688C
S3150800B3E01B6E43F001027B681A660023FB607B68CC
S3150800B3F01B689B68FB607B681B681A687B681B6810
S3150800B40022F040021A60FB68BB691B0A03F00103BD
S3150800B410002B0CD07B681B6E43F008027B681A660B
S3150800B4200023BB607B681B689B68BB60BB687B6846
S3150800B4301B6E002B4FD07B681B685A687B681B689D
S3150800B44022F0E0025A607B68012283F85D20FB69DE
S3150800B45003F00203002B04D1FB6903F00103002B60
S3150800B46034D07B681B685A687B681B6822F0030225
S3150800B4705A607B689B6D002B11D07B689B6D184AC0
S3150800B4809A637B689B6D1846FDF7DEFC0346002B26
S3150800B49005D07B681B6E43F040027B681A667B68A2
S3150800B4A05B6D002B16D07B685B6D0D4A9A637B68D3
S3150800B4B05B6D1846FDF7C8FC0346002B0AD07B686F
S3150800B4C01B6E43F040027B681A6603E07868F9F75A
S3150800B4D0C1FB00E000BF00BF2037BD4680BD00BFEE
S3150800B4E0BDB6000880B483B000AF786000BF0C37E3
S3150800B4F0BD465DF8047B704780B483B000AF7860C2
S3150800B50000BF0C37BD465DF8047B704780B584B034
S3150800B51000AF78607B689B6AFB60FAF79DFCB860B1
S3150800B5207B681B681B6803F02003202B3CD0FB6854
S3150800B5301B685A68FB681B6822F020025A60FB6881
S3150800B5409B68002B0DD1FB685B68B3F5827F08D139
S3150800B550FB681B685A68FB681B6822F003025A607E
S3150800B56007E0FB681B685A68FB681B6822F0010243
S3150800B5705A60BA686421F86800F0D4F90346002BCB
S3150800B58002D0FB6820221A66FB680022A3F8462030
S3150800B590FB68012283F85D20FB681B6E002B03D035
S3150800B5A0F868F9F757FB02E0F868F9F733FB103744
S3150800B5B0BD4680BD80B584B000AF78607B689B6A65
S3150800B5C0FB60FAF749FCB8607B681B681B6803F0E8
S3150800B5D02003202B30D0FB681B685A68FB681B6861
S3150800B5E022F020025A60BA686421F86800F0F2F97D
S3150800B5F00346002B05D0FB681B6E43F02002FB6850
S3150800B6001A66FB681B685A68FB681B6822F0030207
S3150800B6105A60FB680022DA87FB680022A3F84620F6
S3150800B620FB68012283F85D20FB681B6E002B03D0A4
S3150800B630F868F9F70FFB02E0F868F9F7CBFA103764
S3150800B640BD4680BD80B584B000AF78607B689B6AD4
S3150800B650FB60F868FFF746FF00BF1037BD4680BDA0
S3150800B66080B584B000AF78607B689B6AFB60F86839
S3150800B670FFF742FF00BF1037BD4680BD80B584B0D6
S3150800B68000AF78607B689B6AFB60FB681B685A683A
S3150800B690FB681B6822F003025A60FB681B6E43F0C6
S3150800B6A01002FB681A66FB68012283F85D20F868B9
S3150800B6B0F9F7D0FA00BF1037BD4680BD80B584B013
S3150800B6C000AF78607B689B6AFB60FB680022A3F882
S3150800B6D04620FB680022DA87F868F9F7BBFA00BF4C
S3150800B6E01037BD4680BD000080B588B000AFF86051
S3150800B6F0B9603B601346FB71FAF7AEFB0246BB6ABC
S3150800B7009B1A3A681344FB61FAF7A6FBB861394BF2
S3150800B7101B685B011B0DFA6902FB03F37B6154E0AE
S3150800B7203B68B3F1FF3F50D0FAF796FB0246BB6978
S3150800B730D31AFA699A4202D9FB69002B3DD1FB68F4
S3150800B7401B685A68FB681B6822F0E0025A60FB68AF
S3150800B7505B68B3F5827F11D1FB689B68B3F5004F30
S3150800B76004D0FB689B68B3F5806F07D1FB681B683C
S3150800B7701A68FB681B6822F040021A60FB689B6A1D
S3150800B780B3F5005F0FD1FB681B681A68FB681B6876
S3150800B79022F400521A60FB681B681A68FB681B686B
S3150800B7A042F400521A60FB68012283F85D20FB68A8
S3150800B7B0002283F85C20032317E07B69002B01D164
S3150800B7C00023FB617B69013B7B61FB681B689A6808
S3150800B7D0BB681340BA689A420CBF01230023DBB248
S3150800B7E01A46FB799A429BD1002318462037BD4654
S3150800B7F080BD00BFA800002080B58AB000AFF86001
S3150800B800B9607A603B600023FB75FAF725FB0246B0
S3150800B8103B6B9B1A3A6813447B62FAF71DFB386246
S3150800B820FB681B680C33FB613D4B1A6813469B008B
S3150800B8301344DA00D31A1B0D7A6A02FB03F3BB61C1
S3150800B84060E0BB68B3F5C06F07D17B68002B04D1F5
S3150800B850FB691B78DBB2FB75FB7D3B68B3F1FF3FE9
S3150800B86050D0FAF7F9FA02463B6AD31A7A6A9A422C
S3150800B87002D97B6A002B3DD1FB681B685A68FB68B6
S3150800B8801B6822F0E0025A60FB685B68B3F5827FAA
S3150800B89011D1FB689B68B3F5004F04D0FB689B6821
S3150800B8A0B3F5806F07D1FB681B681A68FB681B68CD
S3150800B8B022F040021A60FB689B6AB3F5005F0FD15D
S3150800B8C0FB681B681A68FB681B6822F400521A603A
S3150800B8D0FB681B681A68FB681B6842F400521A600A
S3150800B8E0FB68012283F85D20FB68002283F85C2050
S3150800B8F0032310E0BB69002B01D100237B62BB69DF
S3150800B900013BBB61FB681B689A68BB6813407A6891
S3150800B9109A4296D1002318462837BD4680BD00BFF7
S3150800B920A800002080B586B002AFF860B9607A60DA
S3150800B930FB685B68B3F5827F11D1FB689B68B3F53A
S3150800B940004F04D0FB689B68B3F5806F07D1FB688E
S3150800B9501B681A68FB681B6822F040021A607B683D
S3150800B9600093BB6800228021F868FFF7BDFE0346F6
S3150800B970002B07D0FB681B6E43F02002FB681A6693
S3150800B980032323E0FB685B68B3F5827F1DD1FB6860
S3150800B9909B68B3F5004F04D0FB689B68B3F5806FCE
S3150800B9A013D17B680093BB6800224FF4C061F86826
S3150800B9B0FFF722FF0346002B07D0FB681B6E43F0F8
S3150800B9C02002FB681A66032300E000231846103796
S3150800B9D0BD4680BD80B586B002AFF860B9607A60B2
S3150800B9E07B680093BB6800224FF4C051F868FFF7E4
S3150800B9F003FF0346002B07D0FB681B6E43F02002AB
S3150800BA00FB681A66032327E07B680093BB6800225D
S3150800BA108021F868FFF768FE0346002B07D0FB680D
S3150800BA201B6E43F02002FB681A66032314E07B684A
S3150800BA300093BB6800224FF4C061F868FFF7DCFE8C
S3150800BA400346002B07D0FB681B6E43F02002FB68F9
S3150800BA501A66032300E0002318461037BD4680BD4A
S3150800BA6080B483B000AF78607B689B6843F00102BE
S3150800BA707B689A6000BF0C37BD465DF8047B70474B
S3150800BA8080B483B000AF786039607B689B6823F028
S3150800BA9018023B681A437B689A6000BF0C37BD469C
S3150800BAA05DF8047B704780B483B000AF7860396076
S3150800BAB07B683A685A6100BF0C37BD465DF8047B5F
S3150800BAC0704780B483B000AF786039607B683A68A5
S3150800BAD01A6000BF0C37BD465DF8047B704780B41A
S3150800BAE085B000AF78600B467B807B68FB60FB689F
S3150800BAF07A881A8000BF1437BD465DF8047B704704
S3150800BB0080B483B000AF78607B681B689BB2184628
S3150800BB100C37BD465DF8047B7047000080B485B0DD
S3150800BB2000AF7860084B9A6C07497B6813438B64AF
S3150800BB30054B9A6C7B681340FB60FB6800BF1437A3
S3150800BB40BD465DF8047B70470010024080B590B092
S3150800BB5000AF0346FB710523BB760023FB63002376
S3150800BB60BB6300237B6300233B630023FB62002344
S3150800BB70BB6200237B6200233B620023FB614FF01C
S3150800BB8000024FF00003C7E904230023FB760023D5
S3150800BB90FB8102F04FF90346002B02D00E2300F07A
S3150800BBA023BF02F0B7F8A34B01221A70A24B1B68F9
S3150800BBB09BB24FF6FF72934205D09F4B1B689A02C1
S3150800BBC09E4B134001E04FF480234FF4F032B2FB52
S3150800BBD0F3F101FB03F3D31ADB0AFB6342E0FB6BC9
S3150800BBE003F58033DA02944B1B689BB24FF6FF715C
S3150800BBF08B4205D0904B1B689902904B0B4001E095
S3150800BC004FF480234FF4F031B1FBF3F18A4B1B68F4
S3150800BC109BB24FF6FF70834205D0874B1B6898028C
S3150800BC20864B034001E04FF4802301FB03F31344E2
S3150800BC30BB6300237B630EE0BA6B7B6B1344804ABD
S3150800BC401360BA6B7B6B1344D3E90023C7E904235B
S3150800BC507B6B08337B637B6BB3F5006FECD3FB6BB5
S3150800BC600133FB63744B1B689BB24FF6FF7293421A
S3150800BC7005D0714B1B689A02704B134001E04FF4D4
S3150800BC8080234FF4F032B2FBF3F101FB03F3D31A2E
S3150800BC90DB0A0433FA6B9A42A1D3664B00221A7068
S3150800BCA0654B1B689BB24FF6FF72934205D0624BF9
S3150800BCB01B689A02614B134001E04FF480234FF44E
S3150800BCC0F032B2FBF3F101FB03F3D31ADB0AFB6391
S3150800BCD048E0FB6B03F58033DA02574B1B689BB2CF
S3150800BCE04FF6FF718B4205D0534B1B689902534B95
S3150800BCF00B4001E04FF480234FF4F031B1FBF3F130
S3150800BD004D4B1B689BB24FF6FF70834205D04A4BDA
S3150800BD101B689802494B034001E04FF4802301FB5E
S3150800BD2003F31344BB63B86B01F092FF0346BB767B
S3150800BD30BB7E022B02D0BB7E012B03D1FB6A0133EB
S3150800BD40FB620CE0BB7E032B09D1BB6A002B01D139
S3150800BD50FB6B3B62FB6B7B62BB6A0133BB62FB6BB3
S3150800BD600133FB63344B1B689BB24FF6FF72934259
S3150800BD7005D0314B1B689A02304B134001E04FF453
S3150800BD8080234FF4F032B2FBF3F101FB03F3D31A2D
S3150800BD90DB0A0433FA6B9A429BD3FB6A002B40F00A
S3150800BDA0B380BB6A002B00F0A980234B1B689BB2AB
S3150800BDB04FF6FF72934205D01F4B1B689A021F4B22
S3150800BDC0134001E04FF480234FF4F032B2FBF3F155
S3150800BDD001FB03F3D31ADB0A3A6AD31A033303F0D7
S3150800BDE00301154B1B689BB24FF6FF72934205D0B1
S3150800BDF0114B1B689A02114B134001E04FF4802344
S3150800BE004FF4F032B2FBF3F000FB03F3D31ADB0A6C
S3150800BE100B4403F58033DA02074B1B689BB24FF6D7
S3150800BE20FF718B420ED0044B1B689902034B0B40E3
S3150800BE300AE000BFE4040020E075FF1F00FCFF03D2
S3150800BE40E00400204FF480234FF4F031B1FBF3F106
S3150800BE50A94B1B689BB24FF6FF70834205D0A64BD1
S3150800BE601B689802A54B034001E04FF4802301FBB1
S3150800BE7003F31344184601F0EBFE0346042B43D1A3
S3150800BE809D4B1B689BB24FF6FF72934205D09A4BA7
S3150800BE901B689A02994B134001E04FF480234FF434
S3150800BEA0F032B2FBF3F101FB03F3D31ADB0A7A6A29
S3150800BEB0D31A013303F003018F4B1B689BB24FF66D
S3150800BEC0FF72934205D08C4B1B689A028B4B13402A
S3150800BED001E04FF480234FF4F032B2FBF3F000FB9D
S3150800BEE003F3D31ADB0A0B440121184601F09EFD21
S3150800BEF00346002B08D0022300F076BD002000F090
S3150800BF007BFD034600F070BD7B4B1B689BB24FF66A
S3150800BF10FF72934205D0784B1B689A02774B134001
S3150800BF2001E04FF480234FF4F032B2FBF3F101FB4A
S3150800BF3003F3D31ADB0AFB6355E1FB6B03F5803386
S3150800BF40DA026D4B1B689BB24FF6FF718B4205D028
S3150800BF50694B1B689902694B0B4001E04FF480233B
S3150800BF604FF4F031B1FBF3F1634B1B689BB24FF60C
S3150800BF70FF70834205D0604B1B6898025F4B0340F5
S3150800BF8001E04FF4802301FB03F31344BB63B86B52
S3150800BF9001F05EFE0346BB76BB7E012B40F0208196
S3150800BFA0554B1B689BB24FF6FF72934205D0524B16
S3150800BFB01B689A02514B134001E04FF480234FF45B
S3150800BFC0F032B2FBF3F101FB03F3D31ADB0AFA6B87
S3150800BFD09A4200F08380484B1B689BB24FF6FF726B
S3150800BFE0934205D0444B1B689A02444B134001E028
S3150800BFF04FF480234FF4F032B2FBF3F101FB03F365
S3150800C000D31ADB0A0233FA6B9A4267D03A4B1B689B
S3150800C0109BB24FF6FF72934205D0374B1B689A02C4
S3150800C020364B134001E04FF480234FF4F032B2FB55
S3150800C030F3F101FB03F3D31ADB0AFA6BD31A0333C2
S3150800C04003F003012C4B1B689BB24FF6FF72934219
S3150800C05005D0294B1B689A02284B134001E04FF480
S3150800C06080234FF4F032B2FBF3F000FB03F3D31A4C
S3150800C070DB0A0B4403F58033DA021F4B1B689BB2BD
S3150800C0804FF6FF718B4205D01B4B1B6899021B4B61
S3150800C0900B4001E04FF480234FF4F031B1FBF3F18C
S3150800C0A0154B1B689BB24FF6FF70834205D0124BA7
S3150800C0B01B689802114B034001E04FF4802301FBF3
S3150800C0C003F31344184601F0C3FD0346032B02D1BC
S3150800C0D00023FB766EE00123FB766BE0064B1B68BC
S3150800C0E09BB24FF6FF7293420AD0034B1B689A0223
S3150800C0F0024B134006E000BFE075FF1F00FCFF037C
S3150800C1004FF480234FF4F032B2FBF3F101FB03F353
S3150800C110D31ADB0AFA6BD31A013303F00301AD4BCA
S3150800C1201B689BB24FF6FF72934205D0A94B1B685A
S3150800C1309A02A94B134001E04FF480234FF4F032E2
S3150800C140B2FBF3F000FB03F3D31ADB0A0B4403F547
S3150800C1508033DA029F4B1B689BB24FF6FF718B4206
S3150800C16005D09C4B1B6899029B4B0B4001E04FF492
S3150800C17080234FF4F031B1FBF3F1964B1B689BB269
S3150800C1804FF6FF70834205D0924B1B689802924B7C
S3150800C190034001E04FF4802301FB03F313441846E0
S3150800C1A001F056FD0346002B02D10023FB7601E081
S3150800C1B00123FB76FB7E002B12D1FB6BDAB2874B91
S3150800C1C01A7001220021002001F0BAF80346B3F5DF
S3150800C1D0807F02D00C2300F007BC0123FB611EE020
S3150800C1E0FB6B0133FB637B4B1B689BB24FF6FF72FD
S3150800C1F0934205D0774B1B689A02774B134001E0B0
S3150800C2004FF480234FF4F032B2FBF3F101FB03F352
S3150800C210D31ADB0A0433FA6B9A42FFF48EAE002374
S3150800C2203B636C4B1B689BB24FF6FF72934205D07B
S3150800C230684B1B689A02684B134001E04FF4802351
S3150800C2404FF4F032B2FBF3F101FB03F3D31ADB0A26
S3150800C250FB6355E1FB6B03F58033DA025D4B1B6824
S3150800C2609BB24FF6FF718B4205D05A4B1B68990259
S3150800C270594B0B4001E04FF480234FF4F031B1FBEA
S3150800C280F3F1544B1B689BB24FF6FF70834205D0FF
S3150800C290504B1B689802504B034001E04FF4802333
S3150800C2A001FB03F31344BB63B86B01F0D1FC0346EF
S3150800C2B0BB76BB7E022B40F01B81464B1B689BB2AC
S3150800C2C04FF6FF72934205D0424B1B689A02424BC7
S3150800C2D0134001E04FF480234FF4F032B2FBF3F140
S3150800C2E001FB03F3D31ADB0AFA6B9A4200F0898042
S3150800C2F0384B1B689BB24FF6FF72934205D0354BFD
S3150800C3001B689A02344B134001E04FF480234FF424
S3150800C310F032B2FBF3F101FB03F3D31ADB0A023363
S3150800C320FA6B9A426DD02B4B1B689BB24FF6FF7285
S3150800C330934205D0274B1B689A02274B134001E00E
S3150800C3404FF480234FF4F032B2FBF3F101FB03F311
S3150800C350D31ADB0AFA6BD31A033303F003011D4B16
S3150800C3601B689BB24FF6FF72934205D0194B1B68A8
S3150800C3709A02194B134001E04FF480234FF4F03230
S3150800C380B2FBF3F000FB03F3D31ADB0A0B4403F505
S3150800C3908033DA020F4B1B689BB24FF6FF718B4254
S3150800C3A005D00C4B1B6899020B4B0B4001E04FF470
S3150800C3B080234FF4F031B1FBF3F1064B1B689BB2B7
S3150800C3C04FF6FF7083420BD0024B1B689802024B54
S3150800C3D0034007E0E075FF1F00FCFF03DE040020B2
S3150800C3E04FF4802301FB03F31344184601F030FC95
S3150800C3F00346032B02D10023FB7669E00123FB7673
S3150800C40066E0A74B1B689BB24FF6FF72934205D0B6
S3150800C410A34B1B689A02A34B134001E04FF48023F9
S3150800C4204FF4F032B2FBF3F101FB03F3D31ADB0A44
S3150800C430FA6BD31A013303F00301994B1B689BB2BD
S3150800C4404FF6FF72934205D0954B1B689A02954B9F
S3150800C450134001E04FF480234FF4F032B2FBF3F0BF
S3150800C46000FB03F3D31ADB0A0B4403F58033DA0225
S3150800C4708B4B1B689BB24FF6FF718B4205D0884BDE
S3150800C4801B689902874B0B4001E04FF480234FF459
S3150800C490F031B1FBF3F1824B1B689BB24FF6FF708C
S3150800C4A0834205D07E4B1B6898027E4B034001E011
S3150800C4B04FF4802301FB03F31344184601F0C8FB2D
S3150800C4C00346002B02D10023FB7601E00123FB760D
S3150800C4D0FB7E002B11D13B6B002B07D1FB6BDAB22D
S3150800C4E0714B1A703B6B01333B6306E00A237BE210
S3150800C4F0BB7E032B01D1FB6B7B62FB6B0133FB63BA
S3150800C500674B1B689BB24FF6FF72934205D0644B8C
S3150800C5101B689A02634B134001E04FF480234FF4E3
S3150800C520F032B2FBF3F101FB03F3D31ADB0A04334F
S3150800C530FA6B9A42FFF48EAE3B6B002B47D17B6AAF
S3150800C540D9B2574B1B689BB24FF6FF72934205D080
S3150800C550534B1B689A02534B134001E04FF4802358
S3150800C5604FF4F032B2FBF3F000FB03F3D31ADB0A05
S3150800C570DBB2CB1ADBB20133DBB203F00303D9B269
S3150800C580474B1B689BB24FF6FF72934205D0444B4C
S3150800C5901B689A02434B134001E04FF480234FF483
S3150800C5A0F032B2FBF3F000FB03F3D31ADB0ADBB27B
S3150800C5B00B44DAB23C4B1A703B4B1B7802211846E7
S3150800C5C001F034FA0346002B01D002230CE2374B64
S3150800C5D000221A80364B20221A6020237B6345E00E
S3150800C5E0314B1B7803F58033DA022D4B1B689BB25F
S3150800C5F04FF6FF718B4205D0294B1B689902294BD0
S3150800C6000B4001E04FF480234FF4F031B1FBF3F116
S3150800C610234B1B689BB24FF6FF70834205D0204B15
S3150800C6201B6898021F4B034001E04FF4802301FB6F
S3150800C63003F31A447B6B1344D3E90023C7E90423A5
S3150800C640D7E90423B3F1FF3F08BFB2F1FF3F12D089
S3150800C650164B1B8801339AB2144B1A80144B1B686D
S3150800C6600833134A13607B6B08337B637B6BB3F524
S3150800C670006FB5D300E000BF0B4B1B78FB630A4B7A
S3150800C6801B783B627AE0064B1B689BB24FF6FF723B
S3150800C69093420FD0024B1B689A02024B13400BE0E1
S3150800C6A0E075FF1F00FCFF03DE040020DC04002009
S3150800C6B0D40000204FF480234FF4F032B2FBF3F19C
S3150800C6C001FB03F3D31ADB0AFA6BD31A033303F01D
S3150800C6D00301A84B1B689BB24FF6FF72934205D025
S3150800C6E0A44B1B689A02A44B134001E04FF4802325
S3150800C6F04FF4F032B2FBF3F000FB03F3D31ADB0A74
S3150800C7000B44FB63FB6B03F58033DA02994B1B681A
S3150800C7109BB24FF6FF718B4205D0964B1B68990268
S3150800C720954B0B4001E04FF480234FF4F031B1FBF9
S3150800C730F3F1904B1B689BB24FF6FF70834205D00E
S3150800C7408C4B1B6898028C4B034001E04FF4802306
S3150800C75001FB03F31344184601F07AFA0346BB7645
S3150800C760BB7E032B08D1854B1B88FC339AB2834BBF
S3150800C7701A80FB6B3B6201E00A2335E17D4B1B689F
S3150800C7809BB24FF6FF72934205D07A4B1B689A020A
S3150800C790794B134001E04FF480234FF4F032B2FB9B
S3150800C7A0F3F101FB03F3D31ADB0AFA6B9A421BD0A7
S3150800C7B0704B1B689BB24FF6FF72934205D06D4BC8
S3150800C7C01B689A026C4B134001E04FF480234FF428
S3150800C7D0F032B2FBF3F101FB03F3D31ADB0A02339F
S3150800C7E0FA6B9A427FF44FAF654B1B781846614B3C
S3150800C7F01B689BB24FF6FF72934205D05D4B1B68D0
S3150800C8009A025D4B134001E04FF480234FF4F03257
S3150800C810B2FBF3F101FB03F3D31ADB0AC31A0133A4
S3150800C82003F00301534B1B689BB24FF6FF7293420A
S3150800C83005D0504B1B689A024F4B134001E04FF44A
S3150800C84080234FF4F032B2FBF3F000FB03F3D31A64
S3150800C850DB0A0B44FB63FB6B03F58033DA02454BBB
S3150800C8601B689BB24FF6FF718B4205D0414B1B6884
S3150800C8709902414B0B4001E04FF480234FF4F0310D
S3150800C880B1FBF3F13B4B1B689BB24FF6FF7083423B
S3150800C89005D0384B1B689802374B034001E04FF42C
S3150800C8A0802301FB03F31344BB6384E0FB79002B6D
S3150800C8B008D10121F86B01F075FA0346002B12D056
S3150800C8C0012391E04FF40061B86B00F0B0FB03461A
S3150800C8D0102B08D10121F86B01F064FA0346002BEE
S3150800C8E001D0012380E0234B1B689BB24FF6FF72F1
S3150800C8F0934205D01F4B1B689A021F4B134001E059
S3150800C9004FF480234FF4F032B2FBF3F101FB03F34B
S3150800C910D31ADB0AFA6BD31A013303F00301154B5A
S3150800C9201B689BB24FF6FF72934205D0114B1B68EA
S3150800C9309A02114B134001E04FF480234FF4F03272
S3150800C940B2FBF3F000FB03F3D31ADB0A0B44FB63D9
S3150800C950FB6B03F58033DA02064B1B689BB24FF676
S3150800C960FF718B420ED0034B1B689902024B0B409A
S3150800C9700AE000BFE075FF1F00FCFF03DC0400208F
S3150800C980DE0400204FF480234FF4F031B1FBF3F1BD
S3150800C990174B1B689BB24FF6FF70834205D0144BAA
S3150800C9A01B689802134B034001E04FF4802301FBF8
S3150800C9B003F31344BB63FA6B3B6A9A427FF476AF80
S3150800C9C001F016FAFB69002B0DD10021002000F0BA
S3150800C9D093FF0346FB81FB89002B04D0FB89122BAE
S3150800C9E001D0022300E0002318464037BD4680BD2B
S3150800C9F0E075FF1F00FCFF0380B584B000AF034657
S3150800CA00FB710023FB6001F015FA0346002B01D0E9
S3150800CA100E23BFE0614B1B689BB24FF6FF72934231
S3150800CA2005D05E4B1B689A025D4B134001E04FF43C
S3150800CA3080234FF4F032B2FBF3F101FB03F3D31A70
S3150800CA40DB0AFB6048E0FB79002B08D10121F86876
S3150800CA5001F0A8F90346002B3BD001239AE0FB68B6
S3150800CA6003F58033DA024D4B1B689BB24FF6FF7114
S3150800CA708B4205D0494B1B689902494B0B4001E094
S3150800CA804FF480234FF4F031B1FBF3F1434B1B68AD
S3150800CA909BB24FF6FF70834205D0404B1B68980245
S3150800CAA03F4B034001E04FF4802301FB03F313449B
S3150800CAB04FF40061184600F0BAFA0346102B08D165
S3150800CAC00121F86801F06EF90346002B01D0012315
S3150800CAD060E0FB680133FB60304B1B689BB24FF686
S3150800CAE0FF72934205D02D4B1B689A022C4B1340BC
S3150800CAF001E04FF480234FF4F032B2FBF3F101FB6F
S3150800CB0003F3D31ADB0A0433FA689A429BD301F07B
S3150800CB106FF9224B1B689BB24FF6FF72934205D002
S3150800CB201E4B1B689A021E4B134001E04FF48023EC
S3150800CB304FF4F032B2FBF3F101FB03F3D31ADB0A2D
S3150800CB400221184600F072FF0346002B01D002238B
S3150800CB5020E0144B00221A80104B1B689BB24FF63C
S3150800CB60FF72934205D00D4B1B689A020C4B13407B
S3150800CB7001E04FF480234FF4F032B2FBF3F101FBEE
S3150800CB8003F3D31ADB0ADAB2074B1A70074B2022D3
S3150800CB901A60002318461037BD4680BDE075FF1F92
S3150800CBA000FCFF03DC040020DE040020D400002083
S3150800CBB080B584B000AF03463960FB80FB88002B44
S3150800CBC016D0FB884FF6FF72934211D00023BB6044
S3150800CBD00023FB8107F10802FB881146184600F07E
S3150800CBE0F7F80346FB81BA683B681A60FB8900E0E0
S3150800CBF0082318461037BD4680BD80B582B000AF01
S3150800CC0003463960FB80FB88002B0BD0FB884FF668
S3150800CC10FF72934206D0FB883968184600F0E8F997
S3150800CC20034600E0082318460837BD4680BD0000C5
S3150800CC3080B586B000AF00237B6100233B610023EB
S3150800CC40FB600023BB600523FB710523BB715E4BAC
S3150800CC501B689BB24FF6FF72934205D05A4B1B686E
S3150800CC609A025A4B134001E04FF480234FF4F032F6
S3150800CC70B2FBF3F101FB03F3D31ADB0A7B6181E014
S3150800CC807B6903F58033DA024F4B1B689BB24FF67C
S3150800CC90FF718B4205D04C4B1B6899024B4B0B40DE
S3150800CCA001E04FF480234FF4F031B1FBF3F1464B2A
S3150800CCB01B689BB24FF6FF70834205D0424B1B6838
S3150800CCC09802424B034001E04FF4802301FB03F333
S3150800CCD01344FB60F86800F0BBFF0346FB71FB7961
S3150800CCE0042B4CD17B6901333B6136E03B6903F584
S3150800CCF08033DA02344B1B689BB24FF6FF718B42C6
S3150800CD0005D0314B1B689902304B0B4001E04FF4BC
S3150800CD1080234FF4F031B1FBF3F12B4B1B689BB228
S3150800CD204FF6FF70834205D0274B1B689802274BA6
S3150800CD30034001E04FF4802301FB03F31344BB6077
S3150800CD40B86800F085FF0346BB71BB79042B01D098
S3150800CD50052334E03B6901333B617B6902333A6959
S3150800CD609A42C3D30221786901F01CF80346002BC6
S3150800CD7001D0012323E001F03BF800231FE07B6983
S3150800CD8002337B61104B1B689BB24FF6FF729342CE
S3150800CD9005D00D4B1B689A020C4B134001E04FF46B
S3150800CDA080234FF4F032B2FBF3F101FB03F3D31AFD
S3150800CDB0DB0A04337A699A42FFF462AF0523184600
S3150800CDC01837BD4680BD00BFE075FF1F00FCFF0396
S3150800CDD080B58AB000AF03463960FB804FF0000289
S3150800CDE04FF00003C7E9042300237B6200233B625C
S3150800CDF00023FB610023FB600523FB76002000F07F
S3150800CE003BF978627B6AB3F1FF3F01D10323E7E080
S3150800CE107B6A03F58033DA02734B1B689BB24FF6C5
S3150800CE20FF718B4205D0704B1B6899026F4B0B4004
S3150800CE3001E04FF480234FF4F031B1FBF3F16A4B74
S3150800CE401B689BB24FF6FF70834205D0664B1B6882
S3150800CE509802664B034001E04FF4802301FB03F37D
S3150800CE6013443B62386A00F0F3FE0346FB76AAE0F9
S3150800CE704FF4FF63FB613FE03A6AFB691344D3E969
S3150800CE800023C7E90423D7E90423B3F1FF3F08BF0A
S3150800CE90B2F1FF3F2DD03B8AFA889A4229D1D7E9C9
S3150800CEA004014FF000024FF000030A0000233B8AFA
S3150800CEB01946104600F042FF0346FB60D7E9040115
S3150800CEC04FF000024FF00003020C42EA01420B0C3D
S3150800CED093B21A46FB6893420BD1D7E904014FF087
S3150800CEE000024FF000030A0000233B681A60002383
S3150800CEF076E0FB69083BFB61FB691F2BBCD83A4B04
S3150800CF001B689BB24FF6FF72934205D0364B1B68DF
S3150800CF109A02364B134001E04FF480234FF4F03267
S3150800CF20B2FBF3F101FB03F3D31ADB0A7A6AD31ACD
S3150800CF30033303F003012C4B1B689BB24FF6FF72B9
S3150800CF40934205D0284B1B689A02284B134001E0F0
S3150800CF504FF480234FF4F032B2FBF3F000FB03F3F7
S3150800CF60D31ADB0A0B447B627B6A03F58033DA0249
S3150800CF701D4B1B689BB24FF6FF718B4205D01A4BAF
S3150800CF801B689902194B0B4001E04FF480234FF4BC
S3150800CF90F031B1FBF3F1144B1B689BB24FF6FF70EF
S3150800CFA0834205D0104B1B689802104B034001E0E2
S3150800CFB04FF4802301FB03F313443B62386A00F005
S3150800CFC047FE0346FB76FB7E022B3FF451AFFB7E02
S3150800CFD0032B3FF44DAFFB7E042B3FF449AF0723E9
S3150800CFE018462837BD4680BDE075FF1F00FCFF03C5
S3150800CFF080B584B000AF03463960FB800023FB810F
S3150800D000FB883968184600F077FC0346FB81FB89E4
S3150800D010122B07D1FB8800223968184600F090F9D0
S3150800D020034600E0FB8918461037BD4680BD80B42C
S3150800D03085B000AF786039601123FB810023BB609F
S3150800D0400FE07A68BB681344D3E90023B3F1FF3FC6
S3150800D05008BFB2F1FF3F01D01023FB81BB6808333C
S3150800D060BB60BA683B689A42EBD3FB89184614370B
S3150800D070BD465DF8047B704780B586B000AF0346B1
S3150800D080FB710523FB750523BB7500233B61002354
S3150800D090FB600023BB60A64B1B783B613B6903F52D
S3150800D0A08033DA02A34B1B689BB24FF6FF718B42A3
S3150800D0B005D0A04B1B6899029F4B0B4001E04FF42B
S3150800D0C080234FF4F031B1FBF3F19A4B1B689BB206
S3150800D0D04FF6FF70834205D0964B1B689802964B15
S3150800D0E0034001E04FF4802301FB03F31344184681
S3150800D0F000F0AEFD0346FB758E4B1B689BB24FF6E0
S3150800D100FF72934205D08B4B1B689A028A4B1340D9
S3150800D11001E04FF480234FF4F032B2FBF3F101FB48
S3150800D12003F3D31ADB0A3A69D31A013303F003016E
S3150800D130804B1B689BB24FF6FF72934205D07D4B1E
S3150800D1401B689A027C4B134001E04FF480234FF48E
S3150800D150F032B2FBF3F000FB03F3D31ADB0A0B44FD
S3150800D160FB60FB6803F58033DA02724B1B689BB2DF
S3150800D1704FF6FF718B4205D06E4B1B6899026E4BBA
S3150800D1800B4001E04FF480234FF4F031B1FBF3F18B
S3150800D190684B1B689BB24FF6FF70834205D0654B00
S3150800D1A01B689802644B034001E04FF4802301FB9F
S3150800D1B003F31344184600F04BFD0346BB755D4B5D
S3150800D1C01B689BB24FF6FF72934205D0594B1B68FA
S3150800D1D09A02594B134001E04FF480234FF4F03282
S3150800D1E0B2FBF3F101FB03F3D31ADB0A3A69D31A4C
S3150800D1F0033303F003014F4B1B689BB24FF6FF72D4
S3150800D200934205D04B4B1B689A024B4B134001E0E7
S3150800D2104FF480234FF4F032B2FBF3F000FB03F334
S3150800D220D31ADB0A0B44BB60FB79022B71D0022BA5
S3150800D23077DC002B60D0012B73D1FB7D022B2AD122
S3150800D2403E4B1B68B3F5006F01D23B696BE0BB7DB3
S3150800D250042B07D1FFF7ECFC0346002B02D04FF056
S3150800D260FF3360E00321386900F0E0FB0346002B3A
S3150800D27002D04FF0FF3356E00221F86800F0D6FBE3
S3150800D2800346002B02D04FF0FF334CE02B4B2022F5
S3150800D2901A60FB6847E0FB7D012B2AD1274B1B68E8
S3150800D2A0B3F5006F01D23B693DE0BB7D042B07D186
S3150800D2B0FFF7BEFC0346002B02D04FF0FF3332E0E7
S3150800D2C00321386900F0B2FB0346002B02D04FF069
S3150800D2D0FF3328E00121F86800F0A8FB0346002B7D
S3150800D2E002D04FF0FF331EE0144B20221A60FB6871
S3150800D2F019E04FF0FF3316E0FB7D022B01D13B69A5
S3150800D30011E0FB7D012B01D1BB680CE04FF0FF3328
S3150800D31009E0BB7D002B01D1FB6804E04FF0FF3329
S3150800D32001E04FF0FF3318461837BD4680BD00BFF1
S3150800D330DE040020E075FF1F00FCFF03D400002078
S3150800D34080B58AB000AF03463960FB8013467B710F
S3150800D350052387F827300023BB6100233B6200239F
S3150800D360FB614FF000024FF00003C7E904230023D6
S3150800D370FB810023BB607B79002B01D1022300E0EF
S3150800D38001231846FFF778FE38623B6AB3F1FF3F80
S3150800D39001D10423A1E2AE4B00221A803B6ADAB21D
S3150800D3A0AC4B1A70AC4B20221A607B79002B08D143
S3150800D3B00121386A00F03AFB0346002B01D002230C
S3150800D3C08BE2A64B1B689BB24FF6FF72934205D0C1
S3150800D3D0A24B1B689A02A24B134001E04FF480232C
S3150800D3E04FF4F032B2FBF3F101FB03F3D31ADB0A75
S3150800D3F03A6AD31A033303F00301984B1B689BB2AE
S3150800D4004FF6FF72934205D0944B1B689A02944BD1
S3150800D410134001E04FF480234FF4F032B2FBF3F0EF
S3150800D42000FB03F3D31ADB0A0B443B623B6A03F5A2
S3150800D4308033DA02894B1B689BB24FF6FF718B4229
S3150800D44005D0864B1B689902854B0B4001E04FF4CB
S3150800D45080234FF4F031B1FBF3F1804B1B689BB28C
S3150800D4604FF6FF70834205D07C4B1B6898027C4BB5
S3150800D470034001E04FF4802301FB03F31344BB612F
S3150800D480B86900F0E5FB034687F8273097F8273098
S3150800D490022B04D097F82730042B40F0FA8097F82F
S3150800D4A02730022B08D10421386A00F0BFFA034658
S3150800D4B0002B01D0022310E2684B1B689BB24FF683
S3150800D4C0FF72934205D0654B1B689A02644B134062
S3150800D4D001E04FF480234FF4F032B2FBF3F101FB85
S3150800D4E003F3D31ADB0A3A6AD31A033303F00301A8
S3150800D4F05A4B1B689BB24FF6FF72934205D0574BA7
S3150800D5001B689A02564B134001E04FF480234FF4F0
S3150800D510F032B2FBF3F000FB03F3D31ADB0A0B4439
S3150800D5203B623B6A03F58033DA024C4B1B689BB2BD
S3150800D5304FF6FF718B4205D0484B1B689902484B42
S3150800D5400B4001E04FF480234FF4F031B1FBF3F1C7
S3150800D550424B1B689BB24FF6FF70834205D03F4B88
S3150800D5601B6898023E4B034001E04FF4802301FB01
S3150800D57003F31344BB61B86900F06AFB034687F8F6
S3150800D58027307BE097F82730032B08D10421386A27
S3150800D59000F04CFA0346002B01D002239DE12F4BE5
S3150800D5A01B689BB24FF6FF72934205D02B4B1B6844
S3150800D5B09A022B4B134001E04FF480234FF4F032CC
S3150800D5C0B2FBF3F101FB03F3D31ADB0A3A6AD31A67
S3150800D5D0033303F00301214B1B689BB24FF6FF721E
S3150800D5E0934205D01D4B1B689A021D4B134001E060
S3150800D5F04FF480234FF4F032B2FBF3F000FB03F351
S3150800D600D31ADB0A0B443B623B6A03F58033DA0222
S3150800D610124B1B689BB24FF6FF718B4205D00F4B1E
S3150800D6201B6899020E4B0B4001E04FF480234FF420
S3150800D630F031B1FBF3F1094B1B689BB24FF6FF7053
S3150800D64083420FD0054B1B689802054B03400BE03D
S3150800D650DC040020DE040020D4000020E075FF1F53
S3150800D66000FCFF034FF4802301FB03F31344BB6163
S3150800D670B86900F0EDFA034687F8273097F827309F
S3150800D680032B3FF47FAF97F82730042B3FF47AAF8C
S3150800D69008E07B79012B03D197F82730032B01D0BB
S3150800D6A00A231AE17B79012B40F0CB802023FB610A
S3150800D6B045E08C4B1B7803F58033DA028A4B1B68EE
S3150800D6C09BB24FF6FF718B4205D0874B1B689902B8
S3150800D6D0864B0B4001E04FF480234FF4F031B1FB49
S3150800D6E0F3F1814B1B689BB24FF6FF70834205D05E
S3150800D6F07D4B1B6898027D4B034001E04FF4802365
S3150800D70001FB03F31A44FB691344D3E90023C7E971
S3150800D7100423D7E90423B3F1FF3F08BFB2F1FF3F63
S3150800D72012D0734B1B8801339AB2714B1A80714B16
S3150800D7301B6808336F4A1360FB690833FB61FB6992
S3150800D740B3F5006FB5D300E000BF664B1B783B62AC
S3150800D7500023FB6170E0644B1B689BB24FF6FF72B7
S3150800D760934205D0604B1B689A02604B134001E058
S3150800D7704FF480234FF4F032B2FBF3F101FB03F3CD
S3150800D780D31ADB0A3A6AD31A033303F00301564B5A
S3150800D7901B689BB24FF6FF72934205D0524B1B682B
S3150800D7A09A02524B134001E04FF480234FF4F032B3
S3150800D7B0B2FBF3F000FB03F3D31ADB0A0B443B621C
S3150800D7C03B6A03F58033DA02474B1B689BB24FF678
S3150800D7D0FF718B4205D0444B1B689902434B0B40A3
S3150800D7E001E04FF480234FF4F031B1FBF3F13E4BE7
S3150800D7F01B689BB24FF6FF70834205D03A4B1B68F5
S3150800D80098023A4B034001E04FF4802301FB03F3EF
S3150800D8101344184600F01CFA034687F8273097F891
S3150800D8202730032B0CD1324B1B88FC339AB2304B72
S3150800D8301A80FB690133FB61FB69032B8BD900E076
S3150800D84000BFFB883968184600F056F80346002BD7
S3150800D85001D0022341E0264B1B88022B03D9244B17
S3150800D8601B88023B00E00123FB6126E0FB88FA697E
S3150800D8709A421FD0FB699BB207F108021146184667
S3150800D880FFF7A6FA0346FB81FB89002B0DD1FB693E
S3150800D8909BB2BA681146184600F02EF80346FB817B
S3150800D8A0FB89002B06D0FB8917E0FB89072B01D0E3
S3150800D8B0FB8912E0FB690133FB61FB69062BD5D9AD
S3150800D8C0084B1B780221184600F0B0F80346002BD7
S3150800D8D001D0022301E04FF4807318462837BD466D
S3150800D8E080BD00BFDE040020E075FF1F00FCFF03BB
S3150800D8F0DC040020D40000202DE9F04F8BB000AFE7
S3150800D90003463961FB8200237B62444B1B88B3F5CF
S3150800D910FC7F01D312237CE00120FFF7ADFB3862C0
S3150800D9200023FB613B6AB3F1FF3F01D1032370E09B
S3150800D9303B6A03F58033D902394B1B689BB24FF615
S3150800D940FF72934205D0364B1B689A02354B13403B
S3150800D95001E04FF480234FF4F032B2FBF3F0304B82
S3150800D9601B689BB24FF6FF72934205D02C4B1B687F
S3150800D9709A022C4B134001E04FF4802300FB03F37B
S3150800D9800B44FB613B69002B05D1FB8A002B02D1B6
S3150800D99000237B6206E0FB8A1946386900F0CEF957
S3150800D9A003467B62204B1A68FB69D0183B69002244
S3150800D9B0BB60FA604FF000024FF00003B9680B0035
S3150800D9C00022796A090400268A46B34642EA0A040E
S3150800D9D043EA0B05FB8A00229846914644EA080367
S3150800D9E03B6045EA09037B60D7E9002300F0C2F9EA
S3150800D9F00346002B01D002230BE00B4B1B680833B0
S3150800DA00094A1360054B1B8801339AB2034B1A80E7
S3150800DA10002318462C37BD46BDE8F08FDC040020ED
S3150800DA20E075FF1F00FCFF03D400002080B586B018
S3150800DA3000AF78600B46FB7000237B6100233B61D7
S3150800DA400023FB600023BB607B6803F58033DA02A2
S3150800DA507C4B1B689BB24FF6FF718B4205D0794B06
S3150800DA601B689902784B0B4001E04FF480234FF472
S3150800DA70F031B1FBF3F1734B1B689BB24FF6FF70A5
S3150800DA80834205D06F4B1B6898026F4B034001E039
S3150800DA904FF4802301FB03F313447B617B6803F592
S3150800DAA08033DA02674B1B689BB24FF6FF718B42D5
S3150800DAB005D0644B1B689902634B0B4001E04FF499
S3150800DAC080234FF4F031B1FBF3F15E4B1B689BB238
S3150800DAD04FF6FF70834205D05A4B1B6898025A4B83
S3150800DAE0034001E04FF4802301FB03F3134408339A
S3150800DAF03B617B6803F58033DA02524B1B689BB2A5
S3150800DB004FF6FF718B4205D04E4B1B6899024E4B60
S3150800DB100B4001E04FF480234FF4F031B1FBF3F1F1
S3150800DB20484B1B689BB24FF6FF70834205D0454BA6
S3150800DB301B689802444B034001E04FF4802301FB25
S3150800DB4003F313441033FB607B6803F58033DA0272
S3150800DB503C4B1B689BB24FF6FF718B4205D0394B85
S3150800DB601B689902384B0B4001E04FF480234FF4B1
S3150800DB70F031B1FBF3F1334B1B689BB24FF6FF70E4
S3150800DB80834205D02F4B1B6898022F4B034001E0B8
S3150800DB904FF4802301FB03F313441833BB60FB786F
S3150800DBA0013B032B44D801A252F823F0BDDB000841
S3150800DBB0DFDB000801DC000819DC00084FF0AA3298
S3150800DBC04FF0AA33786900F0D5F80346002B01D048
S3150800DBD0022333E07B68DAB21C4B1A702DE04FF053
S3150800DBE0AA324FF0AA33386900F0C4F80346002B6E
S3150800DBF001D0022322E07B68DAB2144B1A701CE0CB
S3150800DC004FF0AA324FF0AA33F86800F0B3F803468B
S3150800DC10002B0FD0022311E04FF0AA324FF0AA339F
S3150800DC20B86800F0A7F80346002B05D0022305E0E4
S3150800DC3000BF02E000BF00E000BF00231846183707
S3150800DC40BD4680BDE075FF1F00FCFF03DE04002013
S3150800DC5080B48BB000AF78604FF000024FF000033D
S3150800DC60C7E908234FF000024FF00003C7E906236F
S3150800DC704FF000024FF00003C7E904234FF00002FB
S3150800DC804FF00003C7E902237B68D3E90023C7E9FD
S3150800DC9008237B680833D3E90023C7E906237B6892
S3150800DCA01033D3E90023C7E904237B681833D3E983
S3150800DCB00023C7E90223D7E90223B3F1FF3F08BFD0
S3150800DCC0B2F1FF3F01D004231EE0D7E90423B3F1E4
S3150800DCD0FF3F08BFB2F1FF3F01D0032314E0D7E9A5
S3150800DCE00623B3F1FF3F08BFB2F1FF3F01D002237D
S3150800DCF00AE0D7E90823B3F1FF3F08BFB2F1FF3FB7
S3150800DD0001D0012300E0002318462C37BD465DF8F4
S3150800DD10047B704780B500AF4FF48050FDF7FEFED8
S3150800DD2048F205010448FDF7BEFE08210248FDF742
S3150800DD30A7FE00BF80BD00BF0030024080B582B09C
S3150800DD4000AF78600B467B800948FDF789FE796845
S3150800DD500748FDF7B6FE7B8819460548FDF7BFFE5E
S3150800DD600348FDF7CDFE034618460837BD4680BD75
S3150800DD700030024080B584B000AFF860C7E90023E0
S3150800DD80074B4CF2FB321A61D7E90023F9680020E9
S3150800DD90FBF77AF9034618461037BD4680BD00BF23
S3150800DDA00020024080B58AB000AF78600B467B80C1
S3150800DDB00023FB8401233B620023FB6000233B61B5
S3150800DDC07B88FB617B68BB613B6A7B6107F10C0260
S3150800DDD007F1100311461846FBF7A8FA0346002B6D
S3150800DDE001D00123FB84FB8C18462837BD4680BD2D
S3150800DDF080B400AF0E4B1B680D4A23F48063136092
S3150800DE000B4B1B680A4A43F480531360084B1B6884
S3150800DE10074A23F480531360054B1B68044A43F4EE
S3150800DE208063136000BFBD465DF8047B704700BF82
S3150800DE300020024080B400AF00231846BD465DF8B6
S3150800DE40047B704780B483B000AF03463960FB712A
S3150800DE5097F90730002B0ADB3B68DAB20C4997F9C9
S3150800DE6007301201D2B20B4483F800230AE03B685C
S3150800DE70DAB20849FB7903F00F03043B1201D2B268
S3150800DE800B441A7600BF0C37BD465DF8047B704715
S3150800DE9000E100E000ED00E080B500AF00216FF082
S3150800DEA00400FFF7CFFF00BF80BD000080B483B039
S3150800DEB000AFEFF305833B603B68002B03D06FF0A0
S3150800DEC005037B600CE00A4B1B68002B05D1084B49
S3150800DED001221A6000237B6002E04FF0FF337B606B
S3150800DEE07B6818460C37BD465DF8047B704700BF53
S3150800DEF0E804002080B582B000AFEFF305833B60ED
S3150800DF003B68002B03D06FF005037B6010E00B4BDA
S3150800DF101B68012B09D1FFF7BFFF084B02221A60C5
S3150800DF2002F054FA00237B6002E04FF0FF337B6077
S3150800DF307B6818460837BD4680BD00BFE804002048
S3150800DF4080B582B000AFEFF305833B603B68002BDA
S3150800DF5003D06FF005037B6013E002F041FF034630
S3150800DF60002B02D0022B03D007E001237B6008E0D8
S3150800DF7002F09CFA00237B6003E04FF0FF337B60DE
S3150800DF8000BF7B6818460837BD4680BD80B58EB091
S3150800DF9004AFF860B9607A6000233B61EFF305834C
S3150800DFA07B617B69002B7ED1FB68002B7BD08023AD
S3150800DFB03B621823FB6100237B624FF0FF33BB6192
S3150800DFC07B68002B45D07B681B68002B02D07B68DA
S3150800DFD01B687B627B689B69002B02D07B689B6908
S3150800DFE0FB61FB69002B08D0FB69382B05D87B68D9
S3150800DFF05B6803F00103002B01D0002354E07B6823
S3150800E0005B69002B03D07B685B699B083B627B6876
S3150800E0109B68002B0ED07B68DB68BB2B0AD97B6814
S3150800E0201B69002B06D07B685B69002B02D0012395
S3150800E030BB6110E07B689B68002B0CD17B68DB68B2
S3150800E040002B08D17B681B69002B04D10023BB6118
S3150800E05001E00023BB61BB69012B10D17B681B69FA
S3150800E0607A68926802920193FB690093BB683A6AE0
S3150800E070796AF86801F048FF03463B6113E0BB691B
S3150800E080002B10D13B6A9AB207F110030193FB6982
S3150800E0900093BB68796AF86801F093FF0346012B81
S3150800E0A001D000233B613B6918462837BD4680BD31
S3150800E0B080B586B000AF78607B683B61EFF3058377
S3150800E0C0FB60FB68002B03D06FF005037B610BE058
S3150800E0D03B69002B03D16FF003037B6104E0002347
S3150800E0E07B61386902F0FCF87B6918461837BD462B
S3150800E0F080BD80B584B000AF7860EFF30583BB6060
S3150800E100BB68002B03D06FF00503FB6007E0002314
S3150800E110FB607B68002B02D0786802F0ADF8FB68DC
S3150800E12018461037BD4680BD80B584B000AF78600C
S3150800E130786803F033FCF860FB68002B05D0FB68B1
S3150800E1401B68FA6852681046984700BF1037BD46E4
S3150800E15080BD000080B58CB002AFF8607A603B6085
S3150800E1600B46FB7200233B62EFF305833B613B6979
S3150800E170002B63D1FB68002B60D0082003F09CFEBF
S3150800E18078617B69002B59D07B69FA681A607B69CC
S3150800E1907A685A60FB7A002B02D10023FB6101E002
S3150800E1A00123FB614FF0FF33BB6100237B623B68B1
S3150800E1B0002B1CD03B681B68002B02D03B681B68F1
S3150800E1C07B623B689B68002B06D03B68DB682B2B81
S3150800E1D002D90123BB610CE03B689B68002B08D180
S3150800E1E03B68DB68002B04D10023BB6101E00023F8
S3150800E1F0BB61BB69012B0CD13B689B680193124B31
S3150800E20000937B69FA690121786A03F048F8386255
S3150800E2100BE0BB69002B08D10B4B00937B69FA69AD
S3150800E2200121786A03F01AF838623B6A002B05D197
S3150800E2307B69002B02D0786903F00AFF3B6A18460F
S3150800E2402837BD4680BD00BF29E1000880B588B0E3
S3150800E25002AF786039607B683B61EFF30583FB604A
S3150800E260FB68002B03D06FF005037B6117E03B6961
S3150800E270002B03D16FF003037B6110E000230093AA
S3150800E28000233A680421386903F082F80346012B13
S3150800E29002D100237B6102E06FF002037B617B6998
S3150800E2A018461837BD4680BD80B586B000AF786081
S3150800E2B000237B61EFF30583FB60FB68002B2DD100
S3150800E2C04FF0FF333B617B68002B15D07B689B685A
S3150800E2D0002B06D07B68DB681F2B02D901233B6124
S3150800E2E00CE07B689B68002B08D17B68DB68002BF9
S3150800E2F004D100233B6101E000233B613B69012B0C
S3150800E30006D17B689B68184600F05EFB786105E0DD
S3150800E3103B69002B02D100F08EFB78617B691846B9
S3150800E3201837BD4680BD000080B586B000AF78605E
S3150800E33039607B683B613B69002B04D03B6803F07E
S3150800E3407F43002B03D06FF003037B6128E0EFF3D4
S3150800E3500583FB60FB68002B1DD00023BB6007F11B
S3150800E36008031A463968386900F086FD0346002B0B
S3150800E37003D16FF002037B6112E03B687B61BB68E7
S3150800E380002B0DD0094B4FF080521A60BFF34F8F08
S3150800E390BFF36F8F04E03968386900F0A5FC78612F
S3150800E3A07B6918461837BD4680BD00BF04ED00E0FE
S3150800E3B080B586B000AF786039607B683B613B69A1
S3150800E3C0002B04D03B6803F07F43002B03D06FF08B
S3150800E3D003037B6119E0EFF30583FB60FB68002B01
S3150800E3E00ED0386900F05CFC78613968386900F04D
S3150800E3F043FC0346002B08D16FF002037B6104E05F
S3150800E4003968386900F000FC78617B691846183766
S3150800E410BD4680BD80B58CB002AFF860B9607A6041
S3150800E4203B60FB68BB61BB69002B04D0BB6803F08B
S3150800E4307F43002B03D06FF00303FB614BE0EFF340
S3150800E44005837B617B69002B03D06FF00503FB61B5
S3150800E45041E07B6803F00103002B02D001237B62B5
S3150800E46001E000237B627B6803F00203002B02D0E5
S3150800E47000233B6201E001233B623B6800937B6A11
S3150800E4803A6AB968B86900F0F1FAF8617B6803F08E
S3150800E4900103002B10D0BA68FB691340BA689A4288
S3150800E4A019D03B68002B03D06FF00103FB6112E023
S3150800E4B06FF00203FB610EE0BA68FB691340002B9C
S3150800E4C009D13B68002B03D06FF00103FB6102E022
S3150800E4D06FF00203FB61FB6918462837BD4680BD0D
S3150800E4E080B588B000AF78600023FB61EFF3058341
S3150800E4F0BB60BB68002B74D17B68002B03D07B689C
S3150800E5005B68BB6101E00023BB61BB6903F00103E3
S3150800E510002B02D001237B6101E000237B61BB69EC
S3150800E52003F00803002B5CD14FF0FF333B617B6897
S3150800E530002B15D07B689B68002B06D07B68DB68B0
S3150800E5404F2B02D901233B610CE07B689B68002BAB
S3150800E55008D17B68DB68002B04D100233B6101E00E
S3150800E56000233B613B69012B12D17B69002B07D045
S3150800E5707B689B681946042000F0B5FEF86116E032
S3150800E5807B689B681946012000F0ADFEF8610EE035
S3150800E5903B69002B0BD17B69002B04D0042000F0CB
S3150800E5A08AFEF86103E0012000F085FEF861FB6948
S3150800E5B0002B0CD07B68002B03D07B681B68FB60A4
S3150800E5C001E00023FB60F968F86901F03FFCFB698C
S3150800E5D0002B06D07B69002B03D0FB6943F00103AF
S3150800E5E0FB61FB6918462037BD4680BD80B586B0FD
S3150800E5F000AF786039607B6823F001033B617B6874
S3150800E60003F00103FB6000237B61EFF30583BB6026
S3150800E610BB68002B03D06FF005037B612CE03B69D8
S3150800E620002B03D16FF003037B6125E0FB68002B09
S3150800E63011D03968386900F0A5FE0346012B1BD0B6
S3150800E6403B68002B03D06FF001037B6114E06FF089
S3150800E65002037B6110E03968386901F043F9034623
S3150800E660012B09D03B68002B03D06FF001037B61B7
S3150800E67002E06FF002037B617B6918461837BD46D6
S3150800E68080BD80B586B000AF78607B6823F0010353
S3150800E6903B617B6803F00103FB6000237B61EFF3BA
S3150800E6A00583BB60BB68002B03D06FF005037B6155
S3150800E6B01FE03B69002B03D16FF003037B6118E071
S3150800E6C0FB68002B09D0386900F028FE0346012BA9
S3150800E6D00FD06FF002037B610BE0002300220021BC
S3150800E6E0386900F085FE0346012B02D06FF002035D
S3150800E6F07B617B6918461837BD4680BD80B58AB0F0
S3150800E70002AFF860B9607A600023FB61EFF3058316
S3150800E7103B613B69002B5FD1FB68002B5CD0BB6873
S3150800E720002B59D04FF0FF33BB617B68002B29D0F3
S3150800E7307B689B68002B12D07B68DB684F2B0ED951
S3150800E7407B681B69002B0AD07B685A69FB68B96825
S3150800E75001FB03F39A4202D30123BB6114E07B68F1
S3150800E7609B68002B10D17B68DB68002B0CD17B687B
S3150800E7701B69002B08D17B685B69002B04D1002339
S3150800E780BB6101E00023BB61BB69012B0BD17B6830
S3150800E7901A697B689B6800210091B968F86800F0DF
S3150800E7A09BFCF86108E0BB69002B05D10022B9681B
S3150800E7B0F86800F009FDF861FB69002B0CD07B684E
S3150800E7C0002B03D07B681B687B6101E000237B611B
S3150800E7D07969F86901F03AFBFB6918462037BD46A6
S3150800E7E080BD000080B588B000AFF860B9603B60B6
S3150800E7F01346FB71FB68BB610023FB61EFF30583DE
S3150800E8007B617B69002B28D0BB69002B05D0BB68D0
S3150800E810002B02D03B68002B03D06FF00303FB618B
S3150800E82038E000233B6107F110020023B968B86994
S3150800E83000F0DCFE0346012B03D06FF00203FB61F8
S3150800E84028E03B69002B25D0154B4FF080521A6003
S3150800E850BFF34F8FBFF36F8F1CE0BB69002B02D04D
S3150800E860BB68002B03D16FF00303FB6112E00023A2
S3150800E8703A68B968B86900F0BBFD0346012B09D0B0
S3150800E8803B68002B03D06FF00103FB6102E06FF0D9
S3150800E8900203FB61FB6918462037BD4680BD00BFF1
S3150800E8A004ED00E080B588B000AFF860B9607A6022
S3150800E8B03B60FB68BB610023FB61EFF305837B616B
S3150800E8C07B69002B28D0BB69002B05D0BB68002BC1
S3150800E8D002D03B68002B03D06FF00303FB6137E0DF
S3150800E8E000233B6107F110031A46B968B86901F0BD
S3150800E8F005F90346012B03D06FF00203FB6127E0FD
S3150800E9003B69002B24D0154B4FF080521A60BFF399
S3150800E9104F8FBFF36F8F1BE0BB69002B02D0BB681C
S3150800E920002B03D16FF00303FB6111E03A68B96865
S3150800E930B86900F0F7FE0346012B09D03B68002BA7
S3150800E94003D06FF00103FB6102E06FF00203FB6185
S3150800E950FB6918462037BD4680BD00BF04ED00E0C0
S3150800E96080B485B000AFF860B9607A60FB68074A82
S3150800E9701A60BB68064A1A607B6880221A6000BF64
S3150800E9801437BD465DF8047B704700BFEC040020D1
S3150800E990A805002080B485B000AFF860B9607A6039
S3150800E9A0FB68074A1A60BB68064A1A607B684FF418
S3150800E9B080721A6000BF1437BD465DF8047B704745
S3150800E9C0A80700206408002080B586B000AF7860EC
S3150800E9D07B68002B0AD14FF0500383F31188BFF3ED
S3150800E9E06F8FBFF34F8F3B6100BFFEE72023BB60ED
S3150800E9F0BB68202B0AD04FF0500383F31188BFF36E
S3150800EA006F8FBFF34F8FFB6000BFFEE77B687B61AC
S3150800EA107B69002B0AD07B6900221A607B69043364
S3150800EA20184600F03DFA7B6901221A777B69184679
S3150800EA301837BD4680BD80B582B000AF202003F0F0
S3150800EA403BFA78607B68002B0AD07B6800221A6044
S3150800EA507B680433184600F023FA7B6800221A778D
S3150800EA607B6818460837BD4680BD000080B590B063
S3150800EA7000AFF860B9607A603B60FB687B6300238F
S3150800EA80BB6300233B63FB68002B0AD14FF050039E
S3150800EA9083F31188BFF36F8FBFF34F8F3B6200BFBD
S3150800EAA0FEE7BB6803F07F43002B0AD04FF0500304
S3150800EAB083F31188BFF36F8FBFF34F8FFB6100BFDE
S3150800EAC0FEE7BB68002B0AD14FF0500383F3118889
S3150800EAD0BFF36F8FBFF34F8FBB6100BFFEE702F036
S3150800EAE07FF90346002B02D1BB6C002B01D1012311
S3150800EAF000E00023002B0AD14FF0500383F311885E
S3150800EB00BFF36F8FBFF34F8F7B6100BFFEE701F046
S3150800EB10CDFC7B6B1B68FB623A68B968F86A00F043
S3150800EB2088F9B862BB6A002B0ED0FB6AFB63002328
S3150800EB30BB647B68002B28D07B6B1A68BB68DB43F9
S3150800EB401A407B6B1A6020E0BB6C002B04D1FB6A71
S3150800EB50FB6301233B6318E07B68002B03D0BB6B88
S3150800EB6043F08073BB633B68002B03D0BB6B43F059
S3150800EB708063BB637B6B181DBA68BB6B1343BA6CA7
S3150800EB80194601F091FE0023FB6301F09DFC7862B3
S3150800EB90BB6C002B31D07B6A002B07D1194B4FF089
S3150800EBA080521A60BFF34F8FBFF36F8F02F08EFA51
S3150800EBB0F863FB6B03F00073002B1AD103F05AF8C5
S3150800EBC07B6B1B68FB633A68B968F86B00F031F930
S3150800EBD00346002B09D07B68002B06D07B6B1A688E
S3150800EBE0BB68DB431A407B6B1A6001233B6303F067
S3150800EBF071F8FB6B23F07F43FB63FB6B18464037CA
S3150800EC00BD4680BD04ED00E080B586B000AF7860F3
S3150800EC1039607B687B617B68002B0AD14FF0500313
S3150800EC2083F31188BFF36F8FBFF34F8FFB6000BF6D
S3150800EC30FEE73B6803F07F43002B0AD04FF05003F2
S3150800EC4083F31188BFF36F8FBFF34F8FBB6000BF8D
S3150800EC50FEE703F00FF87B691B683B617B691A685E
S3150800EC603B68DB431A407B691A6003F033F83B695B
S3150800EC7018461837BD4680BD80B584B000AF7860A9
S3150800EC80396000233A687968044802F0A7FEF860FC
S3150800EC90FB6818461037BD4680BD00BF19EE000850
S3150800ECA080B489B000AF78607B68FB61EFF31182AE
S3150800ECB04FF0500383F31188BFF36F8FBFF34F8F65
S3150800ECC0FA60BB60FB68BB61FB691B687B61BB695B
S3150800ECD03B613B6983F3118800BF7B69184624377B
S3150800ECE0BD465DF8047B704780B58EB000AF78608E
S3150800ECF0396000233B637B68BB620023FB627B6849
S3150800ED00002B0AD14FF0500383F31188BFF36F8F9E
S3150800ED10BFF34F8F3B6100BFFEE73B6803F07F43BD
S3150800ED20002B0AD04FF0500383F31188BFF36F8F7F
S3150800ED30BFF34F8FFB6000BFFEE7BB6A04337B62FD
S3150800ED407B6A08333B6201F0B1FB7B6ADB687B6355
S3150800ED50BB6A1A683B681A43BB6A1A603CE07B6B5D
S3150800ED605B68FB617B6B1B68BB610023FB62BB694D
S3150800ED7003F07F437B61BB6923F07F43BB617B69FB
S3150800ED8003F08063002B08D1BB6A1A68BB6913407D
S3150800ED90002B0BD00123FB6208E0BB6A1A68BB692B
S3150800EDA01340BA699A4201D10123FB62FB6A002B20
S3150800EDB010D07B6903F08073002B03D03A6BBB69D4
S3150800EDC013433B63BB6A1B6843F000731946786BB1
S3150800EDD001F036FEFB697B637A6B3B6A9A42BED1C9
S3150800EDE0BB6A1A683B6BDB431A40BB6A1A6001F0C0
S3150800EDF06BFBBB6A1B6818463837BD4680BD80B5B5
S3150800EE0082B000AF7860396039687868FFF76CFFC0
S3150800EE1000BF0837BD4680BD80B582B000AF7860B8
S3150800EE20396039687868FFF7EFFE00BF0837BD46D6
S3150800EE3080BD80B487B000AFF860B9607A600023FF
S3150800EE407B617B68002B07D1FA68BB681340002BEF
S3150800EE500AD001237B6107E0FA68BB681340BA68E9
S3150800EE609A4201D101237B617B6918461C37BD464E
S3150800EE705DF8047B7047000080B586B000AFF86087
S3150800EE80B9607A607B68BA68F968044802F0A6FD3A
S3150800EE9078617B6918461837BD4680BDFFED0008C6
S3150800EEA080B483B000AF78607B6803F108027B68A2
S3150800EEB05A607B684FF0FF329A607B6803F108025C
S3150800EEC07B68DA607B6803F108027B681A617B68F5
S3150800EED000221A6000BF0C37BD465DF8047B7047F8
S3150800EEE080B483B000AF78607B6800221A6100BFE7
S3150800EEF00C37BD465DF8047B704780B485B000AF1B
S3150800EF00786039607B685B68FB603B68FA685A60C2
S3150800EF10FB689A683B689A60FB689B683A685A601F
S3150800EF20FB683A689A603B687A681A617B681B686E
S3150800EF305A1C7B681A6000BF1437BD465DF8047B0F
S3150800EF40704780B485B000AF786039603B681B684D
S3150800EF50BB60BB68B3F1FF3F03D17B681B69FB60ED
S3150800EF600CE07B680833FB6002E0FB685B68FB60CB
S3150800EF70FB685B681B68BA689A42F6D2FB685A68EF
S3150800EF803B685A603B685B683A689A603B68FA680F
S3150800EF909A60FB683A685A603B687A681A617B68C7
S3150800EFA01B685A1C7B681A6000BF1437BD465DF89B
S3150800EFB0047B704780B485B000AF78607B681B69B6
S3150800EFC0FB607B685B687A6892689A607B689B6876
S3150800EFD07A6852685A60FB685B687A689A4203D115
S3150800EFE07B689A68FB685A607B6800221A61FB682E
S3150800EFF01B685A1EFB681A60FB681B68184614379C
S3150800F000BD465DF8047B704780B584B000AF786074
S3150800F01039607B68FB60FB68002B0AD14FF0500310
S3150800F02083F31188BFF36F8FBFF34F8FBB6000BFA9
S3150800F030FEE702F01FFEFB681A68FB68DB6BF968DF
S3150800F040096C01FB03F31A44FB689A60FB6800220B
S3150800F0509A63FB681A68FB685A60FB681A68FB685B
S3150800F060DB6B013BF968096C01FB03F31A44FB6887
S3150800F070DA60FB68FF2283F84420FB68FF2283F8E6
S3150800F08045203B68002B14D1FB681B69002B1AD05E
S3150800F090FB681033184601F06FFC0346002B12D0AC
S3150800F0A00C4B4FF080521A60BFF34F8FBFF36F8F30
S3150800F0B009E0FB6810331846FFF7F2FEFB682433B5
S3150800F0C01846FFF7EDFE02F005FE01231846103735
S3150800F0D0BD4680BD04ED00E080B58EB002AFF86095
S3150800F0E0B9607A603B60FB68002B0AD14FF0500389
S3150800F0F083F31188BFF36F8FBFF34F8FBB6200BFD7
S3150800F100FEE73B68002B0AD14FF0500383F31188C2
S3150800F110BFF36F8FBFF34F8F7B6200BFFEE77B683D
S3150800F120002B02D0BB68002B01D0012300E000238E
S3150800F130002B0AD14FF0500383F31188BFF36F8F6A
S3150800F140BFF34F8F3B6200BFFEE77B68002B02D1FF
S3150800F150BB68002B01D1012300E00023002B0AD154
S3150800F1604FF0500383F31188BFF36F8FBFF34F8FB0
S3150800F170FB6100BFFEE750237B617B69502B0AD0F9
S3150800F1804FF0500383F31188BFF36F8FBFF34F8F90
S3150800F190BB6100BFFEE77B693B68FB62FB6A002B2D
S3150800F1A00DD0FB6A012283F8462097F83820FB6ABF
S3150800F1B0009313467A68B968F86800F03FF8FB6A66
S3150800F1C018463037BD4680BD80B58AB002AFF860B4
S3150800F1D0B9601346FB71FB68002B0AD14FF0500348
S3150800F1E083F31188BFF36F8FBFF34F8F3B6100BF67
S3150800F1F0FEE7FB68BA6802FB03F3FB61FB69503361
S3150800F200184602F059FEB861BB69002B11D0BB69DC
S3150800F2107B617B6950337B61BB69002283F846209A
S3150800F220FA79BB69009313467A69B968F86800F0F9
S3150800F23005F8BB6918462037BD4680BD80B584B041
S3150800F24000AFF860B9607A60FB70BB68002B03D129
S3150800F250BB69BA691A6002E0BB697A681A60BB6959
S3150800F260FA68DA63BB69BA681A640121B869FFF7F4
S3150800F270CBFEBB69FA7883F84C2000BF1037BD4631
S3150800F28080BD80B582B000AF78607B68002B0ED059
S3150800F2907B6800229A607B6800221A607B680022DD
S3150800F2A0DA60002300220021786800F0A1F800BF88
S3150800F2B00837BD4680BD80B586B000AF0346FB71F2
S3150800F2C001237B6100233B61FB791A46396978691A
S3150800F2D0FFF77AFFF860F868FFF7D3FFFB68184670
S3150800F2E01837BD4680BD80B588B002AF0346396081
S3150800F2F0FB7101237B6100233B61FB7900933B682B
S3150800F300002239697869FFF7E7FEF860F868FFF7C1
S3150800F310B8FFFB6818461837BD4680BD90B587B05C
S3150800F32000AF78607B683B613B69002B0AD14FF0E0
S3150800F330500383F31188BFF36F8FBFF34F8FFB60C2
S3150800F34000BFFEE73B699C6801F03AFD03469C4214
S3150800F35011D13B69DB685A1E3B69DA603B69DB6899
S3150800F360002B05D1002300220021386900F040F85F
S3150800F37001237B6101E000237B617B6918461C370A
S3150800F380BD4690BD90B587B000AF786039607B68A0
S3150800F3903B613B69002B0AD14FF0500383F3118878
S3150800F3A0BFF36F8FBFF34F8FFB6000BFFEE73B696C
S3150800F3B09C6801F005FD03469C4207D13B69DB6862
S3150800F3C05A1C3B69DA6001237B610CE039683869AD
S3150800F3D000F088FA78617B69002B04D03B69DB680A
S3150800F3E05A1C3B69DA607B6918461C37BD4690BDD6
S3150800F3F080B58EB000AFF860B9607A603B600023D4
S3150800F4007B63FB683B633B6B002B0AD14FF05003D1
S3150800F41083F31188BFF36F8FBFF34F8FBB6200BFB3
S3150800F420FEE7BB68002B03D13B6B1B6C002B01D19D
S3150800F430012300E00023002B0AD14FF0500383F389
S3150800F4401188BFF36F8FBFF34F8F7B6200BFFEE754
S3150800F4503B68022B03D13B6BDB6B012B01D10123EC
S3150800F46000E00023002B0AD14FF0500383F31188E4
S3150800F470BFF36F8FBFF34F8F3B6200BFFEE701F00C
S3150800F480AFFC0346002B02D17B68002B01D1012378
S3150800F49000E00023002B0AD14FF0500383F31188B4
S3150800F4A0BFF36F8FBFF34F8FFB6100BFFEE702F01C
S3150800F4B0E1FB3B6B9A6B3B6BDB6B9A4202D33B6877
S3150800F4C0022B29D13A68B968386B00F0AFFBF862AD
S3150800F4D03B6B5B6A002B10D03B6B2433184601F05C
S3150800F4E04BFA0346002B13D03F4B4FF080521A605D
S3150800F4F0BFF34F8FBFF36F8F0AE0FB6A002B07D06D
S3150800F500394B4FF080521A60BFF34F8FBFF36F8F9E
S3150800F51002F0E0FB012363E07B68002B03D102F0D5
S3150800F520D9FB00235CE07B6B002B06D107F11403A3
S3150800F530184601F0E7FA01237B6302F0CBFB00F0E3
S3150800F540B5FF02F097FB3B6B93F844305BB2B3F11F
S3150800F550FF3F03D13B6B002283F844203B6B93F8B3
S3150800F56045305BB2B3F1FF3F03D13B6B002283F812
S3150800F570452002F0AFFB3A1D07F114031146184661
S3150800F58001F0D6FA0346002B24D1386B00F046FC6E
S3150800F5900346002B18D03B6B10337A681146184681
S3150800F5A001F05EF9386B00F0D1FB00F08DFF0346E1
S3150800F5B0002B7FF47CAF0C4B4FF080521A60BFF3E0
S3150800F5C04F8FBFF36F8F72E7386B00F0BFFB00F009
S3150800F5D07BFF6CE7386B00F0B9FB00F075FF002382
S3150800F5E018463837BD4680BD04ED00E080B590B0BA
S3150800F5F000AFF860B9607A603B60FB68BB63BB6BC1
S3150800F600002B0AD14FF0500383F31188BFF36F8F95
S3150800F610BFF34F8FBB6200BFFEE7BB68002B03D169
S3150800F620BB6B1B6C002B01D1012300E00023002BD0
S3150800F6300AD14FF0500383F31188BFF36F8FBFF3DE
S3150800F6404F8F7B6200BFFEE73B68022B03D1BB6B83
S3150800F650DB6B012B01D1012300E00023002B0AD12B
S3150800F6604FF0500383F31188BFF36F8FBFF34F8FAB
S3150800F6703B6200BFFEE702F0DFFBEFF311824FF0BB
S3150800F680500383F31188BFF36F8FBFF34F8FFA616F
S3150800F690BB61FB697B63BB6B9A6BBB6BDB6B9A428B
S3150800F6A002D33B68022B2FD1BB6B93F8453087F802
S3150800F6B03330BB6B9B6BFB623A68B968B86B00F07A
S3150800F6C0B5FA97F93330B3F1FF3F12D1BB6B5B6ADA
S3150800F6D0002B16D0BB6B2433184601F04DF90346B0
S3150800F6E0002B0ED07B68002B0BD07B6801221A609A
S3150800F6F007E097F833300133DBB25AB2BB6B83F8B5
S3150800F70045200123FB6301E00023FB637B6B7B61E0
S3150800F7107B6983F3118800BFFB6B18464037BD46EB
S3150800F72080BD000080B58CB000AFF860B9607A6023
S3150800F7300023FB62FB68BB62BB6A002B0AD14FF051
S3150800F740500383F31188BFF36F8FBFF34F8F3B626C
S3150800F75000BFFEE7BB68002B03D1BB6A1B6C002BFE
S3150800F76001D1012300E00023002B0AD14FF05003FA
S3150800F77083F31188BFF36F8FBFF34F8FFB6100BF11
S3150800F780FEE701F02DFB0346002B02D17B68002B18
S3150800F79001D1012300E00023002B0AD14FF05003CA
S3150800F7A083F31188BFF36F8FBFF34F8FBB6100BF21
S3150800F7B0FEE702F05FFABB6A9B6B7B627B6A002BF3
S3150800F7C01FD0B968B86A00F09BFA7B6A5A1EBB6AF2
S3150800F7D09A63BB6A1B69002B0FD0BB6A10331846A5
S3150800F7E001F0CAF80346002B07D03D4B4FF0805274
S3150800F7F01A60BFF34F8FBFF36F8F02F06BFA0123C6
S3150800F80069E07B68002B03D102F064FA002362E00A
S3150800F810FB6A002B06D107F11003184601F072F9AE
S3150800F8200123FB6202F056FA00F040FE02F022FACB
S3150800F830BB6A93F844305BB2B3F1FF3F03D1BB6AAE
S3150800F840002283F84420BB6A93F845305BB2B3F1D3
S3150800F850FF3F03D1BB6A002283F8452002F03AFA3B
S3150800F8603A1D07F110031146184601F061F90346DF
S3150800F870002B23D1B86A00F0BBFA0346002B17D039
S3150800F880BB6A24337A681146184600F0E9FFB86A5D
S3150800F89000F05CFA00F018FE0346002B89D1104BE5
S3150800F8A04FF080521A60BFF34F8FBFF36F8F80E718
S3150800F8B0B86A00F04BFA00F007FE7AE7B86A00F07B
S3150800F8C045FA00F001FEB86A00F092FA0346002BEA
S3150800F8D03FF46FAF002318463037BD4680BD00BFE2
S3150800F8E004ED00E080B58EB000AF78603960002383
S3150800F8F07B637B68FB6200233B63FB6A002B0AD1B0
S3150800F9004FF0500383F31188BFF36F8FBFF34F8F08
S3150800F9103B6200BFFEE7FB6A1B6C002B0AD04FF068
S3150800F920500383F31188BFF36F8FBFF34F8FFB61CB
S3150800F93000BFFEE701F054FA0346002B02D13B68EC
S3150800F940002B01D1012300E00023002B0AD14FF040
S3150800F950500383F31188BFF36F8FBFF34F8FBB61DB
S3150800F96000BFFEE702F086F9FB6A9B6BBB62BB6AC7
S3150800F970002B24D0BB6A5A1EFB6A9A63FB6A1B6873
S3150800F980002B04D101F0BAFB0246FB6A9A60FB6AB7
S3150800F9901B69002B0FD0FB6A1033184600F0ECFFEA
S3150800F9A00346002B07D0544B4FF080521A60BFF322
S3150800F9B04F8FBFF36F8F02F08DF9012397E03B68F5
S3150800F9C0002B11D13B6B002B0AD04FF0500383F369
S3150800F9D01188BFF36F8FBFF34F8F7B6100BFFEE7C0
S3150800F9E002F078F9002382E07B6B002B06D107F141
S3150800F9F00C03184601F086F801237B6302F06AF9C6
S3150800FA0000F054FD02F036F9FB6A93F844305BB215
S3150800FA10B3F1FF3F03D1FB6A002283F84420FB6A57
S3150800FA2093F845305BB2B3F1FF3F03D1FB6A00227E
S3150800FA3083F8452002F04EF93A4607F10C031146C1
S3150800FA40184601F075F80346002B32D1F86A00F023
S3150800FA50CFF90346002B26D0FB6A1B68002B09D179
S3150800FA6002F008F9FB6A9B68184601F0D7F9386373
S3150800FA7002F030F9FB6A24333A681146184600F05A
S3150800FA80EFFEF86A00F062F900F01EFD0346002B4F
S3150800FA907FF468AF184B4FF080521A60BFF34F8F50
S3150800FAA0BFF36F8F5EE7F86A00F050F900F00CFDBF
S3150800FAB058E7F86A00F04AF900F006FDF86A00F01F
S3150800FAC097F90346002B3FF44DAF3B6B002B0DD047
S3150800FAD002F0D0F8F86A00F091F87862FB6A9B6841
S3150800FAE0796A184601F070FA02F0F4F8002318460D
S3150800FAF03837BD4680BD00BF04ED00E080B58EB046
S3150800FB0000AFF860B9607A60FB683B633B6B002B1B
S3150800FB100AD14FF0500383F31188BFF36F8FBFF3F9
S3150800FB204F8F3B6200BFFEE7BB68002B03D13B6BE0
S3150800FB301B6C002B01D1012300E00023002B0AD106
S3150800FB404FF0500383F31188BFF36F8FBFF34F8FC6
S3150800FB50FB6100BFFEE702F06FF9EFF311824FF089
S3150800FB60500383F31188BFF36F8FBFF34F8FBA61CA
S3150800FB707B61BB69FB623B6B9B6BBB62BB6A002B01
S3150800FB802FD03B6B93F8443087F82730B968386B29
S3150800FB9000F0B6F8BB6A5A1E3B6B9A6397F9273092
S3150800FBA0B3F1FF3F12D13B6B1B69002B16D03B6BA1
S3150800FBB01033184600F0E0FE0346002B0ED07B6893
S3150800FBC0002B0BD07B6801221A6007E097F82730D4
S3150800FBD00133DBB25AB23B6B83F8442001237B63C3
S3150800FBE001E000237B63FB6A3B613B6983F3118871
S3150800FBF000BF7B6B18463837BD4680BD80B485B0DC
S3150800FC0000AF78607B685B6A002B06D07B681B6B4D
S3150800FC101B68C3F13803FB6001E00023FB60FB6847
S3150800FC2018461437BD465DF8047B704780B586B024
S3150800FC3000AFF860B9607A6000237B61FB689B6B54
S3150800FC403B61FB681B6C002B0DD1FB681B68002B06
S3150800FC504DD1FB689B68184601F048F97861FB6846
S3150800FC6000229A6043E07B68002B19D1FB6858682C
S3150800FC70FB681B6C1A46B96802F058FBFB685A68A1
S3150800FC80FB681B6C1A44FB685A60FB685A68FB6879
S3150800FC909B689A422BD3FB681A68FB685A6026E071
S3150800FCA0FB68D868FB681B6C1A46B96802F03EFB0D
S3150800FCB0FB68DA68FB681B6C5B421A44FB68DA600F
S3150800FCC0FB68DA68FB681B689A4207D2FB689A6881
S3150800FCD0FB681B6C5B421A44FB68DA607B68022B84
S3150800FCE005D13B69002B02D03B69013B3B613B696F
S3150800FCF05A1CFB689A637B6918461837BD4680BD4F
S3150800FD0080B582B000AF786039607B681B6C002BC9
S3150800FD1018D07B68DA687B681B6C1A447B68DA60E3
S3150800FD207B68DA687B689B689A4203D37B681A68A3
S3150800FD307B68DA607B68D9687B681B6C1A4638680A
S3150800FD4002F0F4FA00BF0837BD4680BD80B584B01E
S3150800FD5000AF786001F08EFF7B6893F84530FB733F
S3150800FD6011E07B685B6A002B12D07B682433184647
S3150800FD7000F002FE0346002B01D000F03BFFFB7BA0
S3150800FD80013BDBB2FB7397F90F30002BE9DC00E08F
S3150800FD9000BF7B68FF2283F8452001F09BFF01F036
S3150800FDA069FF7B6893F84430BB7311E07B681B6975
S3150800FDB0002B12D07B681033184600F0DDFD034691
S3150800FDC0002B01D000F016FFBB7B013BDBB2BB73F7
S3150800FDD097F90E30002BE9DC00E000BF7B68FF22B4
S3150800FDE083F8442001F076FF00BF1037BD4680BD7A
S3150800FDF080B584B000AF786001F03CFF7B689B6BF0
S3150800FE00002B02D10123FB6001E00023FB6001F017
S3150800FE1061FFFB6818461037BD4680BD80B584B0C3
S3150800FE2000AF786001F026FF7B689A6B7B68DB6B16
S3150800FE309A4202D10123FB6001E00023FB6001F036
S3150800FE4049FFFB6818461037BD4680BD80B485B0AB
S3150800FE5000AF786039600023FB6014E00F4AFB6846
S3150800FE6052F83330002B0BD10C49FB683A6841F83D
S3150800FE7033200A4AFB68DB0013447A685A6006E0B6
S3150800FE80FB680133FB60FB68072BE7D900BF00BF9F
S3150800FE901437BD465DF8047B704700BF640C00202C
S3150800FEA080B586B000AFF860B9607A60FB687B61A0
S3150800FEB001F0E0FE7B6993F844305BB2B3F1FF3F93
S3150800FEC003D17B69002283F844207B6993F8453087
S3150800FED05BB2B3F1FF3F03D17B69002283F845206B
S3150800FEE001F0F8FE7B699B6B002B06D17B692433F6
S3150800FEF07A68B968184600F013FD7869FFF726FF97
S3150800FF0000BF1837BD4680BD80B58EB004AFF86017
S3150800FF10B9607A603B607B6B002B0AD14FF05003C7
S3150800FF2083F31188BFF36F8FBFF34F8F3B6200BF18
S3150800FF30FEE7BB6B002B0AD14FF0500383F3118801
S3150800FF40BFF36F8FBFF34F8FFB6100BFFEE7BC2384
S3150800FF503B613B69BC2B0AD04FF0500383F31188F1
S3150800FF60BFF36F8FBFF34F8FBB6100BFFEE73B69DF
S3150800FF70BB6B002B1ED07B6B002B1BD0BB6B7B6235
S3150800FF807B6A7A6B1A637B6A022283F8B92000239C
S3150800FF9003937B6A029307F1140301933B6B009367
S3150800FFA03B687A68B968F86800F050F8786A00F033
S3150800FFB0F3F801E000237B617B6918462837BD46C4
S3150800FFC080BD80B58CB004AFF860B9603B6013465D
S3150800FFD0FB80FB889B00184601F06EFF78617B6901
S3150800FFE0002B0ED0BC2001F067FFF861FB69002BDF
S3150800FFF003D0FB697A691A6305E0786902F028F884
S3150801000001E00023FB61FB69002B17D0FB69002285
S3150801001083F8B920FA8800230393FB690293FB6AE4
S315080100200193BB6A00933B68B968F86800F00EF85B
S31508010030F86900F0B1F80123BB6102E04FF0FF3324
S31508010040BB61BB6918462037BD4680BD80B588B0FF
S3150801005000AFF860B9607A603B603B6B186B7B68F0
S315080100609B001A46A52102F06FF93B6B1A6B7B6858
S3150801007003F18043013B9B001344BB61BB6923F039
S315080100800703BB61BB6903F00703002B0AD04FF0D6
S31508010090500383F31188BFF36F8FBFF34F8F7B61D3
S315080100A000BFFEE7BB68002B1FD00023FB6112E0EF
S315080100B0BA68FB69134419783A6BFB6913443433FC
S315080100C00A461A70BA68FB6913441B78002B06D0D6
S315080100D0FB690133FB61FB690F2BE9D900E000BF1E
S315080100E03B6B002283F8432003E03B6B002283F835
S315080100F03420BB6A372B01D93723BB623B6BBA6AFB
S31508010100DA623B6BBA6ADA643B6B00221A653B6BAF
S3150801011004331846FEF7E4FE3B6B18331846FEF720
S31508010120DFFE3B6B3A6B1A61BB6AC3F138023B6B64
S315080101309A613B6B3A6B5A623B6B0022C3F8B42057
S315080101403B6B002283F8B8203B6B543360220021B5
S31508010150184602F0F9F83B6B0C4A9A653B6B0C4A58
S31508010160DA653B6B0B4A1A663A68F968B86901F0B1
S3150801017055FC02463B6B1A60FB6A002B02D0FB6AF0
S315080101803A6B1A6000BF2037BD4680BDD02A0108E8
S31508010190F02A0108B02A010880B582B000AF78605C
S315080101A001F068FD2D4B1B6801332C4A13602C4B5B
S315080101B01B68002B09D12A4A7B681360274B1B68E9
S315080101C0012B10D100F03AFD0DE0264B1B68002BE0
S315080101D009D1234B1B68DA6A7B68DB6A9A4202D823
S315080101E01F4A7B681360204B1B6801331E4A136044
S315080101F01D4B1A687B685A647B68DA6A1B4B1B6855
S315080102009A4203D97B68DB6A184A13607B68DA6A03
S3150801021013469B0013449B00154A1A447B68043312
S3150801022019461046FEF769FE01F054FD0D4B1B6891
S31508010230002B0ED00A4B1B68DA6A7B68DB6A9A4286
S3150801024007D20C4B4FF080521A60BFF34F8FBFF3A2
S315080102506F8F00BF0837BD4680BD00BF78110020EB
S31508010260A40C002084110020941100208011002084
S31508010270A80C002004ED00E080B584B000AF7860DA
S315080102800023FB607B68002B17D0134B1B68002BE0
S315080102900AD04FF0500383F31188BFF36F8FBFF372
S315080102A04F8FBB6000BFFEE700F000F900217868B8
S315080102B000F038FF00F008F9F860FB68002B07D159
S315080102C0064B4FF080521A60BFF34F8FBFF36F8F03
S315080102D000BF1037BD4680BDA011002004ED00E027
S315080102E080B584B000AF786001F0C4FC7B68002B50
S315080102F002D1304B1B6800E07B68FB60FB68043366
S315080103001846FEF757FEFB689B6A002B04D0FB686C
S3150801031018331846FEF74EFEFB680433194626487D
S31508010320FEF7EBFDFB6893F8B830DBB2012B03D17E
S31508010330FB68002283F8B82001F0CCFC1F4B1B6830
S31508010340002B05D001F096FC00F01AFD01F0C2FC65
S31508010350184B1B68FA689A4227D1184B1B68002B61
S3150801036017D0174B1B68002B0AD04FF0500383F3A5
S315080103701188BFF36F8FBFF34F8FBB6000BFFEE7D6
S31508010380104B4FF080521A60BFF34F8FBFF36F8F38
S315080103900BE0094B1A680C4B1B689A4203D1054BB3
S315080103A000221A6001E000F0F7F900BF1037BD46D8
S315080103B080BD00BFA40C0020641100208411002018
S315080103C0A011002004ED00E07811002080B58AB064
S315080103D004AF0023BB6000237B603A46391D07F151
S315080103E008031846FEF7BCFA39687B68BA680292B0
S315080103F001930023009300230A4624492448FFF762
S3150801040083FD0346234A1360224B1B68002B02D047
S3150801041001237B6101E000237B617B69012B02D10A
S3150801042000F0D4FE78617B69012B1BD14FF0500394
S3150801043083F31188BFF36F8FBFF34F8F3B6100BF03
S31508010440154B1B685433154A1360154B4FF0FF3291
S315080104501A60144B01221A60134B00221A6001F02C
S3150801046067FB0EE07B69B3F1FF3F0AD14FF05003FA
S3150801047083F31188BFF36F8FBFF34F8FFB6000BF04
S31508010480FEE700BF1837BD4680BD00BF1826010824
S315080104900D0C01089C110020A40C0020DC00002092
S315080104A098110020841100207C11002080B400AF2F
S315080104B0044B1B680133034A136000BFBD465DF850
S315080104C0047B7047A011002080B584B000AF0023DB
S315080104D0FB600023BB60424B1B68002B0AD14FF01F
S315080104E0500383F31188BFF36F8FBFF34F8F3B60C0
S315080104F000BFFEE701F0BEFB394B1B68013B384ADA
S315080105001360374B1B68002B62D1364B1B68002BD7
S315080105105ED02FE0344BDB68DB68FB60FB68183381
S315080105201846FEF747FDFB6804331846FEF742FDF9
S31508010530FB68DA6A2D4B1B689A4203D9FB68DB6AAA
S315080105402A4A1360FB68DA6A13469B0013449B0028
S31508010550274A1A44FB68043319461046FEF7CDFCB0
S31508010560FB68DA6A234B1B68DB6A9A4202D3224B81
S3150801057001221A601C4B1B68002BCBD1FB68002B90
S3150801058001D000F0FDFB1D4B1B687B607B68002BCF
S3150801059010D000F047F80346002B02D0164B012273
S315080105A01A607B68013B7B607B68002BF1D1134B9A
S315080105B000221A60104B1B68002B09D00123BB606F
S315080105C00F4B4FF080521A60BFF34F8FBFF36F8FF7
S315080105D001F080FBBB6818461037BD4680BD00BFD9
S315080105E0A011002078110020381100208011002068
S315080105F0A80C0020A40C00208C11002088110020D2
S3150801060004ED00E080B483B000AF054B1B687B6046
S315080106107B6818460C37BD465DF8047B704700BFFA
S315080106207C11002080B586B000AF00237B614F4B5B
S315080106301B68002B40F08F804D4B1B6801333B61D3
S315080106404B4A3B6913603B69002B20D1494B1B6818
S315080106501B68002B0AD04FF0500383F31188BFF3B0
S315080106606F8FBFF34F8F3B6000BFFEE7414B1B689F
S31508010670FB60414B1B683F4A13603F4AFB681360A6
S315080106803E4B1B6801333D4A136000F079FB3C4B36
S315080106901B683A699A4249D3364B1B681B68002B7B
S315080106A004D1374B4FF0FF321A603FE0314B1B68DC
S315080106B0DB68DB68BB60BB685B687B603A697B6843
S315080106C09A4203D22E4A7B6813602FE0BB68043333
S315080106D01846FEF76FFCBB689B6A002B04D0BB6803
S315080106E018331846FEF766FCBB68DA6A254B1B68A1
S315080106F09A4203D9BB68DB6A224A1360BB68DA6A85
S3150801070013469B0013449B001F4A1A44BB680433D3
S3150801071019461046FEF7F1FBBB68DA6A1B4B1B68E4
S31508010720DB6A9A42B8D301237B61B5E7174B1B688D
S31508010730DA6A154913469B0013449B000B441B6850
S31508010740012B01D901237B61114B1B68002B07D0B3
S3150801075001237B6104E00F4B1B6801330D4A1360CB
S315080107607B6918461837BD4680BD00BFA011002019
S315080107707C11002030110020341100209011002036
S315080107809811002080110020A80C0020A40C00203C
S315080107908C1100208811002080B485B000AF2A4B47
S315080107A01B68002B03D0294B01221A6046E0274B10
S315080107B000221A60264B1B68FB6010E0FB68002BC1
S315080107C00AD14FF0500383F31188BFF36F8FBFF33C
S315080107D04F8F7B6000BFFEE7FB68013BFB601D494D
S315080107E0FA6813469B0013449B000B441B68002BB5
S315080107F0E4D0FA6813469B0013449B00154A134438
S31508010800BB60BB685B685A68BB685A60BB685A6854
S31508010810BB6808339A4204D1BB685B685A68BB68EF
S315080108205A60BB685B68DB680B4A1360084AFB6859
S315080108301360094B1B685433084A136000BF143709
S31508010840BD465DF8047B7047A01100208C1100207D
S3150801085080110020A80C0020A40C0020DC00002038
S3150801086080B584B000AF786039607B68002B0AD107
S315080108704FF0500383F31188BFF36F8FBFF34F8F88
S31508010880FB6000BFFEE7074B1B68183319467868FB
S31508010890FEF757FB0121386800F044FC00BF10370A
S315080108A0BD4680BDA40C002080B586B000AFF860B7
S315080108B0B9607A60FB68002B0AD14FF0500383F3C5
S315080108C01188BFF36F8FBFF34F8F7B6100BFFEE7C0
S315080108D0114B1B68002B0AD14FF0500383F3118883
S315080108E0BFF36F8FBFF34F8F3B6100BFFEE70B4B23
S315080108F01B68BA6842F000429A61084B1B681833B4
S315080109001946F868FEF7F9FA0121786800F00AFC39
S3150801091000BF1837BD4680BDA0110020A40C0020D9
S3150801092080B586B000AFF860B9607A60FB68002BC5
S315080109300AD14FF0500383F31188BFF36F8FBFF3CA
S315080109404F8F7B6100BFFEE70A4B1B6818331946B8
S31508010950F868FEF7D2FA7B68002B02D04FF0FF3316
S31508010960BB607968B86800F0DDFB00BF1837BD4683
S3150801097080BD00BFA40C002080B586B000AF7860AA
S315080109807B68DB68DB683B613B69002B0AD14FF06A
S31508010990500383F31188BFF36F8FBFF34F8FFB604B
S315080109A000BFFEE73B6918331846FEF703FB1E4BEB
S315080109B01B68002B1DD13B6904331846FEF7FAFA6A
S315080109C03B69DA6A194B1B689A4203D93B69DB6AA8
S315080109D0164A13603B69DA6A13469B0013449B0067
S315080109E0134A1A443B69043319461046FEF785FA39
S315080109F005E03B69183319460E48FEF77EFA3B694E
S31508010A00DA6A0D4B1B68DB6A9A4205D901237B61B9
S31508010A100A4B01221A6001E000237B617B691846B3
S31508010A201837BD4680BD00BFA011002080110020E7
S31508010A30A80C002038110020A40C00208C110020DD
S31508010A4080B586B000AF78603960294B1B68002BEA
S31508010A500AD14FF0500383F31188BFF36F8FBFF3A9
S31508010A604F8F3B6100BFFEE73B6843F000427B685E
S31508010A701A607B68DB687B617B69002B0AD14FF0C2
S31508010A80500383F31188BFF36F8FBFF34F8FFB605A
S31508010A9000BFFEE77868FEF78DFA7B6904331846CE
S31508010AA0FEF788FA7B69DA6A124B1B689A4203D900
S31508010AB07B69DB6A0F4A13607B69DA6A13469B0016
S31508010AC013449B000C4A1A447B69043319461046A1
S31508010AD0FEF713FA7B69DA6A084B1B68DB6A9A42E6
S31508010AE002D9074B01221A6000BF1837BD4680BDDF
S31508010AF0A011002080110020A80C0020A40C0020C1
S31508010B008C11002080B483B000AF7860064B1A6858
S31508010B107B681A60054B1A687B685A6000BF0C37F8
S31508010B20BD465DF8047B7047901100207C110020BA
S31508010B3080B588B000AF786039607B68002B0AD130
S31508010B404FF0500383F31188BFF36F8FBFF34F8FB5
S31508010B503B6100BFFEE73B68002B0AD14FF050030B
S31508010B6083F31188BFF36F8FBFF34F8FFB6000BF0D
S31508010B70FEE701F07FF81D4B1B68BB617B685B686C
S31508010B80BA69D31A7B613B681B68B3F1FF3F02D18F
S31508010B900023FB6123E07B681A68154B1B689A42A0
S31508010BA007D07B685B68BA699A4202D30123FB6165
S31508010BB015E03B681B687A699A420BD23B681A684A
S31508010BC07B69D21A3B681A607868FFF79BFF002396
S31508010BD0FB6104E03B6800221A600123FB6101F016
S31508010BE079F8FB6918462037BD4680BD7C1100207F
S31508010BF09011002080B400AF034B01221A6000BF98
S31508010C00BD465DF8047B70478C11002080B582B023
S31508010C1000AF786000F052F8064B1B68012BF9D932
S31508010C20054B4FF080521A60BFF34F8FBFF36F8F9A
S31508010C30F0E700BFA80C002004ED00E080B582B003
S31508010C4000AF00237B600CE07A6813469B001344CF
S31508010C509B00124A13441846FEF722F97B680133B2
S31508010C607B607B68372BEFD90D48FEF719F90D48DC
S31508010C70FEF716F90C48FEF713F90C48FEF710F9BA
S31508010C800B48FEF70DF90B4B054A1A600A4B054A44
S31508010C901A6000BF0837BD4680BD00BFA80C0020FA
S31508010CA0081100201C110020381100204C110020C9
S31508010CB064110020301100203411002080B582B063
S31508010CC000AF19E000F0D6FF104BDB68DB687B60EC
S31508010CD07B6804331846FEF76DF90D4B1B68013B1B
S31508010CE00B4A13600B4B1B68013B0A4A136000F061
S31508010CF0F1FF786800F010F8064B1B68002BE1D16C
S31508010D0000BF00BF0837BD4680BD00BF4C1100209B
S31508010D10781100206011002080B584B000AF78609A
S31508010D207B685433184601F025FB7B6893F8B93084
S31508010D30002B08D17B681B6B184601F089F9786886
S31508010D4001F086F918E07B6893F8B930012B03D1D5
S31508010D50786801F07DF90FE07B6893F8B930022BCA
S31508010D600AD04FF0500383F31188BFF36F8FBFF397
S31508010D704F8FFB6000BFFEE700BF1037BD4680BD41
S31508010D8080B483B000AF0C4B1B681B68002B04D1E1
S31508010D900A4B4FF0FF321A6008E0074B1B68DB6805
S31508010DA0DB687B607B685B68044A136000BF0C37AD
S31508010DB0BD465DF8047B704730110020981100206C
S31508010DC080B483B000AF054B1B687B607B6818460F
S31508010DD00C37BD465DF8047B704700BFA40C0020A4
S31508010DE080B483B000AF0B4B1B68002B02D10123E3
S31508010DF07B6008E0084B1B68002B02D102237B604D
S31508010E0001E000237B607B6818460C37BD465DF818
S31508010E10047B704784110020A011002080B584B09E
S31508010E2000AF78607B68BB600023FB607B68002BA2
S31508010E3051D0BB68DA6A2A4B1B68DB6A9A4241D2EF
S31508010E40BB689B69002B06DB254B1B68DB6AC3F174
S31508010E503802BB689A61BB685969BB68DA6A134686
S31508010E609B0013449B001F4A1344994222D1BB6835
S31508010E7004331846FEF79EF8194B1B68DA6ABB68F5
S31508010E80DA62BB68DA6A184B1B689A4203D9BB68EF
S31508010E90DB6A154A1360BB68DA6A13469B0013447A
S31508010EA09B00104A1A44BB68043319461046FEF7DC
S31508010EB024F804E00A4B1B68DA6ABB68DA62012384
S31508010EC0FB6008E0BB68DA6C054B1B68DB6A9A4273
S31508010ED001D20123FB60FB6818461037BD4680BD69
S31508010EE0A40C0020A80C00208011002080B586B033
S31508010EF000AF78607B683B6100237B617B68002BD0
S31508010F0056D02E4B1B683A699A420AD04FF05003C5
S31508010F1083F31188BFF36F8FBFF34F8FFB6000BF59
S31508010F20FEE73B691B6D002B0AD14FF0500383F393
S31508010F301188BFF36F8FBFF34F8FBB6000BFFEE70A
S31508010F403B691B6D5A1E3B691A653B69DA6A3B693F
S31508010F50DB6C9A422CD03B691B6D002B28D13B696F
S31508010F6004331846FEF726F83B69DA6C3B69DA6200
S31508010F703B69DB6AC3F138023B699A613B69DA6A04
S31508010F800F4B1B689A4203D93B69DB6A0C4A13600B
S31508010F903B69DA6A13469B0013449B00094A1A44C3
S31508010FA03B69043319461046FDF7A7FF01237B6108
S31508010FB07B6918461837BD4680BD00BFA40C0020C2
S31508010FC080110020A80C002080B588B000AF786099
S31508010FD039607B68BB6101237B617B68002B6AD022
S31508010FE0BB691B6D002B0AD14FF0500383F311889F
S31508010FF0BFF36F8FBFF34F8FFB6000BFFEE7BB697F
S31508011000DB6C3A689A4202D93B68FB6102E0BB692C
S31508011010DB6CFB61BB69DB6AFA699A424BD0BB6937
S315080110201B6D7A699A4246D1254B1B68BA699A4261
S315080110300AD14FF0500383F31188BFF36F8FBFF3C3
S315080110404F8FBB6000BFFEE7BB69DB6A3B61BB69CB
S31508011050FA69DA62BB699B69002B04DBFB69C3F198
S315080110603802BB699A61BB6959693A6913469B009B
S3150801107013449B00134A134499421CD1BB69043398
S315080110801846FDF797FFBB69DA6A0F4B1B689A4248
S3150801109003D9BB69DB6A0C4A1360BB69DA6A134672
S315080110A09B0013449B00074A1A44BB69043319463B
S315080110B01046FDF722FF00BF2037BD4680BD00BFA1
S315080110C0A40C0020A80C00208011002080B483B055
S315080110D000AF094B1B689B697B60074B1B68DA6A83
S315080110E0054B1B68C2F138029A617B6818460C37B2
S315080110F0BD465DF8047B7047A40C002080B400AFA0
S31508011100074B1B68002B04D0054B1B681A6D01326F
S315080111101A65034B1B681846BD465DF8047B704784
S31508011120A40C002080B584B000AF78603960214BEB
S315080111301B68FB60204B1B6804331846FDF73AFF12
S315080111407B68B3F1FF3F0AD13B68002B07D01A4BE6
S315080111501B68043319461948FDF7CFFE26E0FA68DD
S315080111607B681344BB60144B1B68BA685A60BA683B
S31508011170FB689A4209D2124B1A680F4B1B68043353
S3150801118019461046FDF7DDFE10E00E4B1A680A4BAC
S315080111901B68043319461046FDF7D3FE0A4B1B6834
S315080111A0BA689A4202D2084ABB68136000BF103770
S315080111B0BD4680BD7C110020A40C002064110020CE
S315080111C034110020301100209811002080B58AB012
S315080111D004AF00237B6100F0A1FB1C4B1B68002BAD
S315080111E021D00023FB600023BB603A1D07F10801EB
S315080111F007F10C031846FDF7CDFB7968BB68FA6859
S31508011200029201930223009300230A4610491148CA
S31508011210FEF77AFE0346104A13600F4B1B68002B34
S3150801122001D001237B617B69002B0AD14FF0500362
S3150801123083F31188BFF36F8FBFF34F8F3B6100BFF5
S31508011240FEE77B6918461837BD4680BDD4110020D4
S3150801125020260108C5140108D811002080B588B0D8
S3150801126002AFF860B9607A603B602C2000F024FE7A
S3150801127078617B69002B0DD07B69002283F82820D1
S315080112807B6901933B6A00933B687A68B968F86899
S3150801129000F043F87B6918461837BD4680BD80B50E
S315080112A08AB002AFF860B9607A603B602C233B6173
S315080112B03B692C2B0AD04FF0500383F31188BFF3F7
S315080112C06F8FBFF34F8FBB6100BFFEE73B69FB6AB8
S315080112D0002B0AD14FF0500383F31188BFF36F8FA8
S315080112E0BFF34F8F7B6100BFFEE7FB6AFB61FB69BA
S315080112F0002B0DD0FB69022283F82820FB69019394
S31508011300BB6A00933B687A68B968F86800F005F823
S31508011310FB6918462037BD4680BD80B586B000AF4B
S31508011320F860B9607A603B60BB68002B0AD14FF060
S31508011330500383F31188BFF36F8FBFF34F8F7B6120
S3150801134000BFFEE77B6A002B1ED000F0E7FA7B6A36
S31508011350FA681A607B6ABA689A617B6A3A68DA61DE
S315080113607B6A3A6A1A627B6A04331846FDF7B8FD46
S315080113707B68002B08D07B6A93F8283043F0040376
S31508011380DAB27B6A83F8282000BF1837BD4680BDCC
S3150801139080B58AB000AFF860B9607A603B60002317
S315080113A07B62FB68002B0AD14FF0500383F3118847
S315080113B0BFF36F8FBFF34F8F3B6200BFFEE71A4B38
S315080113C01B68002B2AD0BB683B617B687B61FB6885
S315080113D0BB61BB68052B18DCFFF702FD0346022B30
S315080113E009D1114B186807F1100100233A6BFDF773
S315080113F0FFFF786212E00C4B186807F11001002311
S315080114000022FDF7F5FF786208E0074B186807F137
S31508011410100100233A68FEF7E9F878627B6A1846F4
S315080114202837BD4680BD00BFD411002080B588B0DD
S3150801143002AF78603960224B1B68DB68DB687B6129
S315080114407B6904331846FDF7B5FD7B6993F82830A7
S3150801145003F00403002B22D07B699A697B68D118B3
S315080114607B683A68786900F0D1F80346002B1FD0EB
S315080114700023009300237A6800217869FFF788FF23
S3150801148038613B69002B13D14FF0500383F3118860
S31508011490BFF36F8FBFF34F8FFB6000BFFEE77B691A
S315080114A093F8283023F00103DAB27B6983F8282000
S315080114B07B691B6A7869984700BF1837BD4680BDA6
S315080114C0CC11002080B584B000AF786007F108031D
S315080114D0184600F057F8F860BB681946F86800F036
S315080114E003F800F0D5F8F1E780B584B000AF78606D
S315080114F03960FEF7DBFF07F10803184600F066F8C6
S31508011500F860BB68002B30D13B68002B0AD17A689A
S31508011510FB689A4206D8FEF7D7FFF9687868FFF79D
S3150801152085FF24E03B68002B08D0134B1B681B681A
S31508011530002B01D1012300E000233B600F4B186803
S315080115407A68FB68D31A3A681946FEF7A9FCFEF7CA
S31508011550BBFF0346002B0AD1094B4FF080521A6094
S31508011560BFF34F8FBFF36F8F01E0FEF7ADFF00BFEB
S315080115701037BD4680BD00BFD0110020D411002010
S3150801158004ED00E080B485B000AF78600E4B1B68AF
S315080115901B68002B01D1012200E000227B681A603A
S315080115A07B681B68002B05D1074B1B68DB681B682A
S315080115B0FB6001E00023FB60FB6818461437BD4653
S315080115C05DF8047B704700BFCC11002080B584B05C
S315080115D000AF7860FFF716F8F8600B4B1B68FA68DE
S315080115E09A4205D200F036F97B6801221A6002E0B8
S315080115F07B6800221A60044AFB681360FB68184678
S315080116001037BD4680BD00BFDC11002080B586B00D
S3150801161000AFF860B9607A603B6000237B61FB68C4
S31508011620BA685A60FB68FA681A61BA687B689A42AE
S3150801163012D87A683B68D21AFB689B699A4202D328
S3150801164001237B611BE0104B1A68FB6804331946BA
S315080116501046FDF776FC12E07A683B689A4206D294
S31508011660BA683B689A4202D301237B6107E0074BBC
S315080116701A68FB68043319461046FDF762FC7B6954
S3150801168018461837BD4680BDD0110020CC11002060
S3150801169080B58EB002AFCAE07B68002B18DA3B1D15
S315080116A00433FB62FB6A002B0AD14FF0500383F324
S315080116B01188BFF36F8FBFF34F8FFB6100BFFEE742
S315080116C0FB6A1B68FA6A5068FA6A92681146984773
S315080116D07B68002BC0F2AA80FB68BB62BB6A5B69A8
S315080116E0002B04D0BB6A04331846FDF763FC3B465E
S315080116F01846FFF76BFF78627B68092B00F2978023
S3150801170001A252F823F000BF311701083117010869
S3150801171031170108A5170108B917010803180108A7
S315080117203117010831170108A5170108B91701086A
S31508011730BB6A93F8283043F00103DAB2BB6A83F82F
S315080117402820BA68BB6A9B69D118BB687A6AB86AE5
S31508011750FFF75CFF0346002B69D0BB6A1B6AB86AB0
S315080117609847BB6A93F8283003F00403002B5ED030
S31508011770BA68BB6A9B691A440023009300230021B7
S31508011780B86AFFF705FE38623B6A002B4FD14FF066
S31508011790500383F31188BFF36F8FBFF34F8FBB617C
S315080117A000BFFEE7BB6A93F8283023F00103DAB2DB
S315080117B0BB6A83F828203AE0BB6A93F8283043F0DD
S315080117C00103DAB2BB6A83F82820BA68BB6A9A6150
S315080117D0BB6A9B69002B0AD14FF0500383F311882A
S315080117E0BFF36F8FBFF34F8F7B6100BFFEE7BB6A05
S315080117F09A697B6AD1187B6A7A6AB86AFFF706FF23
S3150801180015E0BB6A93F8283003F00203002B03D1D5
S31508011810B86A00F01DFC0AE0BB6A93F8283023F089
S315080118200103DAB2BB6A83F8282000E000BF084B3F
S315080118301B68391D00221846FDF774FF0346002B65
S315080118407FF42AAF00BF00BF3037BD4680BD00BF59
S31508011850D411002080B588B002AF48E02D4B1B6833
S31508011860DB681B683B612B4B1B68DB68DB68FB602D
S31508011870FB6804331846FDF79DFBFB681B6AF8688D
S315080118809847FB6893F8283003F00403002B2ED001
S31508011890FB689B693A691344BB60BA683B699A421B
S315080118A00ED9FB68BA685A60FB68FA681A61194B5F
S315080118B01A68FB68043319461046FDF742FB16E021
S315080118C00023009300233A690021F868FFF760FDB9
S315080118D078607B68002B0AD14FF0500383F3118897
S315080118E0BFF36F8FBFF34F8F3B6000BFFEE7094B16
S315080118F01B681B68002BB1D1064B1B687B61064B25
S315080119001B68044A1360044A7B69136000BF1837D1
S31508011910BD4680BDCC110020D011002080B582B013
S3150801192002AF00F0A7F9154B1B68002B20D114480C
S31508011930FDF7B6FA1348FDF7B3FA134B104A1A60C6
S31508011940124B104A1A6000230093114B114A1021B9
S315080119500A20FDF7C1FB0346084A1360074B1B68BB
S31508011960002B05D0054B1B680B491846FEF76EFA86
S3150801197000F0B0F900BFBD4680BD00BFD4110020FC
S31508011980A4110020B8110020CC110020D01100208C
S3150801199080120020E01100202826010880B586B0B3
S315080119A000AF78607B687B617B68002B0AD14FF0BA
S315080119B0500383F31188BFF36F8FBFF34F8FFB601B
S315080119C000BFFEE700F056F97B69DB693B6100F071
S315080119D081F93B6918461837BD4680BD80B58AB07E
S315080119E000AFF860B9607A603B606FF001037B6114
S315080119F0FB68BB61BB68FB617B683B62064B186889
S31508011A0007F1140100233A68FDF7F0FD78627B6A55
S31508011A1018462837BD4680BDD411002080B485B04C
S31508011A2000AFF860B9607A60FB68043BFB60FB684D
S31508011A304FF080721A60FB68043BFB60BB6823F0B9
S31508011A400102FB681A60FB68043BFB600C4AFB68F1
S31508011A501A60FB68143BFB607A68FB681A60FB68CE
S31508011A60043BFB60FB686FF002021A60FB68203BCF
S31508011A70FB60FB6818461437BD465DF8047B704762
S31508011A80851A010880B485B000AF00237B60124B2C
S31508011A901B68B3F1FF3F0AD04FF0500383F3118857
S31508011AA0BFF36F8FBFF34F8FFB6000BFFEE74FF0A9
S31508011AB0500383F31188BFF36F8FBFF34F8FBB605A
S31508011AC000BF00BF7B68002BFCD000BF00BF1437E6
S31508011AD0BD465DF8047B7047D80000200000000071
S31508011AE0074B19680868B0E8F04F80F30988BFF317
S31508011AF06F8F4FF0000080F311887047AFF30080B5
S31508011B00A40C002000BF00BF08480068006880F3E5
S31508011B1008884FF0000080F3148862B661B6BFF3F7
S31508011B204F8FBFF36F8F00DF00BF00BF08ED00E0E6
S31508011B3080B586B000AF464B1B68464A93420AD128
S31508011B404FF0500383F31188BFF36F8FBFF34F8FA5
S31508011B503B6100BFFEE73E4B1B683F4A93420AD1F1
S31508011B604FF0500383F31188BFF36F8FBFF34F8F85
S31508011B70FB6000BFFEE7394B7B617B691B78DBB2F3
S31508011B807B607B69FF221A707B691B78DBB2FB706D
S31508011B90FB78DBB203F05003DAB2314B1A70314BE2
S31508011BA007221A6009E02F4B1B68013B2D4A136077
S31508011BB0FB78DBB25B00DBB2FB70FB78DBB203F0D0
S31508011BC08003802BEFD0274B1B68C3F10703042B37
S31508011BD00AD04FF0500383F31188BFF36F8FBFF319
S31508011BE04F8FBB6000BFFEE71E4B1B681B021D4AD9
S31508011BF013601C4B1B6803F4E0631A4A13607B6885
S31508011C00DAB27B691A70184B1B68174A43F47003DA
S31508011C101360154B1B68144A43F07043136000F0B8
S31508011C20DDF8124B00221A6000F0FCF8104B1B6815
S31508011C300F4A43F040431360FFF766FFFEF7ACFD1A
S31508011C40FFF720FF002318461837BD4680BD00BFA1
S31508011C5000ED00E071C20F4170C20F4100E400E0DF
S31508011C60D0120020D412002020ED00E0D800002078
S31508011C7034EF00E080B483B000AF4FF0500383F334
S31508011C801188BFF36F8FBFF34F8F7B6000BF0F4B78
S31508011C901B6801330D4A13600C4B1B68012B0FD1CE
S31508011CA00B4B1B68DBB2002B0AD04FF0500383F3B2
S31508011CB01188BFF36F8FBFF34F8F3B6000BFFEE7FD
S31508011CC000BF0C37BD465DF8047B7047D80000207D
S31508011CD004ED00E080B483B000AF124B1B68002B03
S31508011CE00AD14FF0500383F31188BFF36F8FBFF307
S31508011CF04F8F7B6000BFFEE70A4B1B68013B094A11
S31508011D001360084B1B68002B05D100233B603B6819
S31508011D1083F3118800BF00BF0C37BD465DF8047B0D
S31508011D20704700BFD8000020000000000000000036
S31508011D30EFF30980BFF36F8F154B1A681EF0100F6A
S31508011D4008BF20ED108A20E9F04F10602DE909003F
S31508011D504FF0500080F31188BFF34F8FBFF36F8F99
S31508011D60FEF71AFD4FF0000080F3118809BC1968C7
S31508011D700868B0E8F04F1EF0100F08BFB0EC108AE3
S31508011D8080F30988BFF36F8F704700BFAFF30080F8
S31508011D90A40C002000BF00BF80B582B000AF4FF091
S31508011DA0500383F31188BFF36F8FBFF34F8F7B60A7
S31508011DB000BFFEF737FC0346002B03D0064B4FF056
S31508011DC080521A6000233B603B6883F3118800BF89
S31508011DD000BF0837BD4680BD04ED00E080B400AF02
S31508011DE00B4B00221A600B4B00221A600A4B1B6828
S31508011DF00A4AA2FB03239B09094A013B1360044BC8
S31508011E0007221A6000BFBD465DF8047B704700BF14
S31508011E1010E000E018E000E0A8000020D34D6210B1
S31508011E2014E000E0DFF80C00016841F4700101607C
S31508011E30704700BF88ED00E080B485B000AFEFF3CE
S31508011E400583FB60FB680F2B14D9174AFB681344FB
S31508011E501B78FB72154B1B78FA7A9A420AD24FF015
S31508011E60500383F31188BFF36F8FBFF34F8F7B60E6
S31508011E7000BFFEE70E4B1B6803F4E0620D4B1B68BF
S31508011E809A420AD94FF0500383F31188BFF36F8F33
S31508011E90BFF34F8F3B6000BFFEE700BF1437BD4657
S31508011EA05DF8047B704700BFF0E300E0D012002024
S31508011EB00CED00E0D412002080B58AB000AF78603E
S31508011EC00023FB61FEF7F2FA5B4B1B68002B01D17D
S31508011ED000F020F9594B1A687B681340002B40F033
S31508011EE093807B68002B1DD008227B6813447B6096
S31508011EF07B6803F00703002B14D07B6823F00703E4
S31508011F0008337B607B6803F00703002B0AD04FF088
S31508011F10500383F31188BFF36F8FBFF34F8F7B6134
S31508011F2000BFFEE77B68002B6ED0454B1B687A68BD
S31508011F309A4269D8434B3B62424B1B687B6204E079
S31508011F407B6A3B627B6A1B687B627B6A5B687A6831
S31508011F509A4203D97B6A1B68002BF1D1364B1B6861
S31508011F607A6A9A4250D03B6A1B6808221344FB617D
S31508011F707B6A1A683B6A1A607B6A5A687B68D21A56
S31508011F8008235B009A421FD97A6A7B681344BB61AE
S31508011F90BB6903F00703002B0AD04FF0500383F304
S31508011FA01188BFF36F8FBFF34F8F3B6100BFFEE709
S31508011FB07B6A5A687B68D21ABB695A607B6A7A68F7
S31508011FC05A60B86900F008F91D4B1A687B6A5B68A4
S31508011FD0D31A1B4A13601A4B1A681B4B1B689A4281
S31508011FE003D2174B1B68184A13607B6A5A68134B4E
S31508011FF01B681A437B6A5A607B6A00221A60134B74
S315080120001B680133114A1360FEF75EFAFB6903F098
S315080120100703002B0AD04FF0500383F31188BFF34F
S315080120206F8FBFF34F8FFB6000BFFEE7FB69184652
S315080120302837BD4680BD00BFE0920020F4920020FB
S31508012040E4920020D8920020E8920020EC92002029
S3150801205080B586B000AF78607B687B617B68002BB2
S315080120604DD008235B427A6913447B617B693B61E6
S315080120703B695A68244B1B681340002B0AD14FF061
S31508012080500383F31188BFF36F8FBFF34F8FFB6044
S3150801209000BFFEE73B691B68002B0AD04FF05003CF
S315080120A083F31188BFF36F8FBFF34F8FBB6000BFF8
S315080120B0FEE73B695A68144B1B681340002B1ED078
S315080120C03B691B68002B1AD13B695A680E4B1B6882
S315080120D0DB431A403B695A60FEF7E8F93B695A68DF
S315080120E00A4B1B681344094A1360386900F074F8EF
S315080120F0074B1B680133064A1360FEF7E5F900BF73
S315080121001837BD4680BD00BFF4920020E492002036
S31508012110F092002080B485B000AF4FF40043BB6055
S31508012120274BFB60FB6803F00703002B0CD0FB6809
S315080121300733FB60FB6823F00703FB60BA68FB689B
S31508012140D31A1F4A1344BB60FB687B601D4A7B6830
S3150801215013601C4B00225A607B68BA681344FB6003
S315080121600822FB689B1AFB60FB6823F00703FB60E8
S31508012170FB68154A1360144B1B6800225A60124B00
S315080121801B6800221A607B683B603B68FA68D21AB2
S315080121903B685A600C4B1A683B681A603B685B6877
S315080121A00A4A13603B685B68094A1360094B4FF09A
S315080121B000421A6000BF1437BD465DF8047B7047BC
S315080121C0D8120020D8920020E0920020E892002040
S315080121D0E4920020F492002080B485B000AF7860C4
S315080121E0284BFB6002E0FB681B68FB60FB681B6809
S315080121F07A689A42F7D8FB68BB60FB685B68BA687D
S3150801220013447A689A4208D1FB685A687B685B6806
S315080122101A44FB685A60FB687B607B68BB607B6815
S315080122205B68BA681A44FB681B689A4218D1FB684E
S315080122301A68154B1B689A420DD07B685A68FB6869
S315080122401B685B681A447B685A60FB681B681A68D6
S315080122507B681A6008E00C4B1A687B681A6003E011
S31508012260FB681A687B681A60FA687B689A4202D02A
S31508012270FB687A681A6000BF1437BD465DF8047BAF
S31508012280704700BFD8920020E0920020DFF834D0D2
S31508012290F3F736FD0C480D490D4A002302E0D458E0
S315080122A0C4500433C4188C42F9D30A4A0A4C002391
S315080122B001E013600432A242FBD300F011F8F2F7F1
S315080122C0CFFEFEE7000001200000002040010020AB
S315080122D0202B01084001002000930020FEE70000A2
S315080122E070B50D4D0D4C641BA4100026A64209D1EC
S315080122F00B4D0C4C00F0F2F8641BA4100026A64204
S3150801230005D170BD55F8043B98470136EEE755F8F7
S31508012310043B98470136F2E7102B0108102B0108F8
S31508012320102B0108142B0108704770470A44914283
S3150801233000F1FF3300D1704710B511F8014B03F8CE
S31508012340014F9142F9D110BD02440346934200D18F
S31508012350704703F8011BF9E738B50C4609680546C5
S3150801236009B1FFF7F9FF21462846BDE8384000F0D4
S3150801237069B800002C4B1B68834270B5044651D0DE
S31508012380436A43B1DB68002B4AD1636A196811B104
S31508012390204600F057F8616911B1204600F052F85D
S315080123A0616A11B1204600F04DF8A16B11B12046C2
S315080123B000F048F8E16B11B1204600F043F8216CB2
S315080123C011B1204600F03EF8E16D11B1204600F04A
S315080123D039F8A16D11B1204600F034F8616B11B1DD
S315080123E0204600F02FF8A369E3B1A36A204698476F
S315080123F0A16CB9B12046BDE87040FFF7ADBF495998
S3150801240041B90435636A802DD968F8D1204600F0B0
S3150801241019F8BAE70E68204600F014F83146EFE7D6
S315080124200025EFE770BD00BFDC0000200148FFF77B
S315080124307BBF00BFF89200200148FFF776BF00BFB7
S31508012440F892002037B5002944D051F8043C019090
S31508012450002BA1F10404B8BFE418FFF7E7FF1E4AF1
S315080124600198136833B96360146003B0BDE830405E
S31508012470FFF7E2BFA34208D9256861198B4201BF5C
S3150801248019685B6849192160EDE71A465B680BB163
S31508012490A342FAD911685518A5420BD124682144DB
S315080124A05418A3421160E0D11C685B68536021444B
S315080124B01160DAE702D90C230360D6E725686119AA
S315080124C08B4204BF19685B68636004BF49192160C0
S315080124D05460CAE703B030BDFC920020F8B500BFCE
S315080124E0F8BC08BC9E467047F8B500BFF8BC08BCE6
S30D080124F09E467047000000003A
S315080124F8494E49545F546872656164004D41494EB5
S315080125085F546872656164004D41494E5F43414EA7
S315080125185F52785F51756575650000004D41494EF2
S315080125285F4576656E745F466C61677300000000E7
S315080125384D41494E5F55706461746554696D65729C
S31508012548000000004D41494E5F5761746368646F26
S31508012558670000005045434F5F546872656164001F
S315080125685045434F5F55706461746554696D65726A
S31508012578000000005045434F5F4576656E745F4617
S315080125886C61677300000000564152485F4D7574C7
S3150801259865780000414443445F4D757465780000C9
S315080125A8414E50495F54687265616400414E50490D
S315080125B85F4576656E745F466C6167730000000057
S315080125C8414E50495F4D757465780000535049442A
S315080125D85F4144435F4D757465780000535049441B
S315080125E85F4576656E745F466C6167730000000027
S315080125F854454D505F546872656164005553464C9D
S315080126085F4D75746578000044656661756C74007C
S3150801261849444C4500000000546D72205376630006
S31508012628546D725100000000F824010800000000EA
S31508012638000000000000000000000000000400007F
S315080126482F00000000000000000000000425010812
S315080126580000000000000000000000000000000063
S31508012668000400002100000000000000000000002E
S315080126781025010800000000000000000000000005
S3150801268800000000000000002425010800000000E1
S3150801269800000000000000003825010800000000BD
S315080126A800000000000000004C2501080000000099
S315080126B800000000000000005C2501080000000079
S315080126C800000000000000000000000000040000EF
S315080126D82800000000000000000000006825010825
S315080126E80000000000000000000000007C25010829
S315080126F800000000000000000000000000000000C3
S3150801270801000000000000000100000001000000AF
S3150801271800000000000000C0000040411100000050
S3150801272800000000000000000000C8421100000077
S3150801273800000000000000000000C8421100000067
S3150801274800000000000000000000C8420100000067
S315080127580000B841000020C20000484211000000EC
S31508012768000020410000000000004041110000005F
S31508012778000000C0000000C00000000009000000B9
S3150801278800000000000070C20000C84209000000ED
S3150801279800000000000070C20000C84209000000DD
S315080127A800000000000048C200008C420900000031
S315080127B8000000000000A0C00000604109000000F8
S315080127C800000000000020C10000204109000000A7
S315080127D800000000000000000000A04009000000F9
S315080127E800000000000048C2000016430900000066
S315080127F8000000000000A0410000F04109000000A7
S3150801280800000000000000000000A04009000000C8
S315080128180000000000000000000016430800000040
S315080128280000000000000000010000000800000088
S315080128380000000000000000FFFFFFFF1100000074
S3150801284833335340020000000000804090250108F8
S315080128580300000000000000000000009C25010894
S3150801286803000000000000000000000000002041ED
S315080128780000A040000020410000A0400000000020
S31508012888000004419A996D4100000441A8250108F0
S315080128980000000000000000000000000000000021
S315080128A800040000100000000000000000000000FD
S315080128B8B42501080000000000000000000000001F
S315080128C8C8250108030000000000000000000000F8
S315080128D80004004880000000000000000000000015
S315080128E801000000000000000000000001000000CF
S315080128F800080048008000000000000000000000F1
S3150801290801000000000000000000000001000000AE
S31508012918000400480800000000000000000000004C
S31508012928010000000000000000000000010000008E
S315080129380004004810000000000000000000000024
S31508012948010000000000000000000000010000006E
S315080129580000004800800000000000000000000098
S31508012968010000000000000000000000010000004E
S3150801297800040048400000000100000000000000B3
S31508012988010000000000000001000000000000002E
S3150801299800040048200000000100000000000000B3
S315080129A8010000000000000001000000000000000E
S315080129B8000800480040000001000000000000006F
S315080129C801000000000000000000000001000000EE
S315080129D80000004800010000010000000000000096
S315080129E801000000000000000000000001000000CE
S315080129F8D4250108030000000000000000000000BB
S31508012A08E42501080000000000000000000000009D
S31508012A18F825010800000000000000000000000079
S31508012A280000000000040000180000000000000073
S31508012A380000000004260108030000000000000049
S31508012A480000000010260108000000000000000030
S31508012A580000000000000000000200001800000045
S31508012A68000000000000000000000000000000004F
S31508012A780102030406070809A0860100400D0300A0
S31508012A88801A060000350C0040420F0080841E009B
S31508012A9800093D0000127A000024F40000366E0190
S31508012AA80048E801006CDC02000000000000000094
S31508012AB800000000000000000000000000000000FF
S31508012AC800000000000000000000000000000000EF
S31508012AD800000000000000000000000000000000DF
S31508012AE800000000000000000000000000000000CF
S31508012AF800000000000000000000000000000000BF
S30D08012B080000000000000000B6
S30D08012B10B529000800000000C8
S30D08012B189129000800000000E4
S31508012B2000FF0000340200202C02002000000000F3
S31508012B300000000000000000000000000000000086
S31508012B400000000000000000000000000000000076
S31508012B500000000000000000000000000000000066
S31508012B6000000000004000000000000000E800002E
S31508012B700000000000000000000000000000000046
S31508012B8001000000010000000000000000600000D4
S31508012B9000000000E0E9000000000000000000005D
S31508012BA00100000000000000010000000100000013
S31508012BB000000000E003002000000000F8290108D9
S31508012BC0010000000200000000093D00100000009D
S31508012BD001000000000000000000000000000000E5
S31508012BE000000000010000000000000000000000D5
S31508012BF00000000020000000AAAAAAAAE0000020FE
S31508012C0000000000D02A0108F02A0108B02A0108AC
S31508012C1000000000000000000000000000000000A5
S31508012C200000000000000000000000000000000095
S31508012C300000000000000000000000000000000085
S31508012C400000000000000000000000000000000075
S31508012C500000000000000000000000000000000065
S7050801228D42
